:020000021000EC
:100000006FC04239000000000018011800280128C4
:100010000228032800290129022903290429052986
:10002000062907290829002A012A022A032A042A64
:10003000052AA62AC8CB0300341F0100F0020020C5
:1000400076030020C00200208E0200201C02002047
:100050003E210100862101002C230100C025010062
:10006000B6260100901D01004E1C0100101D01006C
:10007000A01C0100B02C01002C050020142101005F
:100080007429010002690300FA6A0300726B03001D
:10009000B41A0300E81A030040690200E85C020099
:1000A000BA620300AA2901008625030020E30100AB
:1000B000AEE3010006E401004C3501009835010073
:1000C00002340100149F0100CE990100B2A8010082
:1000D00082AC01002EB00100EA8B0100888B010088
:1000E000728F0100368C01005E8B0100E28B0100F3
:1000F000108B0100BA8C0100128D0100C28C01002E
:10010000C68C0100608D01001A8D01004C8D01002C
:100110006E92010076920100B68C0100BE8C010047
:100120005E8D0100729201000E8E0100E4930100C9
:1001300076BE0100F4BE010032BF010078A10100CB
:1001400090A10100CCA10100428501006086010060
:10015000D6860100D65301007A4E01004C7A010088
:10016000FA4E0100787501002AA70300629F030080
:1001700056A40300C0BD030086BC030016C10300E3
:10018000CEC003000EC10300BEC10300F48C030007
:100190004EC10300C8B30300EEB3030016B403005E
:1001A0002EC2030082BA030018BA03009EC20300E5
:1001B000908F03002C90030054900300F68F0300EF
:1001C000BE460300D830030050340300363203002B
:1001D000743C03006263030058620300288D03002F
:1001E0004A2E0100241C0300662503005E2603003E
:1001F00014590300A65903005A5B03007CA50100B3
:10020000964503001C3D0300A22E03000C40030092
:10021000883003003C070020FE1C03003AC10300A5
:10022000D2C003000AC1030006C103004C2501002F
:10023000CAA2010042C103009247030062480300C2
:10024000DE480300BCA403003EC1030046C1030016
:10025000745C02004AC103000A120020D011002081
:100260009CA4030042A603006446030000000000B3
:10027000000000000000000000000000000000007E
:100280006373B60082801C419105110523AEF5FE13
:10029000C5BFB7270020372700209387879B130708
:1002A00047F76373F700828023A007009107D5BF4B
:1002B0004111B7E700E022C480433707200006C69B
:1002C000798C23A0E7180F10000011C199E5B7E75A
:1002D00000E023A08710014545A893073500C20719
:1002E000C183F19BC207C183130740036366F70212
:1002F000372700200325079C372700208326879B6C
:100300006391A602372700200327C7BA69D3C20723
:10031000DD8D0545029765BF372700200325C79B64
:10032000E1BF035765002DE7035745006362F706F9
:10033000B72600203306F74021489386C6BB637872
:10034000C8028328050003D86600138687001D8F26
:100350002A9661172312E6002320160123130600B4
:1003600010C12312F500130788FF2393E60023131F
:10037000B50083D566002105B387F5402393F600C9
:10038000B7E700E023A08710B240224441018280F9
:100390000841BDB7B7E700E003A807003707200012
:1003A00023A0E7183378E8000F10000001E523A030
:1003B00007118280B727002003AE079CB7270020D3
:1003C00003A3879B8146F28763FC670A83A8070023
:1003D000636BF50A63E9A80A138787006362E50A7D
:1003E00003D66700216705076319E600372600205A
:1003F0000347C6A805072306E6A8372600201305ED
:10040000C6BB83D547000357650023930700130637
:10041000C6BB2E97420741832313E5006387C703BA
:10042000372500200325C59B6301F50203D566002F
:1004300009ED83D7460023A016012107BE95A1052B
:100440002392B6002313E600B6879843630A670237
:10045000B726002083A6C69B6304D7028356670095
:1004600085E283D64700835547001843A106AE9620
:100470002392D70098C383576600A1072313F60081
:10048000B7E700E02DB7BE86C6873DBFB7E700E0FF
:100490009843B706200023A0D718758F0F100000CF
:1004A00001C599C1814711E6B7E700E023A0E71035
:1004B0008280B386F50003C80600B306F500850701
:1004C00023800601E317F6FEC5B737E700E01C43BB
:1004D000B70620002320D718F58F0F10000019C190
:1004E00091C111E637E700E02320F71082809105E3
:1004F00003A7C5FF11057D16232EE5FEDDB737E7FF
:1005000000E01C43B70620002320D718F58F0F10FA
:10051000000001C53307C50011E637E700E02320DE
:10052000F71082800505A30FB5FEE31DE5FEF5B7C4
:10053000B7E700E09843B706200023A0D718758FCF
:100540000F1000008147B306F5008386060099E688
:10055000B7E600E023A0E6103E8582808507E5B778
:1005600037E700E01C43B70620002320D718F58F9B
:100570000F10000001C599C1014711EA37E700E0FB
:100580002320F710054582800507E309E6FE3308BE
:10059000E500B386E5000348080083C60600E305CE
:1005A000D8FE37E700E02320F7100145828037E7C7
:1005B00000E01C43B70620002320D718F58F0F104A
:1005C00000001307F6FFBA952A966317C50037E7B0
:1005D00000E02320F7108280FD1503C715000505F4
:1005E000A30FE5FEDDB737E700E01C43B7062000A8
:1005F0002320D718F58F0F10000001C53307C50061
:1006000019E637E700E02320F71001458280050551
:100610008346F5FFE397B6FEE31BE5FE37E700E010
:100620002320F7100545828079714AD037290020B0
:1006300022D40324099E06D626D24ECE52CC56CAC8
:100640005AC85EC662C44DC8372A0020B7290020A8
:10065000B72400201309099E814BB72A002037CB0D
:10066000C901130ACAB79389C9BB938404C08357CD
:10067000240099EF5C44639A0B002320F900032CBB
:10068000C4002285013B6284A9A823A6FB00C5BF44
:1006900083A74A9D82971C443307F5406375F50094
:1006A000D8401D8F2A979306FB3763EBE60623A8F5
:1006B00009008355240003450400972001E0E780EA
:1006C00040CF5C405844A9C70C44D040AE97BE868A
:1006D00063E4B70063E4C700B386C74014C4A28BC9
:1006E0003A8451F4B72700209387C7BB984B8946BB
:1006F00063FBE606791798CBB25022549254025904
:10070000F249624AD24A424BB24B224C4561828046
:1007100063950B002320E9009DB723A6EB0085B766
:1007200003274A021DCB63EDA7023385A740834709
:10073000040091EF03477A01D4405917B307A7008B
:100740003E8563E4E70063E4D7003385D74083A7A1
:1007500009016374F50023A8A900A28B404451B796
:10076000D840BA97D9B723A8070079B7B727002090
:1007700003A7879D411122C406C61384879D11C318
:100780000297B727002083C7879E93F7F70F99E357
:1007900023200400B24022444101828001114AC852
:1007A00037290020832749BE06CE22CC26CA4EC652
:1007B00052C4130949BE81C7829723200900B72478
:1007C0000020938784EA83C75700938484EA858B4B
:1007D00089CF83C7740019476317F70EA3820400FB
:1007E000EF0030708327C90082978327890091C367
:1007F0008297372400209307C4BB03C61700B7298C
:10080000002003A7899C1304C4BB9389899C834758
:10081000040093961700BA9683D60600E9C2834770
:10082000040063E6C70C83270900230004006394D7
:100830000712B727002083A7479D638E0710B727AD
:10084000002083A747C01CC8C53383C7B400639486
:10085000071083C7940081CF83C7740093F7F70F05
:1008600099E7A3840400972003E0E780E0A4B7277A
:10087000002083A707BAE5C31C48F1CF83C77400E3
:100880001547636AF70CB7270020938707EF83C7E4
:10089000C700918BE9E3B727002083C7879E93F7B2
:1008A000F70FD5EB8346140003A6090063CDD70AE2
:1008B0006244F240D2444249B249224A05611723B8
:1008C00001E06700830E83C774001D47E31FF7F044
:1008D000A3820400EF00F0608327090131B7850788
:1008E00093F7F70F2300F400E3E3C7F20DBF860789
:1008F0003E97835507002310070003450400B727E0
:10090000002083A7479E13172500372A0020BA9797
:100910009C43130A0A9D23100A00829783570A00FA
:100920000347040093C7F7FF7D8D9317170003A7B4
:1009300009003E97835707005D8D2310A70083476A
:10094000040081C785072300F400034704008347A0
:100950001400E37AF7ECF2406244D2444249B249CF
:10096000224A0561828013971700329703570700C8
:100970007DF3850725BF37C700408326C720B7070B
:10098000FCFFFD17F58F2326F72001000100B72794
:1009900000209387C7BBC84F832787262326D720ED
:1009A0006A0593C7F7FF99835D8D8280B727002082
:1009B00003A3C79E6303030002831305F00F828025
:1009C0000327851163000712411122C406C683471D
:1009D000C5008345E5042A8493F7C70F2306F50075
:1009E000834697000356C70013958601618563F11E
:1009F000C508635A05060345870093F6F607A30466
:100A0000D700054693E627006314C50093E6170058
:100A10002306D4005C4389075CC3A30AB400032502
:100A200004112E864C43090595348327841103460F
:100A30005401D44303D7C700B296118FD4C3239671
:100A4000E7008947A30DF400B7270020034764039C
:100A500083C7E7B86378F7048347C40093E70701C7
:100A60002306F40081A093E717002306F40075B76E
:100A70009376F60F635D050203458700854513E60F
:100A800027006314B50013E617002306C400A30A69
:100A9000D400A30407008547A30DF4008327841125
:100AA0009C43DDF3B240224401454101828093E73B
:100AB00017002306F400A30AD400A30407000325AB
:100AC00004114C430905D93283278411034654018C
:100AD000D44303D7C700B296118FD4C32396E7003F
:100AE0008D475DBF05458280B727002083A747ABB0
:100AF000411122C406C6858B2A84DDEB41651305AE
:100B000025F5977002E0E780E01C5DC18347A500F2
:100B10002315F50083270412B5E72320A41223220E
:100B2000A41285472311F4042320050083476401A0
:100B300054412316F5000347D4002304E50005477C
:100B4000A304E500372700200327C7EC138517020D
:100B500015811C437D151375F50F9CC25C43DCC2E7
:100B60001C479CC65C47DCC61C4B9CCA5C4BDCCA61
:100B70001C4F9CCE5C4FDCCE19CD9386060213072A
:100B80000702C1BF8327441288C38357240423224A
:100B9000A412850741BFB7270020938707D803D742
:100BA000870005072394E700B24022444101828078
:100BB0008347C40023090400054593C74700230663
:100BC000F400DDB78347850193F7E70FDDEB83473B
:100BD0009501C5EB034625018346C50009CA3727A1
:100BE0000020834565030347F7B863E7E50013F783
:100BF000060149CB014709C6C18A0357651C81C656
:100C00008356A51C36973DCFB727002003D587C054
:100C10001307C71237460F00B335A7024111130659
:100C20000624814622C426C206C67D543305A70287
:100C300097C003E0E78000A7B727002083C737B934
:100C4000B384A700B727002003A787E183270709FC
:100C500063F387003E84184375FBB727002083A702
:100C6000479D829781476364A400B307A440B240C4
:100C70002244B3B7970093C7170092443E854101C1
:100C8000828081473E858280B727002003A7C7ADB9
:100C90003C5BFDFF010001008280011122CC4AC8AB
:100CA0004EC606CE26CA52C456C25AC00347B50025
:100CB00085472A842E8983290509631AF71E8357DD
:100CC0000508035BC503372A002093060AC083DAB0
:100CD0008600130A0AC063F4671B8346050163900C
:100CE000E61A03278511631C07180327450A6318B2
:100CF00007188346F5001D476393E6180355A503BF
:100D0000330BFB409307204E3305650383244409CE
:100D100037460F008146130606243305F502B72730
:100D2000002083C727B9B3549502B3B5AA02BE9475
:100D3000C204C180231394083385AA0297C003E03C
:100D4000E7804096B307350133B5A7002E953E875F
:100D500083264A0019E163E4D7003387D740B38480
:100D60005403B7460F009387F62393860624232067
:100D7000E900A697B3D7D702DA97636CF70E1D8FF9
:100D80002320E900B729002083A7499D8324090077
:100D9000829763E1A4123385A4406350050C83A7B6
:100DA000499D372B0020130B0BC0829703270900A6
:100DB0006368E510198D8357E40303578B008E0792
:100DC000B387E7021307003293870719B3D7E70207
:100DD00063EDA70E374A0F00930AFA23130A0A2479
:100DE0008357040485072310F4048347041499E30C
:100DF00022859D2A2285976002E0E780A0E47DE1BC
:100E0000832604098327C40803274B00B6973E8531
:100E100063E4D70063E4E7003385E7408347F401E8
:100E2000835464082328A4088507A30FF40083577C
:100E30008B00B384F402D694B3D444036363950C5B
:100E4000B304954083A7499D23209900829763EEC0
:100E5000A40A3385A440E34505F8B727002083C7DB
:100E600037B963E2A708B727002023A087E201452E
:100E70009DA883264A00B387F6403E9711B7835456
:100E8000640837470F009307F723B3845403BE94D5
:100E900093070724B3D7F40263E7F900B387F94057
:100EA0002320F900C5B503274A00BA99C5BF23A07E
:100EB0003501C9BDB727002083A747C0BE94E1BD57
:100EC00083274B00998F3E95FDB5A14522859760FC
:100ED00002E0E78040D0A305A402B727002083A743
:100EE000C7BA81EF7D55F2406244D2444249B249CB
:100EF000224A924A024B05618280894515458297B4
:100F0000D5B7B3049740AA9435BF83274B00BE944E
:100F100089B731C901116C0022CC06CE2A84B53BB9
:100F200015CDFD576302F50237270020B2478345F0
:100F300037B963EFB70003459402B385B7402EC6B7
:100F4000971001E0E780E05DF24062440561828035
:100F500037270020032747C0BA97F1BF977002E0F8
:100F6000E780808AD5B78280797126D206D622D4CE
:100F70004AD04ECE52CC56CA5AC85EC68347550395
:100F800003447513AA843E941374F40F930740022C
:100F900063F687001304B4FD1374F40F03AA8413DB
:100FA00083AAC413A38B841222865285D68597B058
:100FB00003E0E780A069058915E503CBD412014958
:100FC0008149337B6403930B50024A865285D68550
:100FD00097B003E0E7808067058915C563916903D1
:100FE0001374F90F238B8412B25022549254025975
:100FF000F249624AD24A424BB24B4561828085092E
:10100000E20993D989410509E31179FDE1BF8327FD
:10101000850903560504797193D60701BD8EC20672
:10102000C182358E1357764093575640898B058B76
:101030005D8F93573640918B5D8F93571640A18BF0
:101040005D8F93171600C18B5D8F9317360093F752
:1010500007025D8F931756009355860093F7070498
:101060001E065D8F1376F60F518F93D7554013D61A
:101070003540118A898BD18F13D67540D18F13D605
:101080001540218AD18F13961500418AD18F13966E
:10109000350013760602D18F139655001376060499
:1010A0009E05D18F93F5F50FCD8FA20745465D8F35
:1010B0003307C70222D42A8426D252CC56CA032A26
:1010C0008413832AC4135AC806D63697420741832D
:1010D00093577740135557400989858BC98F13550E
:1010E00037401189C98F135517402189C98F1315AE
:1010F00017004189C98F1315370013750502C98F71
:101100001315570093558700137505041E07C98FE3
:101110001377F70FD98F13D5354013D75540118961
:10112000098B498F13D57540498F13D515402189F7
:10113000498F139515004189498F13953500137513
:101140000502498F13955500137505049E05498FB7
:1011500093F5F50F4D8F2207D98FB387C7024AD079
:101160004ECE5EC662C4B697C207C18313D777401E
:1011700013D557400989058B498F13D537401189FD
:10118000498F13D517402189498F1395170041893D
:10119000498F1395370013750502498F1395570032
:1011A00093D58700137505049E07498F93F7F70FB2
:1011B000D98F13D5354013D755401189098B498FE5
:1011C00013D57540498F13D515402189498F139543
:1011D00015004189498F1395350013750502498F14
:1011E00013955500137505049E05498F93F5F50F6A
:1011F0004D8F2207D98FB387C7021306500252853D
:10120000D685B697BD8E93940601C18033F6C4028D
:10121000137BF60F97B003E0E780404305890DED9F
:101220008347D41201498149B3849702130C5002B9
:10123000C1804A865285D68597B003E0E780004199
:101240000589937BF90F11C563863403850993F9EA
:10125000F90F0509E31F89FD230B6413B2502254D3
:1012600092540259F249624AD24A424BB24B224C42
:10127000456182805E8BCDB70111B727002022CC5B
:1012800003A487E426CA4AC84EC606CEAA84130918
:101290002500854915C083C7140003473400858B9A
:1012A0006304F700405CFDB71946930544004A8586
:1012B000EFF00FABE31835FF2285F2406244D244D1
:1012C0004249B249056182804111B727002022C4FA
:1012D00003A487E426C24AC006C693042500054934
:1012E00001E82285B24022449244024941018280B1
:1012F000A6851305A40297C002E0E780804FE302B1
:1013000025FF405CF1BF4111B727002022C403A490
:1013100087E426C24AC006C693042500054901E8B1
:101320002285B24022449244024941018280A6852E
:101330001305A40197C002E0E780A04BE30225FF5C
:10134000405CF1BF011122CC604126CA4AC84EC69A
:1013500052C406CEAA841D4A130965058549BC44BA
:101360006364F400054581A803C7D40083474400A3
:10137000631B470503C784026304F7000040C5B739
:101380000347540083C75405E31AF7FE1946CA857C
:1013900013056400EFF0CF9CE31235FF0347C40050
:1013A00083C79402E31CF7FC0357E40083D7A4022D
:1013B000E316F7FC0145F2406244D2444249B24987
:1013C000224A05618280E31BF7FA0347540083C772
:1013D0005405E315F7FA1946CA8513056400EFF0C2
:1013E0002F98E31D35F9F9B70111B727002022CC5A
:1013F00003A407E426CA06CE2AC42EC6854419E4EF
:101400000145F2406244D2440561828083479100E5
:1014100003471400858B6304F7000044CDB71946D9
:101420009305A10013052400EFF08F93E31795FEB9
:101430000545C1BFEFF08FB373000000000000004E
:1014400097120000938282810383020023800200AE
:10145000630F0300F32510342EC097050000938519
:10146000A5FD73901534EF00004A7300203086DC30
:10147000EF006049E65082800000B726002003A7F5
:1014800046AD01114AC81C5F4EC606CE998322CCD8
:1014900026CA858B138946ADB7290020ADCF9307A7
:1014A0000006372400201CDF930784EA83C7670007
:1014B00013070008930484EA6319F70083A709ADB2
:1014C0009C4393F707042383F400834784EA93F74C
:1014D000070489CFB727002083A7479D8297C8CCF0
:1014E000834784EA93F7F70B2304F4EA83C74400A5
:1014F00093F707048DE38547A382F400B727002004
:1015000083A7C7AD3707020098C7130700FC2382E3
:10151000E4009848F8D3032709001C5F9183858B6A
:1015200095C31C5F93E707011CDFB727002083A743
:10153000C7AD054723A20706B7270020938787EA90
:101540002382E70083A709ADD8430583058B19C71C
:10155000D843759BD8C3D843799BD8C3F240624423
:10156000D2444249B24905618280013F7300203074
:101570009317D50063DF0700B727002083A7C7AD07
:101580007D57B8D7B72700209387C7BBD84F05072B
:10159000D8CF9377850085CBB7270020938787EA3C
:1015A00003C72700136717002381E700130700F81C
:1015B0002382E700B727002003A747AD5C57F19BC4
:1015C00093E717005CD79377150085C7B7270020EE
:1015D000938787EA03C7170013671700A380E70004
:1015E000B727002003A747AD5C57F19B93E717008F
:1015F0005CD7937765009DC7B72700201377450018
:10160000938787EA59CF03C7070013671700238022
:10161000E700B727002003A747AD5C57F19B93E78E
:1016200017005CD79317F50063D20702B727002095
:10163000138707D883468707938707D8C18AADCA1F
:101640008347870793E70702230CF7069317E50004
:1016500063D60702B7270020938787EA03C74700AE
:10166000620761876355070005472382E700B727B4
:10167000002083A7C7AD3707020098C79317C5009E
:1016800063D00702B7270020938707D803C79707BF
:10169000058B1DCF03C7970713672700A38CE706A9
:1016A000828003C7370013671700A381E70095B74F
:1016B00003C7870789463D8B6308D70003C78707A1
:1016C0008D463D8BE314D7F81147238CE706BDBF49
:1016D00003C79707118B69D703C79707136787005D
:1016E00075BFB727002083A6C7ADB7270020938713
:1016F00087EA03C70700058B11C723820700A3826F
:101700000700828003C71700058B65FBF85275F34D
:1017100003C75700EDB737270020032847AD8327BD
:1017200088039583858BC1E311C683270803BD8396
:101730002300F60085CA832747AD985B4607935779
:1017400067016356070093E707C0C207C183039789
:101750000600C207C18709C7BA970947B3C7E7029E
:101760002390F6009DCD8345150085CDB727002039
:10177000938787EA83C7670013879500894593F7A6
:10178000070485C33A95834705000547994593F6B5
:10179000F7066398E600E207E187814563D3070017
:1017A000B9452E8582808545EDBF411126C206C60A
:1017B00022C44AC0B724002035ED83A6C4ADAE874D
:1017C000F8527DFF37290020130989EA2301090017
:1017D00037F400E03E85832704D1B285ED9B2328B2
:1017E000F4D0832704D193E787022328F4D0730031
:1017F0005010971003E0E7800094B727002083A7DC
:1018000047ADB70680009843558F98C3D857719B52
:10181000D8D783A7C4ADA3020900A30009000947D4
:1018200098C3832704D193E787002328F4D073005B
:10183000501005A08D476314F504B727002083A737
:1018400047ADB70680009843558F98C3D857719B12
:10185000D8D783A6C4ADB7270020938787EA03C7EC
:101860002700058B19E703C73700058B51CB23826F
:101870000700B240224492440249410182808547D8
:10188000E319F5FCB7F700E003A707D16D9B23A888
:10189000E7D003A707D11367870223A8E7D0730017
:1018A000501003A7C4AD8177FD175447F58F5CC76F
:1018B0000F10000003A7C4ADB7070200130600F81D
:1018C0001CC7B7270020938787EA2382C700B72762
:1018D000002083A747AD9C439D83858B639FA70012
:1018E000930760197CD354C737F700E0832707D1EB
:1018F00093E787002328F7D01DBF9307E01BDDB7D0
:10190000F85231FFBDB7B727002083A7C7AD88477E
:10191000D847798D09C988C7B727002003A307AE28
:10192000630303000283828037270020B72600204C
:10193000138606ED130707EF8347D7008345B601EB
:10194000484AAE97FD8BB355F500A300F600A306F9
:10195000F700858995E903471701814613080002BE
:10196000B3F7E7020147B355E50085899378F70F90
:1019700089C96395D700A30016018280850693F676
:10198000F60F0507E31107FF8280B7270020938732
:1019900087EA83C7570093F7F70FD1EBB7270020EB
:1019A00083A7479D411122C44AC006C626C282971A
:1019B00037290020930709EF8047130909EF6302D5
:1019C000A40663688504018DB7240020938704ED85
:1019D00083C7A70113545500938404ED6363F40493
:1019E000A13783C7A4010327890093965700369730
:1019F0001D8C2324E900E375F4FE224403C5140082
:101A0000B2409244024981454101171303E0670047
:101A10004308B727002083A747C033848740229517
:101A200065B7B240224492440249410182808280DB
:101A3000B727002083A7479D011122CC26CA52C494
:101A400006CE4AC84EC68297B7240020938704EF7B
:101A50008047014A6301A406938404EF6366850608
:101A6000018D37270020930707ED83C7A701135483
:101A70005500137AF501130907ED636BF402B729DA
:101A80000020938909C04D358346A90103A884002D
:101A900083A54900139756004297158C3A866364D4
:101AA00007016364B7003306B74090C4E37DD4FCFC
:101AB0001604336A4401F24062445285D2444249DA
:101AC000B249224A05618280B727002083A747C018
:101AD00033848740229571B7B727002003A7C7AD8D
:101AE0008967938707F47CD3B727002083A787AE45
:101AF00083A60709139656006358060083A60709B4
:101B000013966600634406007453FDF28280000061
:101B1000B72700203727002083A7079C0327879B30
:101B200001456313F700828083D6670081E683D680
:101B3000470036959C43F5B7B727002083A5C7B764
:101B4000372700209387C7B7138605222320C79C19
:101B500003D74700938785FFB72600204111BA9726
:101B6000056523ACF69A06C61D05935637006374C7
:101B7000E500930600203307D60037250020232EEA
:101B8000E59A23A0E522E1162312D60023130600CE
:101B90001CC3998FE1172312F700231307008D3F11
:101BA000B240B72700202391A7BC41018280B7270C
:101BB00000203727002083A7079C8326879B0145A9
:101BC0006393F600828003D7670011E703D74700CD
:101BD0006373E5003A859C43E5B7B7270020B72635
:101BE000002083A7079C03A6869B2A87B305B540E0
:101BF0006314F6003A8529A8938687009C43E3691D
:101C0000D7FEE377F7FE2E85E3E4D5FEE3F2F5FE9B
:101C1000828023AC05FE1C4191E7010001000CC14C
:101C20008280BA8703A787FF6DFF23ACB7FE82804F
:101C3000184183A785FF6319B7001CC1FD5723AC6A
:101C400005FE238FF5FE8280232CF6FEC5BF4111D1
:101C500022C437E400E026C204403707200006C64D
:101C6000F98C2320E4180F10000009E923209410B8
:101C70001545B24022449244410182800347E5FF6A
:101C80009307F00F6306F700232094101145D5B792
:101C900097E0FE1FE7804049014523209410D1BF03
:101CA000411126C2B7E400E04AC003A90400B70707
:101CB000200006C622C43379F90023A0F4180F10BF
:101CC000000009E923A02411B240224492440249B1
:101CD000410182809565938505D0C98D2A842105AF
:101CE000C2054205C181418197E0FE1FE780803532
:101CF00001CDFD5723200500231285002303F500A5
:101D000023A024112105C9B723A0241101456DBFCB
:101D10000111B7E700E04AC803A907004EC637071C
:101D2000200006CE22CC26CAAA893379E90023A056
:101D3000E7180F100000372500200324459C81443C
:101D4000014619E499E8A1654E85EF00700731A8B6
:101D50008347E4FF6397370395C8A6851305459C21
:101D6000C13D75D0A1654E85D92EF2406244B7E7DA
:101D700000E023A0271126854249D244B2490561DB
:101D8000828091E02286032484FF65BFA284E5BFA0
:101D900041114AC037E900E022C403240900370793
:101DA000200006C626C2798C2320E9180F100000F7
:101DB00089E523208910154515A0B727002083C782
:101DC000D7BBAA842E8563F5F400894763EE97009C
:101DD000BD3DB7E700E023A087100D45B240224487
:101DE000924402494101828083A785FF99E703C796
:101DF000E5FF9307F00F6308F700913DB7E700E0B8
:101E000023A087104DBF37250020238F95FE130593
:101E1000459C0135A16526851D2601452320891095
:101E200075BFB727002023A2079C8280B727002018
:101E300083A7079E99E33E85828003D72700631618
:101E4000B70003C70700E308A7FEDC47E5B7B9CD35
:101E5000011106CE22CC26CA8147C14633D7F540B0
:101E6000058B21C312053E9531473305E50237271F
:101E700000208324C79C05443314F4002EC642047A
:101E80004180AA949C40C8408297B24523A0040098
:101E900023A20400A18DF2406244D2442E85056144
:101EA00082808507E39CD7FA0144EDB72E858280B6
:101EB000C1C1797122D406D626D24AD04ECE014471
:101EC0004147B3D78540858BB9CF1205314722955D
:101ED0003305E502B727002003A9C79C8544B394C6
:101EE0008400C204C1809389C79C2A9903270900F2
:101EF00011C7032549002EC60297B2453147330466
:101F0000E40283A709003E941C4489E723200900CA
:101F100023220900B2502254A58D02599254F2494D
:101F20002E85456182800504E31DE4F88144DDB718
:101F30002E8582804111B7E700E026C2844337072F
:101F4000200006C622C4F98C23A0E7180F10000059
:101F5000B727002083A7C7B937240020130484982B
:101F600091C782971C403E9508C031A0B72700203A
:101F700083A7479DFDF70840B74703009387D73FE6
:101F80003305F502B7A72600938737ECB2403E959C
:101F900008C02244B7E700E023A097109244410113
:101FA00082800111B7E700E022CC80434AC837079E
:101FB000200006CE26CA2A892E86798C23A0E7180F
:101FC0000F100000131506019305F004418132C67D
:101FD00097E0FE1FE7800007AA8419C53246CA852C
:101FE00097E0FE1FE780C023B7E700E023A087103B
:101FF000F240624426854249D2440561828079716B
:10200000B7E700E022D480433708200006D626D266
:102010004AD04ECE52CC56CA5AC85EC662C4337439
:10202000040123A007190F10000005E123A0871069
:102030000945B250225492540259F249624AD24A96
:10204000424BB24B224C45618280B727002083A7C8
:10205000479DBA8A368AB28B2E8BAA898297B72778
:10206000002003A7C79C1389C79C8144B146C14780
:10207000338CD40233068701104241E6C165938553
:1020800005F0414597E0FE1FE780C0FB19EDB7273B
:10209000002083A7C7BA81C7814511458297B7E75A
:1020A00000E023A087102D4569B7B726002093864E
:1020B000069E984239E388C2230005008327090061
:1020C00005473317970023260500232475012311A4
:1020D000E50023225501E29723A0370123A26701DF
:1020E00023A4570163040A0023009A00B7E700E025
:1020F00023A08710014535BF3E875C47F5FF48C7E1
:1021000065BF8504E396F4F6B7E700E023A08710E7
:10211000214505B7B727002083A7C79D411122C4D9
:1021200006C6372400201304C4BB89C782975C48C5
:102130003E9548C84848B240224441018280B7E7F2
:1021400000E09843B706200023A0D718758F0F1022
:102150000000B726002083C6D6BB6372D50237269F
:102160000020931615000325869C3695835605009E
:10217000D58D2310B50023A0E7100145828023A050
:10218000E7100D458280B7E700E09843B7062000CE
:1021900023A0D718758F0F100000B726002083C624
:1021A000D6BB6374D502372600209316150003258D
:1021B000869C93C5F5FF369583560500F58D231053
:1021C000B50023A0E7100145828023A0E7100D454C
:1021D0008280011137E700E026CA0443B7062000D9
:1021E00006CE22CC4AC84EC652C4F58C2320D7183E
:1021F0000F100000130705FF1377F70FFD4763E289
:10220000E70AB146B306D502B727002003A7C79C4B
:1022100036971C43D9C71359450005443D893315EA
:10222000A400131405014180AE894A85A285FD3EB4
:102230002A8A39C9A2854A85B937B727002083A7DA
:10224000479D37290020130909C0829783578900C9
:102250002A848146B385370313060064B3B7370376
:1022600013850532B335B500BE95EFA0621CB307E8
:1022700085003E878326490063E4A70063E4D70016
:102280003387D7402324EA00B7E700E023A0971064
:102290000145F2406244D2444249B249224A0561B2
:1022A0008280B7E700E023A097100945DDB7011150
:1022B000B7E700E026CA84433707200006CE22CCC9
:1022C0004AC84EC6F98C23A0E7180F100000BD477E
:1022D00063E8A70431473307E502B727002083A747
:1022E000C79CBA979C438DCF05443314A400420485
:1022F00041802E890145A285153EAA8911C5A28576
:102300000145513523A42901B7E700E023A0971028
:102310000145F2406244D2444249B249056182809B
:10232000B7E700E023A097100945E5B779714AD0D7
:1023300037E900E026D283240900B707200006D63B
:1023400022D44ECE52CC56CA5AC85EC6FD8C23202B
:10235000F9180F100000B727002083C7D7BB637898
:10236000F500B727002083AB479D63970B00B7E7C5
:1023700000E023A0971099A0B7290020938909C0F5
:10238000AE8A03AB490083D58900B74736FE9387F1
:1023900007C83E9BB387C5022A84328A8146B3B5FB
:1023A000C50213850732B337F50013060064BE95E6
:1023B000EFA002086370AB02232099100145B250D0
:1023C000225492540259F249624AD24A424BB24BC9
:1023D00045618280829B83D589002A891306006427
:1023E000B38745038146B3B5450313850732B33739
:1023F000F500BE95EFA0C203B30725013E8903A7F0
:10240000490063E4A70063E4E7003389E740D68529
:102410002285293C09C923242501B7E700E023A030
:102420009710054569BF936504F0C205C181414518
:1024300097E0FE1FE78000C111E9B727002083A7BE
:10244000C7BA95D7A2851145829715B737270020BF
:102450001307079E1C438DE308C385472326050009
:10246000232425012311550123008500A300F50035
:10247000232205005DB7BA87D84775FFC8C7F1BFEB
:102480003971B7E700E026DA84433707200006DE1B
:1024900022DC4AD84ED652D456D25AD05ECE62CC26
:1024A00066CA6AC86EC6F98C23A0E7180F10000030
:1024B0003DC14144B689B28A2E8A2A89B14C372D52
:1024C0000020854D130C0003330B9403930BCD9C1C
:1024D00003A70B005A971C43ADE39375F400B39523
:1024E000BD0013554440C2055686C1811375F50FD2
:1024F000353D21C583A70B00DA9723A0270123A22E
:1025000047016384090023808900B7E700E023A026
:102510009710014521A023A097100945F25062545D
:10252000D2544259B259225A925A025BF24B624C2F
:10253000D24C424DB24D216182800504E31684F9EC
:10254000B7E700E023A097102145C9BF0111B7E705
:1025500000E026CA844322CC4AC84EC63707200072
:1025600006CE2A84AE893289F98C23A0E7180F1091
:1025700000006D3B2285CE8555382A8405C5B727D6
:10258000002083D587C0130600648146B3872503E6
:10259000B3B5250313850732B337F500BE95EF9029
:1025A000326948C013351400F2406244B7E700E0D6
:1025B00023A097104249D244B2490E05056182809A
:1025C0000111B7E700E04AC803A9070022CC4EC6B4
:1025D0003707200006CE26CAAA892E843379E9005F
:1025E00023A0E7180F100000EFF05F84AA8419C140
:1025F00023110500A2854E857936B727002083C7B1
:10260000C7BB639B3701B72700209387079D03D77C
:102610000700598C23908700B7E700E023A027111B
:10262000014591E01945F2406244D2444249B24921
:102630000561828001114EC6B7E900E022CC03A4F7
:102640000900B707200006CE26CA4AC87D8C23A001
:10265000F9180F1000009307F00263E8A704B147D0
:10266000B304F502372900201309C99C8327090008
:10267000A6979C439DCB9377F5008545B395F500D0
:10268000C205C18111812D3F832709000145A6970D
:1026900023A0070023A2070023A08910F240624470
:1026A000D2444249B24905618280B7E700E023A0E5
:1026B00087100945E5B74111B7E700E026C284431A
:1026C00006C622C437072000F98C23A0E7180F1094
:1026D0000000EFF0AFF519E90145B2402244B7E739
:1026E00000E023A09710924441018280B727002088
:1026F00083A7479D00458297B7270020938707C08F
:102700006368A402D843B74636FE938606C83305ED
:10271000A4403697E372E5FC13070064B335E50285
:1027200003D6870081463305E502EF90725075B7F6
:10273000D8433A94C1BF411122C426C23724002095
:10274000B7240020130704C09384C4BB94485843A3
:10275000B727002006C683A7479D130404C06392D1
:10276000E60882975440B74736FE938707C8B69766
:102770003387A7003A856364F7006364D7003305A5
:10278000D740B7240020938784EADC53938484EAFB
:1027900099CBB727002083A687AE3707CDFF7D17DB
:1027A0009C46F98F9CC611E14840B727002083A7BB
:1027B00007BA829719E5DC5085C3EF002201EFF0DC
:1027C0008147DC5091CBB727002003A787AEB7061F
:1027D00033001C47D58F1CC7B240224492444101AC
:1027E0008280829794485840B387A6003E8563E470
:1027F000D700E3E8E7F83385E74061B74111B72731
:10280000002006C623AEA79C0295B240B727002041
:1028100023AAA7BC014541018280994763EAB7001A
:1028200093972500B7250020938545BEBE9588C1A6
:102830008280B727002023ACA79C11C5B7270020B2
:1028400005472384E79E8280B727002023A0079EA8
:10285000B727002023AE079CB727002023AA079C98
:1028600037250020B727002041112384079E714699
:10287000B72700208145130545BE06C623AC079C3B
:1028800022C426C297E0FE1FE780A0A037250020C3
:102890001306800281451304C5BB1305C5BB97E031
:1028A000FE1FE780009FEFF02FA9B7270020938736
:1028B000C7B703C5C70383C7D7038545B72400201F
:1028C0003E958D473305F50299479384C49C39059D
:1028D0001375F50F2301A4003305F5021305052434
:1028E00097D0FE1FE780007688C041C103462400D0
:1028F000994781453306F6021306062497E0FE1F2A
:10290000E78020999C4003472400B7240020938748
:1029100007249384449E0A079CC0BA973727002057
:102920002324F79CEFF0EFCFAD29834714009440A8
:1029300037260100139727003697130606EB10C3BE
:10294000138717001377F70F0A073726010036970A
:102950001306E6E410C313873700890793F7F70FD0
:102960008A07A300E400B69790C3B2402244924481
:1029700041018280372700201307C7BB8347170018
:102980008346270063F0D702B726002083A6469E21
:1029900013861700A300C70013972700369708C3B4
:1029A0003E8582809307F00FE5BF1C4163800712CC
:1029B00041777D8FB70600208947631AD7100357E8
:1029C000450063060710411126C21946AA849305E3
:1029D000F00F610506C622C44AC097E0FE1FE780DB
:1029E000C09905478D47630CE50C9C4491C7D858A6
:1029F000994771C7985C61C737240020130600040B
:102A000081451305C4B797E0FE1FE7808088130651
:102A10000004A6851305C4B797E0FE1FE780408039
:102A20001309C4B70357C9009307C4B709E71307CD
:102A300000102396E70003C7E70001E70547238757
:102A4000E70003D7070101E76D472398E70003C7B5
:102A5000F70001E71547A387E70003C7270101E750
:102A600005472389E70003C7370109E703C7F700D4
:102A7000A389E70003C7570101CB93763700098389
:102A8000238ED702A38EE70203C7470101E755470C
:102A9000238AE70003C7640109E71307C003238BF8
:102AA000E7009C5791C78297B72700202392A7BCC5
:102AB000B72700207D57A385E7B679338147B24019
:102AC0002244924402493E854101828089473E85E5
:102AD000828001114AC837290020130909C08327C1
:102AE000090006CE22CC26CA52C456C24EC68297D0
:102AF000130A0064B3354503835A8900814656861C
:102B000033054503EF90D212B72700201387C7BBC8
:102B1000004FAA840145630694029389C7BB33859D
:102B20008440636E94000325490056868146B33580
:102B3000AA023305AA02EF90B20F018D269523ACAD
:102B40009900F2406244D2444249B249224A924A30
:102B500005618280011122CC2E84B7D503000A853D
:102B600041469385058806CEEF9012461808060464
:102B70003A94B7270020035504FF83D7A7C0F2403B
:102B80006244AA9737450F00130505243355F50213
:102B900005618280B727002083D7A7C051471D4514
:102BA000637CF702794719456378F702130720031E
:102BB00015456373F7021307B0041145637EF700F0
:102BC000130740060D456379F700130760090945AF
:102BD0006374F70013B5B70F8280011122CC06CEC3
:102BE0002A842EC6EFF00FB5B245F240818D33A591
:102BF000A502229562441375F50F056182800111CB
:102C000022CC06CE2A842EC6EFF0CFB2B245F240D7
:102C1000818D33A5A502229562444205418105615B
:102C20008280011122CC06CE2A842EC6EFF08FB00E
:102C3000B245F240818D33B5A5022295624405610B
:102C40008280B72700201387C7B718572DC34111BB
:102C500022C426C24AC006C61389C7B70297B7273F
:102C600000201387C7BB035787002A849384C7BB00
:102C70000DCBBA876373A700AA87C207C183BA8640
:102C80006373E400A286C206C182958F5147635ADE
:102C9000F7008327C90291C38297EFF0511C239458
:102CA0008400B240224492440249410182808280E1
:102CB0000111B727002022CC3724002023A6079E2D
:102CC0009307C4B7DC5706CE26CAAA851304C4B737
:102CD00081C72AC68297B245C1C99C410545C1C377
:102CE000DC41B5CF83D78500BDCB83D7A500A5CB6D
:102CF00037250020930405C05146130505C097D021
:102D0000FE1FE780E05123860400B7270020938749
:102D100007C0944337270020232AD79C0347740118
:102D20000DE303D587009307805737460F0033051F
:102D3000F5021306062481468145EF90626FA30BCE
:102D4000A40003477401A54763E5E700A947A30B67
:102D5000F40037350100130525AD4D340145F2402F
:102D60006244D24405618280B72700209387C7BBA5
:102D700023AE070037070020B7270020938707C03E
:102D80001307677098C337873200FD56130727A1D2
:102D9000D4C398C723860700B7C7004023A4D7260B
:102DA000ADB7011122CC372400209307C4B7884760
:102DB00006CE26CA4AC801E90545F2406244D2441B
:102DC0004249056182801304C4B75C58F5D7185C8A
:102DD00065D77000854582971844B247E30EF7FC2B
:102DE0000355C4009305E004B724002097D0FE1FCC
:102DF000E78040251387C4BB08D39384C4BB4DDD53
:102E00000356C4009305F00F014997D0FE1FE780D9
:102E100040488347E4009050634DF900328597D0D5
:102E2000FE1FE7806030014523A0040223A20402B4
:102E300069B78355C4000844185CB38725038981AA
:102E400005093E9508C20297E9B701114EC6B72998
:102E500000209387C9B79C4726CA4AC852C406CEE9
:102E600022CC56C25AC02A8AAE843289638D071E8C
:102E70009389C9B703A74903630407121307F01F17
:102E80006362A712372400201307C4BB832A0702FA
:102E90001304C4BB639A0A0803D5C90095659385DA
:102EA00015E097D0FE1FE780E01908D02A866DC98B
:102EB00083D5C90083A7490303A589008981829727
:102EC00083A78900832A04025CD089476316FA0825
:102ED000C1476397F40C83D5C9009147938505FCDE
:102EE000B3C5F5028A05D69503C725009307A0054B
:102EF0006314F70A83D705006390470B4A8526863B
:102F0000910597D0FE1FE780A0311C505685639332
:102F100057130145F2406244D2444249B249224A21
:102F2000924A024B056182805850E380E7FA03D54C
:102F3000C9009565938525E097D0FE1FE780801036
:102F4000AA8A39CD83D5C9002A8683A7490303A558
:102F500089008981829795BF8D47631BFA00C1471D
:102F60006390F40483D5C900938545FDF199A5BF0D
:102F700091476318FA006395440383D5C900A115EE
:102F8000F5B793070010631DFA00A14763EA9700A5
:102F900083D5C900C115D9BF1C5056856390570D04
:102FA00029458DBF9D6A637C5509930A05E0194741
:102FB000B3CAEA0203D7C900372B0020B38AEA025A
:102FC000BE9A9307CBBBDC53130BCBBB6395570166
:102FD00003240B021DE003D5C9009305E00497D03C
:102FE000FE1FE78020062A8445DD83D5C90083A71C
:102FF00049032A8689815685829791451307A00542
:10300000898193972500A29783C627006393E604DE
:1030100083D60700639C460385058A052686A2950C
:103020004A8597D0FE1FE780A01F83270B02E3820B
:1030300087EE228597D0FE1FE780000FD9BD21675C
:103040007917E36FA7F4B30A5541ADB783C53700CD
:1030500045BF83270B02E38587F4228597D0FE1FA7
:10306000E780800C35BFB727002083A5C7BD8DD969
:1030700091479306A0058983139727002E9703464F
:103080002700E31FD6F003560700631C460185079F
:103090008A072686BE954A8597D0FE1FE78040188E
:1030A0008DBD83473700C1BFB72700209387C7B7BF
:1030B000984729C3985F1DCF8546631DD5024111EE
:1030C00022C4372400201304C4BB105006C619CEF6
:1030D00083D5C700485089810297085097D0FE1FBA
:1030E000E78080042320040223220402B240224409
:1030F000410182808280011122CC37240020930775
:10310000C4B756C283AA870026CA4AC84EC606CE8E
:1031100052C42A89AE84B2891304C4B7638C0A1CD2
:103120001C5C99EB2945F2406244D2444249B249C1
:10313000224A924A056182805C58EDD79307F01FBE
:1031400063E8A70C372A00209307CABB9C53130AD5
:10315000CABBB9C7084483274A02639FA7048947AB
:103160006317F906C147E39FF4FA0355C40091477A
:10317000130505FC3345F5029317250003250A02C4
:103180002686CE853E959307A0052301F5002310E2
:103190002501110597D0FE1FE7808008014561B722
:1031A0000355C4009305E00497D0FE1FE78080E933
:1031B0002320AA0245F1BDB78355C4005C580326FD
:1031C0000A02898182971C442322FA0249BF8D4753
:1031D000631CF900C147E397F4F40355C4001305D9
:1031E00045FD9377C5FF59BF91476318F900E39BED
:1031F00024F30355C4002115EDB793070010E31322
:10320000F9F2A147E3E097F20355C4004115D1BF9D
:103210009D676378F506930705E01947B3C7E70292
:103220000357C400372A0020B387E702BE9A9307EA
:10323000CABB9C53130ACABBA1CF83274A0263951A
:10324000570703250A0291461308A0059305F00FBE
:1032500093D72600139727002A9703462700631663
:1032600006078358070003463700639C2805B3060A
:10327000D64063C6960485078A072686CE853E9586
:1032800011BF21677917E36FA7E8B307F54049BF7E
:103290000355C4009305E00497D0FE1FE78080DA51
:1032A0002320AA0259F9BDBD8355C4005C580326EA
:1032B0000A0289815685829723225A0359B723101F
:1032C000B70093160601C18261B70356C400B385E7
:1032D00096009105130606FCE366B6E413863400F7
:1032E000719A1106B2962301070123102701A30149
:1032F000D70051B7372A00209307CABB9C53130A43
:10330000CABBA9C303250A0291461308A005930569
:10331000F00F93D72600139727002A97034627001C
:103320006314060583580700034637006398280195
:10333000B306D640E3D196F42310B70093160601E6
:10334000C182C1BF0345E4008357C4009305E00474
:103350003305F5024205418197D0FE1FE78080CEFC
:103360002320AA0245F17DBB0356C4008345E40037
:10337000B385C502338696001106E3E5C5DAB9BF09
:103380000145828083C705002300F50083D725000F
:10339000A300F50083D72500A1832301F50083C78F
:1033A0004500A301F50011458280B727002023AA1C
:1033B000079EB727002023A8079E828029C14111BC
:1033C00026C206C622C4AA8401458DC52E84B7D55F
:1033D0000300228541469385058997D0FE1FE7802B
:1033E00020E483C7040005452306F40083C71400C6
:1033F000A306F400B2402244924441018280014578
:103400008280011122CC26CA06CE0947AA843284C2
:103410006381E50441468147639BC500638FE600F5
:103420006397B6000DA841478147638EE600F240DE
:103430006244D2443E85056182808A852285BD3FF3
:1034400041468A8519A88A85953F41468A85228505
:1034500031A0E39AB6FC2E86A285268597D0FE1F62
:10346000E78040E9AA87E1B7B727002023A8A79EF5
:103470008280B727002023AAA79E8280011122CC38
:103480000354650006CE26CA4AC84EC641C08329E9
:103490008500AE842A8803C9090081471317890172
:1034A000618763550702B147054563FA87045114E4
:1034B000420403552800418033878900A2864E8646
:1034C0008545EFC0E009B337A00085077D1413558B
:1034D0006900420405891379F90341802380F400CF
:1034E000A380A4002381240123928400014719C0F2
:1034F0001387190098C409476383E7000145F24028
:103500006244D2444249B249056182800545C5BF43
:10351000C167F917630AF502D94763F7B7020111CA
:1035200022CC2EC606CE2A84EF90C043B2456368F3
:10353000B50022856244F24005616FA0506AF240F6
:10354000624405450561828005458280C167F9179F
:103550006314F5006F900041411106C6EFA0F056CC
:1035600011E15D45B2404101828091476394F502CB
:10357000834705002300F600834725000347150015
:10358000A207D98F2311F600834735000145230296
:10359000F6008280114582804111814522C426C2F5
:1035A00006C6AA8405252A8409E9B727002083A72F
:1035B000079F81C7F945268582972285B24022441C
:1035C00092444101828039714ED656D25AD006DEDD
:1035D00022DC26DA4AD852D4AA8A2E8BB28941EF4D
:1035E00036C6AD379145EF90A049AA844D492DC903
:1035F000B246054A238034010544630A0B00B685B0
:1036000013851400029B0505131405014180E2098E
:1036100093D9894163D30902C1455685EFA030593A
:10362000654905E933868400A2852685EFB05038C8
:103630002A8905E131044204418091472C085685CE
:10364000231CF10026CE231D8100EFA0E05E2A8915
:1036500001C963070A00268597D0FE1FE780C0AC2A
:10366000F25062544A85D2544259B259225A925A5F
:10367000025B21618280BA84014AADBF011122CC74
:1036800026CA4AC84EC606CE2A893284B689253F44
:10369000AA840DE1B727002083A7479F81CF054764
:1036A0006317E40003C4090005041374F40FA28532
:1036B0004A858297F240624426854249D244B24903
:1036C00005618280AE86B7350100014705469385C6
:1036D00045386DB783D705002300F50083D7050073
:1036E000A183A300F5000945828083D7050023004C
:1036F000F50083D70500A183A300F50083D725003B
:103700002301F50083D72500A183A301F50011450E
:10371000828083D705002300F50083D70500A183AD
:10372000A300F50083D725002301F50083D72500EA
:10373000A183A301F50083C755002302F50083C7C9
:103740006500A302F50003D58500190542054181F6
:10375000828083D705002300F50083D70500A1836D
:10376000A300F5000945828083D705002300F500FA
:1037700083D70500A183A300F50083D7250023018B
:10378000F50083D72500A183A301F50011458280B0
:1037900003D54500060542054181828083D7050097
:1037A0002300F50083D70500A183A300F50003D50E
:1037B0002500090542054181828083D70500230049
:1037C000F50083D70500A183A300F50083D725006A
:1037D0002301F50083D72500A183A301F50003D5BC
:1037E0004500110542054181828083C70500230001
:1037F000F5000545828083D70500411122C406C625
:103800002300F50083D705002E841105A183A30EA4
:10381000F5FE83D725009505230FF5FE83D7D5FF49
:10382000A183A30FF5FE03C6F5FF97D0FE1FE78027
:10383000209F03454400B24022441105410182808B
:103840008947639CF5008347150003470500014540
:10385000A207D98F2310F60082801145828003D7FA
:103860000500D94763FEE702011122CC06CE2EC621
:103870002A84EF90200FB24683D70600636DF500CF
:1038800022856244F240B73501000147094693851D
:10389000456D05610DBBF2406244094505618280BA
:1038A0000945828091479DC583460500FD15C205E7
:1038B0008547C1816392F60213D725008D89914710
:1038C00091E9914701CB05052301D6002310E600BD
:1038D00048C281473E85828009479147E39CE6FEC6
:1038E000C94733D7F502B3F5F502D1BFAE86B73578
:1038F0000100014711469385A56EF1B193F735009C
:1039000091EB8981914789C52310B60048C2814750
:103910003E8582809147EDBF03C745008947631A02
:10392000F702011122CC2A84C84506CEAE86014793
:1039300019C52EC69D45EFE04FAAB2462A872285BB
:103940006244F240B735010019469385257105613F
:103950009DB90945828099E1114582808347050020
:1039600005472311F600E379F7FEFD1593F5F50FF2
:1039700033D7F502B387E702E390F5FE050548C2A9
:103980002310E6000145828083C745000947AE86C3
:103990006385E70041476399E700B73501000147B8
:1039A00021469385657F05B1094582802310B600C5
:1039B00091E1014548C201458280AE86B7350100DC
:1039C0000147294693852575FDBE2310B60091E178
:1039D000014548C201458280AE86B73501000147E6
:1039E000314693858576C5B62310B60091E1014531
:1039F00048C20145828003D74500854763FDE70241
:103A0000011122CC2A84884106CE0DC12EC68545DF
:103A1000EFE0AF9C2A8722856244B246F240B73578
:103A20000100394693850579056171BEF240624413
:103A30000945056182800945828091479DC50347FC
:103A400005008D46914763F2E602FD15C205C1816E
:103A5000B3C6E5023308D7026399050105052310B3
:103A6000D6002311E60048C281473E85828083C785
:103A700045000947AE866385E70041476399E70043
:103A8000B7350100014741469385657F2DBE094545
:103A90008280B335B000139525008280011122CCBD
:103AA00026CA06CE03C785008547AA842E844946C8
:103AB0006310F702613C835724004915130620095F
:103AC00063C8A700F2406244D24409450561828080
:103AD0000347940085476314F700136606044840C3
:103AE00011C58D4532C6EFE04F8F3246A286624443
:103AF000F2402A872685D244B73501009385C579DF
:103B00000561D1B48D4763FFB702834715000347B2
:103B10000500F115A207D98F2310F6008347350061
:103B200003472500C205A207C181D98F2311F600E2
:103B30002312B60089C5110508C6014582802324D9
:103B40000600E5BF11458280011122CC2A848845F8
:103B500006CEAE8611C52EC69545EFE00F88B2465B
:103B60002A8722856244F240B73501005946938581
:103B7000A57B056189BCB335B00013952500828013
:103B8000AE86B7350100014761469385A57E25BC09
:103B90008547114563F4D702834716008345060025
:103BA000A207CD8F2310F7009387E6FF2311F700BC
:103BB00089476386F600090650C3014582802322A7
:103BC0000700E5BF0147814679468145EDBA83D7B5
:103BD00005002300F50083D70500A183A300F500AD
:103BE0000945828083C7250005472300F50003D5DA
:103BF00005006397E7000A050505420541818280BB
:103C0000C9473305F502CDBF03D505000A054205B6
:103C10004181828083D725002300F50003D505006C
:103C200083D725003305F5020505420541818280D1
:103C300003D50500828003D50500828003D50500E9
:103C4000828083D725002300F50003D5050083D7A4
:103C500025003305F502050542054181828083D7A1
:103C600005002300F50083D70500A183A300F5001C
:103C700083D725002301F50083D72500A183A30165
:103C8000F50003D54500110542054181828083D7A7
:103C900005002300F50083D70500A183A300F500EC
:103CA00003D52500090542054181828089471145D8
:103CB000639BF60083471600834606000145A20772
:103CC000D58F2310F700828003D70500D947AE8631
:103CD00063F9E700B745010001470D469385E5BC50
:103CE00071BA0945828011456393A6028347160085
:103CF000834606000145A207D58F2310F7008347AE
:103D0000360083462600A207D58F2311F700828054
:103D100083C725000547FD1793F7F70F6361F70485
:103D200083D705008DCF011122CC2A84C84106CE4D
:103D300015C12EC68945EFD05FEA2A8722856244E5
:103D4000B246F240B74501001546938545BE056170
:103D50006FF0DF92F24062440945056182800945B7
:103D600082809547114563F9D706411122C426C2C6
:103D70004AC006C683471600BA8403470600A20756
:103D80003284D98F2390F4008347360003472600FE
:103D900093054400A207D98F2391F4008947238219
:103DA000F400094613855400368997C0FE1FE7804A
:103DB00020479307A9FF2394F4009947631BF90058
:103DC00023A60400B2402244924402490145410125
:103DD00082801904C0C4FDB7828083D705008DCFCF
:103DE000011122CC2A84C84106CE15C12EC68545B4
:103DF000EFD0BFDE2A8722856244B246F240B74543
:103E000001001D46938585C005616FF03F87F24034
:103E1000624409450561828009458280994763951E
:103E2000F6048947411106C62302F70083471600AE
:103E300083460600B285A207D58F2310F70083477B
:103E400036008346260003464700A207D58F130598
:103E500057002311F700910597C0FE1FE780403CF3
:103E6000B240014541018280D14711456394F6007B
:103E7000C1474DBF828083D705008DCF011122CC71
:103E80002A84C84106CE15C12EC68945EFD0FFD47D
:103E90002A8722856244B246F240B7450100254692
:103EA000938545C105616FF06FFDF240624409459D
:103EB000056182800945828089471145639BF60030
:103EC00083471600834606000145A207D58F2310BD
:103ED000F7008280011122CC2A84C84106CEAE862A
:103EE000014719C52EC68545EFD03FCFB2462A8778
:103EF00022856244F240B74501002D46938505C3F3
:103F000005616FF0AFF711456393A6028347160072
:103F1000834606000145A207D58F2310F70083478B
:103F2000360083462600A207D58F2311F700828032
:103F3000011122CC2A84C84106CEAE8611C52EC6F8
:103F40008545EFD09FC9B2462A8722856244F24058
:103F5000B74501003546938565C305616FF00FF2E3
:103F600093F71600114589EB89476387F600858230
:103F70002312D70010C301458280011122CC2A846C
:103F8000C84106CE15C12EC68545EFD01FC52A876C
:103F900022856244B246F240B74501003D46938512
:103FA000C5C305616FF08FEDF240624409450561BC
:103FB000828083D705008DCF011122CC2A84C8418D
:103FC00006CE15C12EC68945EFD03FC12A8722856E
:103FD0006244B246F240B74501004546938525C488
:103FE00005616FF0AFE9F2406244094505618280E6
:103FF00009458280854763FCD7022304A700A304F8
:10400000B7008347160083450600A207CD8F231013
:10401000F7009387E6FF2311F70089476386F600D0
:10402000090650C30145828023220700E5BF1145E0
:104030008280014781464D4681456FF02FE48D47D0
:10404000114563FBD7028347160083450600A2078C
:10405000CD8F2310F7008347360083452600A20743
:10406000CD8F2311F7009387C6FF2312F7006386D5
:10407000A600110610C70145828023240700E5BF72
:10408000011122CC2A84884506CEAE8611C52EC6E3
:104090009545EFD09FB4B2462A8722856244F2400C
:1040A000B74501005D469385E5C505616FF00FDDFD
:1040B000854711456397F6008347060001452300B5
:1040C000F700828001478146654681456FF00FDB2E
:1040D000011122CC2A84C84106CEAE86014719C5FB
:1040E0002EC68D45EFD07FAFB2462A872285624427
:1040F000F240B74501006D469385E5C805616FF054
:104100008FCC011122CC2A84C84106CEAE8601474D
:1041100019C52EC68D45EFD05FACB2462A872285E1
:104120006244F240B745010075469385E5C80561D4
:104130006FF06FC9011106CE2EC6EFA0201501C980
:10414000B245F2400355250005616FE0A06BF240D7
:10415000494505618280B7270020A38007A2B727C1
:104160000020238007A2B727002023A407A0B72799
:10417000002023A607A0B727002023A807A0B72761
:10418000002023AA07A0B727002023A207A0B72753
:10419000002023A007A0B7270020938747C1370638
:1041A00084033707B40090D337C6070098C31306BB
:1041B00006B83747A000D8C3D0D3370710004166F0
:1041C0009306070AB70550009308060194C723A475
:1041D000170393860501930816F8D4C723A617037F
:1041E000B706D007B7087F00130807051385060137
:1041F000410723A81703B0C393081600938606054A
:1042000013861500D8CBF8C323A8070188CF23AEA7
:10421000070023AA170323AC070223AE070223A437
:104220000704F0C7B4CB23AA0704ACCF23AE07051D
:10423000B8D33707A000F8D71307000AB8DB130775
:10424000C01CF8DB37071400B8DF0547F8DF130799
:1042500010F8E8D323A4070623A0E7088280011101
:1042600026CAAA84214522CC06CE2E8432C636C464
:104270003AC2EFD0FFA21DC9A246124732469307A9
:1042800000FD2300F5009947A30095002301F500E8
:104290002303D500A303E5002312C500AA852285C8
:1042A0006244F240D24405616FD09FAEF240624456
:1042B000D24405618280B727002023A4A7A0828072
:1042C000B727002023A6A7A08280B727002023A815
:1042D000A7A08280B727002023AAA7A0828001116F
:1042E00022CC4AC806CE26CA2A890144B3048900D2
:1042F0006368B400F2406244D2444249056182805E
:104300002EC6EFD03FC393170501C183A183B245E9
:104310002380F4009307140093F7F70F850463F9E3
:10432000B700CA9709042380A7001374F40F7DBF58
:104330003E847DBF411122C437240020130484C968
:1043400003556400C16706C6FD17630FF500B72764
:10435000002003C607D7B7250020938585A1EF90DD
:104360009050FD572313F400B24022444101828053
:1043700009C925151375F50F1335850E134515005D
:1043800082800145828023900500C9C6797122D4BC
:1043900026D24ECE52CC5AC806D64AD056CA5EC68F
:1043A0003684328AAE892A8B814463F34407B3078B
:1043B000940083C70700138914004209939A0701E8
:1043C00093DA0A011359090163840A04CA97634105
:1043D000FA04B307240183CB07005E85513F0DC962
:1043E0009387FAFF2390F90063906B03130519007C
:1043F0002295B250225492540259F249624AD24A4A
:10440000424BB24B45618280D694C204C18071BFD9
:104410000145C5B701458280011122CC3724002017
:1044200026CA4AC84EC6930784C906CE2E89D0CB69
:104430008CCBC8C7AA8441469305F00F4A8597C024
:10444000FE1FE78080F38549130484C9631935038F
:104450000848C145693541469305F00F268597C048
:10446000FE1FE78080F10549631525034844624437
:10447000F240D2444249B249C14505618DB5414639
:1044800081454A8597C0FE1FE78020EFE31535FD83
:10449000C1B741468145268597C0FE1FE780E0ED04
:1044A000E30625FDF2406244D2444249B249056127
:1044B0008280011122CC3724002026CA4EC6AE8449
:1044C000AA8913060002130584C9814506CE4AC88D
:1044D00097C0FE1FE780E0DBB7270020130984C9DF
:1044E000238A97D6A3013901EFE00034130484C96D
:1044F000854719C1814749452300F400F2406244D1
:10450000D2444249B24905618280814781CD19C9AF
:104510008547631BF50083C7550093E707FCA3821B
:10452000F50085473E85828089476317F50083C77C
:10453000550093F7F703E5B70D478547E314E5FE0C
:1045400003C755001377F70313670704A382E50039
:10455000D1BF81478DC105C103C755009306000C2B
:1045600085471377070C6308D700930600048D472F
:104570006303D70089473E858280411122C4005DD4
:1045800006C626C21DC8AA84085009C597C0FE1FCA
:10459000E78080B9485009C597C0FE1FE780C0B8C2
:1045A000085409C597C0FE1FE78000B8228597C050
:1045B000FE1FE78060B723AC0402B240224492445D
:1045C00041018280B7270020938787C919E903C773
:1045D00027001385870101CB372500201305859F10
:1045E0008280138587018280B727002003C5A7C971
:1045F0008280B727002003A547CA8280B727002002
:1046000003A587CA8280B727002083A7C7CA88432B
:104610008280B7270020938787C9D44B984205072B
:1046200098C203C537009307F00F6305F500916545
:104630006FD0FFB08280011122CC06CE2E8432C60C
:10464000EF9070559147B2456310F502B7270020EF
:1046500083A747A195C303A30700630F0300228527
:104660006244F24005610283B727002083A7C7A0F8
:1046700081C703A34700D5B7F240624405450561F1
:104680008280011122CC2A840355450006CE26CA19
:104690004AC84EC6EF90502E3DC92A898344050072
:1046A0008349C500D93D4A85EFA0000E035544005B
:1046B000EF90B04937290020130909A28347090068
:1046C000B9CB639A9704B727002083C517A2268524
:1046D000953419E12300090003554400EF90B04BD5
:1046E0009147631FF500B7270020938787C983563A
:1046F000440003D767006395E6007D572393E700E6
:10470000F2406244D2444249B24905618280814903
:104710009304F00F45B79307F00FE38FF4FA834645
:10472000640003564400034524004E87A685053ED9
:1047300065B779715EC6AA8B2E8552CC56CA5AC807
:1047400006D622D426D24AD04ECEAE8A328B368AB4
:10475000EF9090227DC1045D2A89E5C09C5061459F
:1047600099C3130540039C5481C7510542054181FB
:1047700063050A00710542054181DC5081C75D0572
:1047800042054181EFD0CFD12A8445C96146814598
:1047900097C0FE1FE780E0AFB727002083C947C45A
:1047A0006394090083490900930700FD2300F40086
:1047B000A947A30074012301F400230364018C5072
:1047C000231254011305840191C908C47146930A48
:1047D000440397C0FE1FE780A0A456858C5491C95E
:1047E00048C45146930A450197C0FE1FE78040A385
:1047F0005685630C0A0008C87146D285930AC50124
:1048000097C0FE1FE780C0A15685CC5099C548C807
:104810005D4697C0FE1FE780A0A0A2854E85EFD021
:104820002FD72254B2509254F249624AD24A424B94
:10483000B24B4A850259456189B3B2502254925411
:104840000259F249624AD24A424BB24B45618280D8
:1048500001114EC6AA892E854AC806CE22CC26CA88
:104860002E89EF90701121C9B727002083C447C457
:1048700099E0834405001945EFD08FC22A8405CD05
:104880008145194697C0FE1FE780A0A0930700FD51
:104890002300F400B947A30034012301F4002312DC
:1048A0002401A2856244F2404249B2492685D2449D
:1048B00005616FD0EFCDF2406244D2444249B24923
:1048C0000561828039715ECEAA8B2E8526DA4ED69E
:1048D00052D456D25AD006DE22DC4AD8AE84328B6D
:1048E000B68A3A8ABE8942C6EF90100921CD2A893C
:1048F0004145EFD0EFBA2A8431C54146814597C082
:10490000FE1FE7800099B727002003C547C419E1BF
:1049100003450900930700FD2300F400BD47230170
:10492000F400B247A300740123129400230464012D
:10493000A304540123054401A30534015CC4A285EA
:10494000EFD00FC5F2506254D2544259B259225A94
:10495000925A025BF24B21618280797126D2AA843D
:1049600039454AD04ECE06D622D42EC6B2893689D3
:10497000EFD00FB321C1B2459307000D2310F5000E
:10498000B1472A842312B5002301F500CE8519050D
:10499000194697C0FE1FE780A08823062401A28540
:1049A0002254B2500259F24913F5F40F9254456162
:1049B0006FD00FBEB250225492540259F249456151
:1049C0008280411126C2B7240020938484C903C782
:1049D000340006C622C44AC09307F00F630AF704E6
:1049E0002A893945EFD0CFAB2A8439C1930700FD1E
:1049F0002300F500A3002501230105009385840110
:104A00000D05194697C0FE1FE780808183D784007B
:104A1000A28503C534002315F40083C714002306C0
:104A2000F4002244B2409244024941016FD04FB693
:104A3000B2402244924402494101828001115AC08D
:104A40002A8B314526CA4EC652C456C206CE22CC47
:104A50004AC8AE84B28A368ABA89EFD06FA43DCDF7
:104A60002A842685EF90407111C50347C500A147F0
:104A70006314F704B727002003C9B7C9930700FDE3
:104A80002300F4009D47A30064012301F4002312D6
:104A90009400231354012314440123153401A285E7
:104AA0006244F240D244B249224A924A024B4A85B9
:104AB000424905616FD0CFADB727002003C957D752
:104AC000E31E0BFAB727002083A707B59C47DDD765
:104AD000CE865286D685268582974DB7F2406244AF
:104AE000D2444249B249224A924A024B056182802D
:104AF000011122CC2A84214506CE2EC6EFD04F9A32
:104B000021C1B245930700FD2300F500C5472301ED
:104B1000F50083C73500A301F50083D745002312B4
:104B2000F50083C765002303F50083C77500AA85D8
:104B3000A303F50022856244F24005616FD04FA5C2
:104B4000F240624405618280397162CC2A8C5945F9
:104B500026DA4AD84ED652D456D25AD05ECE06DE87
:104B600022DCAE8432C636C4BA8B3E8BC28A468AF9
:104B70008359010403494104EFD08F9225C932467D
:104B8000930700FDA2462300F5009547A301C50049
:104B9000A30085012301F5002A8419461105A9C245
:104BA000B68597B0FE1FE780A06723066401230A3D
:104BB00024012315740123175401231844012319D8
:104BC0003401A2856254F2504259B259225A925A83
:104BD000025BF24B624C2685D25421616FD04F9B11
:104BE000814597B0FE1FE780C06AC1B7F25062549A
:104BF000D2544259B259225A925A025BF24B624C39
:104C000021618280411122C437240020130484C909
:104C10008347240006C626C28DCBB7240020AA8570
:104C200019461385849F97B0FE1FE780605F034598
:104C300024009385849FEFF05F8D2244B24013855A
:104C4000849F924441016FD0F03EB240224492448E
:104C5000014541018280411126C2B724002093877B
:104C600084C906C622C44AC003C737009307F00FA1
:104C7000938484C96304F7042A892945EFD04F82BD
:104C80002A840DCD930700FD2300F500A147A30062
:104C900025012301F50083C72400B7250020938553
:104CA000859FA301F5001946110597B0FE1FE78007
:104CB000205703C53400A285EFD08F8D03C7240091
:104CC0008D476311F702B727002083A707A199CB6F
:104CD00003A38700630803002244B24092440249C0
:104CE00041010283B2402244924402494101828040
:104CF000797122D406D626D24AD04ECE52CC56CA8C
:104D000009445DCD2A8903550500AE895144EF90D1
:104D1000A046AA8455C537270020930707D783C725
:104D200047008546BA8AFD1793F7F70F494463F9A0
:104D3000F6080347C500A1476314F700639209080A
:104D40009C5C4544B5EF9165938545711305C002A0
:104D500097B0FE1FE780002F88DC2A8A4D442DC1C2
:104D60001306C002814597B0FE1FE780805283572B
:104D7000090093064A0036852311FA00714693050F
:104D8000490036C697B0FE1FE78080498947230057
:104D9000FA0003C5C400B2460356090083C50AD70A
:104DA000611513351500EFA0806F2A846386090012
:104DB000CE852685EF90F04C01C42685EFF0EFFB01
:104DC0002285B250225492540259F249624AD24A80
:104DD00045618280B727002083C747D70547FD1765
:104DE00093F7F70F6378F708894751C6011122CC72
:104DF00026CA4AC84EC652C406CEAA89368AB2848A
:104E00002E89EF9060372A84D14729C9485509C5B2
:104E100097B0FE1FE7804031F1452685EFD06F98AF
:104E200048D4CD4705CD8346C40021478147639FC1
:104E3000E600630D0A000347A5010356050193062A
:104E40002501AA854E85EF90704BAA870347440041
:104E5000630F0900136767002302E400F240624415
:104E6000D2444249B249224A3E8505618280136795
:104E70004700DDB7C9473E8582809307000463EC95
:104E8000A7009317150037250020130545C13E954F
:104E900003550500828041657D158280011122CC79
:104EA0002A842E8526CA06CEAE84EF90E02C1DCD36
:104EB000B7470F009387F723094563E487028145CD
:104EC0000A85414697B0FE1FE780A03CA6852310C7
:104ED00081000A85418023018100A3010100EFA028
:104EE000803BF2406244D244056182804945D5BF8F
:104EF000B72700202389A7D682806FA060547971DC
:104F000052CC2A8A328522D426D24AD04ECE56CAD4
:104F10005AC85EC606D662C4AE8BB28A368BBA84D5
:104F20003E89C2894684EF90202515C92A8C6314D6
:104F30000A0213774B008347450015CF93E72701FB
:104F40002302FC008DEC631C0902639A090205E848
:104F5000ED9B2302FC00832B8C03639F0B06B25056
:104F6000225492540259F249624AD24A424BB24BFD
:104F7000224C45618280F59B93E70701D1B793E707
:104F800047002302FC0001CC1C484146A285232493
:104F9000FC0213058C0197B0FE1FE7806028639127
:104FA0000B02D5D80325CC0209C597B0FE1FE780B8
:104FB000A017F1452685EFC0DFFE2326AC0261BFB6
:104FC000E30B09F80325CC0209C597B0FE1FE78063
:104FD000A015F1454A85C5B79DC483A70B0299EB7F
:104FE000916593853571714597B0FE1FE780800507
:104FF00023A0AB0203A50B0219C57146A68597B085
:10500000FE1FE780E0216388090283A74B0299EB2A
:105010009165938525715D4597B0FE1FE7808002FD
:1050200023A2AB0203A54B0219C55D46CE8597B0FE
:10503000FE1FE780E01E1DC483A78B0299EB9165DC
:1050400093851571514597B0FE1FE780A0FF23A4FB
:10505000AB0203A58B0219C55146A28597B0FE1F6E
:10506000E780001C2254B2509254F249B24B224CB9
:10507000CA865A860259424BD6855285D24A624A1E
:1050800045616FF00FEB011126CA52C406CE22CC47
:105090004AC84EC62A8AAE84EF90000E25C5AA895A
:1050A0003945EFC0FFBF2A8431CDB727002003C99F
:1050B00047C46314090003C909009307000D2310B6
:1050C000F400AD472301F400938569001305340013
:1050D000194697B0FE1FE780A01493F7140085804F
:1050E00085882306F400A306940023154401A285B5
:1050F0006244F240D244B249224A4A85424905619B
:105100006FC01FC9F2406244D2444249B249224AA8
:105110000561828001114EC652C456C206CE22CC11
:1051200026CA4AC8AA8A2E8AB289EF90E0042DCDF9
:105130002A891305C002EFC0BFB62A8435C5B72738
:10514000002083C447C499E0834409009307000DFD
:105150002310F400E9472301F400930569001305C7
:105160003400194697B0FE1FE780800BD2852315C7
:1051700054011305C400414697B0FE1FE780400A62
:10518000CE851305C401414697B0FE1FE780400954
:10519000A2856244F2404249B249224A924A268597
:1051A000D24405616FC0DFBEF2406244D24442493E
:1051B000B249224A924A05618280411122C43724B1
:1051C0000020130404A0084006C619C597B0FE1FAE
:1051D000E78080F523200400B24022444101828010
:1051E000011106CE22CC26CA4AC82EC6EF80D0783E
:1051F00039CDB245B727002003C947C40CD5AA84CE
:1052000063140900034905004145EFC07FA92A84C2
:105210001DCD9307000D2310F500A5472301F500D0
:1052200083C75400938564001105A30FF5FE19464A
:1052300097B0FE1FE780C0FE9C54A285F2405CC47C
:105240006244D2444A85424905616FC07FB4F2404E
:105250006244D2444249056182801D71A2CC86CE4F
:105260002A842EC6EF80507105CD8346C5001147B4
:10527000AA8749456392E6029C5FB24599C383C5FC
:105280006701B70602002308B1009386264710087D
:1052900089452285EF90A075F6406644256182809D
:1052A0005145DDBFB727002083C747D70547FD1706
:1052B00093F7F70F637AF704894721CA411122C493
:1052C00026C24AC006C6B2842E89EF80F06A2A84BC
:1052D000D14705C5630809008347450093E72700C8
:1052E0002302F5004146A6851305840197B0FE1FF1
:1052F000E78000F39C481CD48147B240224492448A
:1053000002493E8541018280C9473E85828079718C
:1053100022D406D62A842EC6EF80106601CDB2456F
:105320002285230EB1006C08EF902072B2502254F7
:10533000456182805145DDBF6F80B07AC1671387B8
:10534000E7FF6395E502B727002083A7C7A091EB8D
:10535000494582804945B240224492440249410174
:10536000828003A30700E30503FE0283411122C4E8
:1053700026C24AC006C6FD172A892E84B284639AC3
:10538000F502B727002083A7C7A091CF9C4381CF08
:10539000829711E9B7270020238027A3B727002091
:1053A000A38097A24DBFA6854A85EFE0BFD845F5FB
:1053B000D5B72E85EF80505C51DD834705000D4544
:1053C000E39B27F922852244B2400249A6859244F4
:1053D00041016FD020439307000463E2A706411107
:1053E000C16722C406C626C2FD172A840945638206
:1053F000F502C547AE846313F4022E85EFD0404812
:1054000037250020130545C106042A942310940073
:105410000145B24022449244410182809307A00397
:105420006316F4002E85EFD0A03ED9BF9307B003DA
:10543000E318F4FC13F5F50FEFD0C03DD1B70945E3
:105440008280411106C622C426C22A84EFE0BFD062
:10545000EF202075EF105016EF60427A37250020BC
:10546000930485C98145130585C91306000297B0C9
:10547000FE1FE78000E2930700F02391F400B727B6
:105480000020138707D7FD562301D700238887D62E
:105490002285224423820400B24092449545410172
:1054A0006F706058597193970501CAD086D6A2D4FF
:1054B000A6D2CECED2CCD6CADAC8DEC6E2C4E6C206
:1054C000EAC06EDEC1872E8963D30756B72A002053
:1054D00003C50AD7B7240020372B0020EFC05F8315
:1054E0002A84372A0020372C0020372D002093846F
:1054F00084C91DE021653345A900B6502654965451
:105500000659F649664AD64A464BB64B264C964C47
:10551000064DF25D65618280834704001307200A0F
:10552000639CE70083C9340003552400C1652286CB
:10553000FD15EFF04F90B9AA13870AD783492700CA
:10554000130710096394E716834714001547639EF9
:10555000E7002285EFF0EF922285EFC04FEF03C501
:105560000AD7EFC0EFFA2A8469B73947639AE7167A
:10557000035544008567A5076315F5040C4483CBE8
:105580000500639D0B00850591C9B72700201946CA
:10559000138507CB97B0FE1FE78080C803C70400C0
:1055A00085476315F71063880B00238004005E8530
:1055B000EFF02FC155B789472380F400EFD0402783
:1055C00061BF896713872700631CE504832B840070
:1055D000638E0B0C83C70B0089EF83C72B0003C7B7
:1055E0001B00A207D98F2394F40083C73B00A3803C
:1055F000F40003C704008947631AF70A83C70B0046
:1056000091C72380040003C50B005DB783C5140058
:1056100003D584008D472380F400EF70C043E5B7C5
:1056200095076318F5001C4403C50700EFF0AFE2CF
:1056300025B7F9771387A7FF2A9742074183914639
:1056400063F1E6049387A7FCAA97C207C183714759
:105650006371F70289671387B7006310E504832736
:105660008AA0E38B07EE9C43A285E38707EE82972F
:1056700015A0370700181307F770B357F700858B8D
:10568000B1CB83270BA1E38907EC9C43E38607ECAE
:1056900022858297E31205EC11A81387C7006310D7
:1056A000E5021C4483C70700E38807EA9307F00F6D
:1056B000E384F9EAA2854E85EFC08FED4DB5B907B9
:1056C000631AF500B727002083A7C7A0E38607E881
:1056D000DC4359BF896793871704E302F5F8F9B7EC
:1056E0003D47639BE7040355440089671387D70050
:1056F000E30AE5FC13879701E306E5FCCD07E31712
:10570000F5FA03D76400C167FD17631FF700B727D9
:10571000002083A7C7A0E38107E4DC43E38E07E210
:105720000965A2854D05A1B7B727002083A747A12A
:10573000E38407E29C43DDB71307E003E398E7F651
:105740008347240005476396E70E834764003727A5
:105750000020930D07A0F1E383A70D00C5CF83CBF5
:105760000700A14903457400930C8400E685EFE02F
:105770005FDE83474401A303A40083580401035858
:10578000E400035744002A86034534003EC2835791
:105790002401E686DE853EC0CE87EFF0EFBA834770
:1057A000340095E7DD47835804010358E40083463D
:1057B0007400835544003EC28357240166873EC06F
:1057C000CE8705465E85EF801054A301A40083A711
:1057D0000D0081C71145EFF05F9E930B0CA203C52E
:1057E0000B00E30B05D683451DA2EFE0BF94E30554
:1057F00005D68346340093071003638AF6000356E8
:10580000440083C50B004E873685EFE05FA523007B
:105810000CA299B383CB3400A9B783270BA183CB08
:1058200034009149A1D3DC4395DF8145014582973E
:1058300015BF29476398E70A83476400372700208C
:10584000930D07A0A5EF83A70D00B5C783CB070075
:10585000A149034574009306840093772500BDCBCE
:105860001376150013034401834704028358C401CF
:105870000358A40103574400034534003EC2835734
:10588000E401DE851ACE3EC0CE87EFF0EFAB834752
:10589000340072438DFFDD478358C4010358A401CF
:1058A00083467400835544003EC28357E4011A873F
:1058B0003EC0CE8739B783CB340059BF83270BA1B5
:1058C00083CB34009149D1D7DC43C1D78145014511
:1058D000829741B7B68536CEEFE0BFC7F2462A863B
:1058E000368359B70947639CE70083278AA0E3857D
:1058F00007C6DC43E38207C622858297B1B92D47EC
:105900006398E70083278AA0E38807C49C47DDB734
:105910000D476397E70022868D450355440011B972
:1059200019476395E7069305610213051031EF608F
:1059300082352C1013052031EF60E23403566400E9
:10594000835781020355440063E8C70083568400EF
:105950000357610263F7E60093050002EFC0507140
:10596000E5BE6374E6002313E40063F4D700231458
:10597000F4000357C4008356A400035684008355E3
:10598000640001488147EFC0706EF9B61D47E38F90
:10599000E7D031476395E7002286B145BDBF354763
:1059A0006398E70083278AA0E38807BADC4799B7A2
:1059B00039476396E7002285EF00F00771BE3D4747
:1059C0006398E70083278AA0E38807B89C4B1DB73C
:1059D00041476396E7002285EF001011B5BE4547A9
:1059E0006396E7000145EF009020BDB64947639DEF
:1059F000E70083270BA1E38B07CADC43E38807CAD0
:105A00008145054582975DB14D47639CE70083273B
:105A10000BA1E38D07C8DC43E38A07C8A2850945CB
:105A2000D5B76147E394E7C82286E145FDB593F712
:105A3000150089CFB727002083A787A089C7DC433B
:105A400099C3014582971345190045BC93F725007A
:105A500091CFB727002083A707A191C7DC4381C757
:105A60008145054582971345290041BC93F74500C0
:105A70000145E38407A8B727002083A747A0372460
:105A80000020130484C991CF85472302F400B7276F
:105A9000002083A707A191C7DC4381C78145054545
:105AA000829748442C10EF90606B2810EFF08F9590
:105AB000B727002083D767C381CF130600643386DE
:105AC000C702B727002003C507D79145EFC01F863F
:105AD000134549001DB4011122CC2A84554506CE38
:105AE00026CAEFF08FB9AA8413054002EFF0EFB891
:105AF0002AC613055002EFF04FB8AA8622856244E9
:105B00003246F240B3359000D24405616FC0B05CBC
:105B1000797122D406D68D472E84631FF50003D7F2
:105B2000A50083D6850003D665000345340083D5E0
:105B30004500EFE0BFF009A889671387D70063111C
:105B4000E50403C5250019E58547B25022543E857A
:105B500045618280B727002083A607A0F5D603C63B
:105B6000360083C50600814802C202C00148814751
:105B700001479106EFE05FFD0545EFF00FE4E9B75F
:105B80001387E700E302E5FC13873701631AE5009A
:105B900003C5250055D9014781460146814551BFBE
:105BA000E507E303F5FAB1476319F500B7270020CD
:105BB00003C5B7C9EFE0DFF341BF41677D178147F8
:105BC000E315E5F803C75500C947E31FF7F683D689
:105BD000E50003D6C5000355840083D5A500EFC0BA
:105BE000105641C95D45EFF04FA93335A000231C85
:105BF000A10083454400035524003008EF8000488D
:105C000083578101B1F36C0813051031EF60A207CF
:105C10009305E10113052031EF60E2068357C101CE
:105C2000035784006374F7002314F4008357E101E1
:105C30000357A40063F4E7002315F400835784009E
:105C40000357A4006374F7002315F40003552400E0
:105C5000EF40B11F0357E4008356C4000356A4006D
:105C6000835584000355240001488147EFC0D03D8F
:105C7000E1BD8547231CF100ADBFB7270020138786
:105C800007D7834677001307F00F638CE60851C9E6
:105C9000411122C426C24AC006C6AA840345A500F3
:105CA000138907D74105EFB0BFFF2A842DC593079D
:105CB000000D2310F500D9472301F50083D74400D8
:105CC0002312F50083C764002303F50083C7740023
:105CD000A303F50083C784002304F50083C7940061
:105CE000A304F50003C6A4002305C50015C2CC44D7
:105CF000410548C497A0FE1FE7808052A285224438
:105D000003457900B2409244024941016FC04F8877
:105D100023260500E5B7B2402244924402494101DE
:105D200082808280C1671387E7FF639EE500B72703
:105D3000002083A707A09DC383C707000D47639D6D
:105D4000A7006FC0B02FFD1749476397F500B7272D
:105D5000002083A707A0F5F73A8582804947EDBF69
:105D6000397122DC06DE26DA4AD84ED652D456D213
:105D70005AD05ECE62CC0347050085472A84630D66
:105D8000F70403468500930695009305E100054559
:105D9000EFE06FDF814719C18347050083460400A8
:105DA00011476383E60437270020032707A38D46A6
:105DB00003471700630AD70285CB1DC70DE10145D4
:105DC000F2506254D2544259B259225A925A025B4A
:105DD000F24B624C2161828081470145C1B7854603
:105DE0006314D70A8D8BE1DF03451400130A2400E6
:105DF000D285EFE00FF637290020A300A400832707
:105E000049A32A8B130949A38149C1C7B72A002096
:105E10009304F00F83C7CAA2138CCAA263FDF902D0
:105E200003250900939B49005E9583470500638421
:105E3000970683471500639067071946D2850905C1
:105E400097A0FE1FE780004B39C583240900034754
:105E50000400DE94B9E4834604009147E381F6F63A
:105E600083270900A9DF03460C0001479305F00FC3
:105E7000E307E6F4BE84C10703C507FF6309B50C59
:105E800005071377F70FEDB78946E31AD7F2858B2D
:105E900099BF054535B7850993F9F90FA5BF88C4A2
:105EA000F5A09147631AF706C84405C583478400E7
:105EB000034605006304F606034704009147631D8B
:105EC000F706C84419C597A0FE1FE780E02523A662
:105ED00004000345840091659385E571050597A04D
:105EE000FE1FE780201605C5034704009147631E87
:105EF000F704C8C483478400930594000505A30FE5
:105F0000F5FE0346840097A0FE1FE780603103453D
:105F100084003335A0006DB5884441BF93059400DB
:105F2000050597A0FE1FE780E03C8547E316F5F8DE
:105F30005545EFE09FF4BDA8884441DD97A0FE1FC2
:105F4000E780801E23A4040069B788C465B7238056
:105F5000D40083471400D28513852400A380F40065
:105F6000194697A0FE1FE780A02B0345840091658A
:105F70009385F571050597A0FE1FE780A00C05C568
:105F8000034704009147E31CF7F0C8C4834784002B
:105F9000930594000505A30FF5FE0346840097A022
:105FA000FE1FE780E02783478400E39407EE034564
:105FB00004007D151335150021B5397122DC26DA70
:105FC0004ED652D406DE4AD856D25AD05ECE2A8455
:105FD0009309250003451500CE85B7240020EFE086
:105FE0004FD7A300A400938404A39C400D472A8AA2
:105FF00083C717006390E70437290020832749A34C
:10600000814A130949A3638E0714B72B002003C7E5
:10601000CBA293970A01C18303250900138BCBA25E
:1060200063E7E70C83460B0003270900814713064B
:10603000F00F79AAF1D3144C034674019305E100E3
:106040000545EFE04FB405CD9840854683470500F0
:10605000034717006310D7028D8BD9FF0145F2501B
:106060006254D2544259B259225A925A025BF24BAC
:10607000216182808946858BE310D7F8F9BF834779
:10608000040011476385E7002D47E399E7FCB72437
:10609000002083A744A3938444A3E9D3814A014900
:1060A000B72B00201DA88840139B4A00834704009B
:1060B0005A95034705006311F70283471500639D56
:1060C00047011946CE85090597A0FE1FE78080226B
:1060D00001C503A904005A99850A03C7CBA2939767
:1060E0000A01C183E3E1E7FCE31809F085BF93945B
:1060F0004A0026950347050083470400631FF70AFB
:1061000083471500639B470B1946CE85090597A069
:10611000FE1FE780201E55C1832709001147BE944A
:10612000834704006385E7002D47639EE70203AAC7
:10613000C4008347740103460A006309F6025285CE
:1061400097A0FE1FE78040FE03457401916593858B
:10615000E571050597A0FE1FE780C0EE1DE5E3830E
:1061600004EC0545EDBD03AA8400E1B70C4C130512
:106170001A0097A0FE1FE780E0178547E311F5FCA2
:106180005545EFE09FCF61DDD1BD83470400114746
:106190006385E7002D476390E702C8C48347740115
:1061A0000505A30FF5FE034674010C4C97A0FE1FD6
:1061B000E78000076DB788C4D5B7850A89BDBA8462
:1061C0004107834507FF638AC5008507C207C1836E
:1061D000E3E7D7FE79B788C491A083470400CE8552
:1061E000138524002380F400834714001946A380FC
:1061F000F40097A0FE1FE780A0020345740191659B
:106200009385F571050597A0FE1FE780A0E331D9BE
:10621000034704009147E310F7FCC8C483477401A7
:106220000505A30FF5FE034674010C4C97A0FE1F55
:10623000E78000FF3DB701114AC837290020130944
:1062400009D70347790006CE22CC26CA4EC693074B
:10625000F00F6304F70851C1AA845145EFB05FA461
:106260002A8425CD9307000D2310F500D54723017F
:10627000F50083C7340093898400CE85A301F5001F
:1062800083D744002312F50083C764002303F5007D
:1062900003C57400EFE0EFABA303A400CE851305A4
:1062A0008400194697A0FE1FE78080F783C7E400AB
:1062B000A285034579002307F40083D7040123183E
:1062C000F40083C724012309F4006244F240D2445D
:1062D0004249B24905616FB0BFABF2406244D2445B
:1062E0004249B24905618280411122C4372400200D
:1062F000130404D70347740006C626C29307F00FA1
:10630000630CF70215C9AA841945EFB07F99AA85D5
:1063100005C59307000D2310F500DD472301F500A7
:1063200083D74400B24092442312F5000345740021
:10633000224441016FB0DFA5B240224492444101A2
:106340008280011122CC37240020832744A306CE6B
:1063500026CA4AC84EC652C48DC3130444A32E8A0B
:10636000AA840149084063129902630C0A0497A0A9
:10637000FE1FE78060DB23200400F2406244D24429
:106380004249B249224A0561828093194900B30704
:106390003501884709C997A0FE1FE780E0D81C4057
:1063A000CE9723A407001C40CE97C84709C997A0E1
:1063B000FE1FE78060D71C40BE9923A6090005098F
:1063C00055B745DD13964400814597A0FE1FE78031
:1063D00040EC144081477D5613F7F70FE37F97F8A1
:1063E0001397470036972300C7008507F5B77971E3
:1063F0004AD037290020832709A306D622D426D2E3
:106400004ECE52CC56CA5AC85EC6C5C7B72A00205F
:10641000AA89130909A3938ACAA2014405E1B727EF
:10642000002083A647A399CA03C60A002A8481478D
:106430009305F00F13F7F70F6368C70813153400BF
:106440002105EFB0FF85AA8401E92145EFB05F8502
:10645000AA8421C50144CD49930700FD2380F4009F
:106460008547A38034012381F400A381840045C8BB
:106470009389840023A23401014A372B0020930B17
:10648000F00F83C70A006373FA0039E88327090015
:10649000A68503C50700EFB0BF8F03C50A0081457D
:1064A0004D350325090097A0FE1FE780E0C7232094
:1064B0000900B250225492540259F249624AD24A17
:1064C000424BB24B45618280139747003697034792
:1064D00007006305B70005041374F40F850799BF1F
:1064E00083274BA393154A00BE9583C70500638499
:1064F00077032380F90083C71500138529007D14D5
:10650000A380F900194689051374F40F97A0FE1FA4
:10651000E78000D1A109050A137AFA0F9DB723A2DB
:106520000400ADB7B727002083A707A3B1C7411167
:1065300022C406C62A841DE10945EFE01F942A867D
:1065400001C9B727002003C507D78545EFB01FDE77
:106550000545EFF04FD82A84054519C8B727002014
:1065600003C507D78545EFC0AF8522854935054569
:10657000B24022444101828001458280896793862E
:10658000B7006316D5009C4503C5070061BF93861D
:10659000C7006318D5009C45854603C5070019C987
:1065A000F5B793861704E300D5FE93872704814649
:1065B000E303F5FE36858280797106D622D426D291
:1065C0004AD04ECE52CC56CA5AC85EC662C471CDAD
:1065D00083473500AA8985C7404115C05945EFE07A
:1065E000DF89931A850193DA8A410149372A00200D
:1065F000130B000DB54B83C73900636EF900B25021
:10660000225492540259F249624AD24A424BB24B46
:10661000224C456182808307840263CF570783271A
:106620000AA3130C0AA3ADCB2285EFF06FF32DC59F
:10663000034584005105EFB0AFE6AA8431CD2310A5
:106640006501230175018347040019469305240061
:10665000A301F5008307840215052303F500834792
:106660001400A30FF5FE97A0FE1FE78060BB034652
:1066700084002386C4001DC61385440188C8930581
:10668000940097A0FE1FE780A0B983270C00A68581
:1066900003C50700EFB0CFEF050913049402137987
:1066A000F90F91BF23A80400CDB7B727002083A717
:1066B00007A3B1D72D3B2254B25092540259F2494C
:1066C000624AD24A424BB24B224C014545616FF0BF
:1066D0008FC0797106D622D426D24AD04ECE52CC63
:1066E00056CA5AC85EC662C469C583473500AA89BE
:1066F00085C7444195C05945EFE02FF8931A8501AD
:1067000093DA8A410149372B0020930B00FD414C5D
:1067100083C73900636EF900B25022549254025973
:10672000F249624AD24A424BB24B224C45618280C6
:106730008387F40063CA5707130A0BA383270A0051
:10674000A5C75145EFB0CFD52A8439CD23007501B7
:10675000A30005002301850183C704001946938522
:106760002400A301F5008387F4001505A306F500B6
:1067700083C71400A30FF5FE97A0FE1FE78040AA71
:1067800083C78400938594001305C400A305F40017
:10679000194697A0FE1FE780A0A883270A00A285BC
:1067A00003C50700EFB0CFDE0509C1041379F90F67
:1067B00085B7B727002083A707A3B9DFEFF03FC352
:1067C0002254B25092540259F249624AD24A424B80
:1067D000B24B224C014545616FF0EFAF5D7186C64B
:1067E000A2C4A6C2CAC04EDE52DC56DA5AD85ED661
:1067F00062D466D26AD06ECE630105288347350025
:10680000AA8495CB832A450063870A025945EFE0A5
:10681000CFE693178501E1873EC60144B7290020E2
:10682000130A000D054CB54C130D00FDC14D03C7F7
:1068300034006361E402B640264496440649F259A6
:10684000625AD25A425BB25B225C925C025DF24DAC
:10685000616182800387CA00B2476349F71603A7C4
:1068600009A3138909A36303071683CB0A0013F74F
:106870000B014DCF4D47639EEB0623800A005685E2
:10688000EFF0AFF36304051403C70A00914763E414
:10689000E7146319870D5145EFB08FC02A8B63074A
:1068A00005122300A501A30005002301B50183C63D
:1068B0000A00194693852A00A301D5008386CA00E1
:1068C0001505A306D50083C61A00A30FD5FE97A011
:1068D000FE1FE780E09483C60A01194693851A01DA
:1068E000A305DB001305CB0097A0FE1FE7804093B4
:1068F000F9A055476398EB0005472380EA00A38B76
:106900000A00B5BF7547E389EBFE49476396EB0084
:1069100009472380EA00A5B741476394EB000D4780
:10692000CDBF6D47E39DEBF41147E5B713F78B003F
:1069300019C32D47F9BF13F61B0013F74B0011C6FF
:1069400019C315475DBF2147E9B713F62B0011C6E0
:1069500019C325475DB719476DBF19C3294755BFEF
:106960001D4745BF03C57A015105EFB06FB32A8BB0
:1069700031CD231045012301950183C60A00194634
:1069800093852A00A301D5008386CA001505230339
:10699000D50083C61A00A30FD5FE97A0FE1FE7807F
:1069A000208803C67A012306CB0001CA13054B01D8
:1069B0002328AB0083A58A0105BF23280B0083266B
:1069C0000900DA8503C50600EFB08FBC0504F10AA3
:1069D0001374F40FA9BD03C57A0113050502EFB0C6
:1069E0002FAC2A8B65D5C9472301F500231045013B
:1069F00003C60A0093F60B0693852A00D18EA301E5
:106A0000D50083C61A0019461505A30FD5FE97A019
:106A1000FE1FE780E08083C68A00194693851A012D
:106A2000A305DB0083C69A0013053B012306DB00A8
:106A300083C6AA00A306DB0083C6BA002307DB00D7
:106A40008386CA00A307DB0083D6EA002318DB0095
:106A500083C60A012309DB009790FE1FE780407C74
:106A600003C67A01A30CCB0011C613050B02232E1B
:106A7000AB0089B7232E0B0099B7B727002083A757
:106A800007A3E38A07DAEFF09F962644B6409644C0
:106A90000649F259625AD25A425BB25B225C925C5E
:106AA000025DF24D014561616FF0EF82B727002072
:106AB00083A707A385CB03C707008D476315A702EC
:106AC000B727002003C507D74111854506C6EFB09B
:106AD0003FAF13050003EFF09F91B2400145410124
:106AE0006FE07FFFC9473E85828079714AD03729A0
:106AF0000020130909A38327090006D622D426D231
:106B0000F9E337240020130404D703474400C9479E
:106B1000298B5DC39165AA849385D57111459790A2
:106B2000FE1FE78020522320A900CD4751C503470F
:106B300074009307F00F6316F70083C70400A303E4
:106B4000F4001146A6859790FE1FE780606D9305BF
:106B500031011305F041EF30C240B7270020938781
:106B600087C903C42700034731013334800011C3B0
:106B7000090413051002EFE04FB01376F50F1377F9
:106B80001600E14715CB154532C6EFE00FAF83C7BE
:106B90002400231CA1001945230AF100EFE0EFAD0A
:106BA000324683C53400231EA1007C0838085408EF
:106BB0002285EFB01052AA87B25022549254025943
:106BC0003E8545618280C547C5BF757126C3B72420
:106BD000002022C506C74AC1CEDE938404D783C7EE
:106BE00044004944A18B638D0718B727002083A771
:106BF00007A34144639607182A89EFE0EFF383C7A0
:106C000084005544637EF516B724002083A704A0B2
:106C1000A68945446396071691659385C5712945F4
:106C20009790FE1FE780004223A0A4A04D44630973
:106C300005142946CA859790FE1FE780605E1305FC
:106C40006002EFE08FA31375F50F93771500614491
:106C5000638807121306000381451364250088002A
:106C60009790FE1FE780E0624145EFE00FA12316F9
:106C7000A1043D45EFE06FA02319A1043545EFE0E5
:106C8000CF9F231CA1043945EFE02F9F231FA104B0
:106C90002145EFE08F9E2312A1061D45EFE0EF9DF9
:106CA00083A704A02315A10683C717006382070EDC
:106CB0002D45EFE08F9C2310A1043145EFE0EF9BC1
:106CC0002313A1041305C002EFE02F9B2317A10497
:106CD0001305B002EFE06F9A231AA1041305900286
:106CE000EFE0AF99231DA1041305A002EFE0EF9898
:106CF0002310A10613058002EFE02F982313A106AD
:106D000013057002EFE06F9783A709A02316A10671
:106D100003C5370093854700EFD02FFF2AD6930590
:106D2000F1031305F041EF30C223B727002093870A
:106D300087C983C527000347F1033256B335B00036
:106D400011C3890583A609A0FC00228703C526007C
:106D50003EC8930721053EC6BC083EC49307E10523
:106D60003EC2DC103EC09308A106130861049C00DB
:106D70009106EFB090362A8401C50D45EFE0EFC3D0
:106D80002285BA402A449A440A49F65949618280C8
:106D90002545EFE08F8E2310A104294505B7B727BD
:106DA000002083C747D70145A18B89C7372500201D
:106DB000130545A26FD0CFD0B72700207D5723867B
:106DC00007A2B7270020A38BE7D6B727002023AA66
:106DD00007A2B727002023A807A237670100B7271B
:106DE0000020938787CB1307C75798C337670100E5
:106DF0001307875BD8C3376701001307276D98C750
:106E0000376701001307C77DD8C73767010013072D
:106E1000A7C798CBB727002037670100938747A201
:106E2000130747D298C337670100130707B1D8C3C8
:106E30008280411122C4372400201304C4A226C238
:106E4000AA8403450400854506C6EFF08FCFB72717
:106E5000002083C747D7A98BA5CF37250020230063
:106E60009400130585CBB7240020EFD0CFC49384C2
:106E700044A39C4099C74D45B240224492444101ED
:106E800082800345040019E10145FDB791659385B2
:106E9000B57112059790FE1FE780C01A88C061DDAA
:106EA00003460400814512069790FE1FE780603E6E
:106EB0008346040090408147FD5513F7F70FE375B3
:106EC000D7FC1397470032972300B7008507F5B723
:106ED000014523000400EFD00FBE7DB7411122C44D
:106EE00037240020032544A006C619C59790FE1F2D
:106EF000E7808023232204A0B24022444101828003
:106F000001111305700306CEEFD03FF72AC6130513
:106F10008003EFD09FF62AC413059003EFD0FFF54E
:106F20002246B245F240AA86054505616FB0B01908
:106F30005D711305D00386C6A2C4A6C2CAC0EFD035
:106F4000DFF32A841305C003EFD03FF3AA841305AF
:106F5000E003EFD09FF22A891305F003EFD0FFF191
:106F60008A871377F50F9376F90F13F6F40F93755D
:106F7000F40F0545EFB07017B64026449644064915
:106F8000616182805971A2D437240020832744A0F4
:106F900086D6A6D2CAD0CECED2CCD6CADAC80545BD
:106FA000638D070C9305F1041305F041EF20727B0C
:106FB0009305F1041305F041EF20B27AB7270020C2
:106FC000938787C983C727000347F104B337F000CD
:106FD00011C38907032744A03EDE0345370093050C
:106FE0004700EFD08FD2032744A02ADC0D4583450C
:106FF00027002EDAEFD07FE82AD81145EFD0FFE73F
:10700000032444A02AD665450347A400034BB400DB
:107010003AD4EFD09FE6AA846945EFD01FE62A89CB
:107020007145EFD09FE5AA896D45EFD01FE52A8A0B
:107030007545EFD09FE4AA8A7945EFD01FE4E204BA
:107040006258F2572257B2564256D2551375F50F71
:1070500093FAFA0F137AFA0F93F9F90F1379F90FDC
:10706000E1842ACC56CA52C84EC64AC426C25AC067
:10707000930844000545EFB07001B650265496546D
:107080000659F649664AD64A464B65618280011127
:1070900022CC06CE26CA8D472E846315F50603C77B
:1070A0003500B7240020E94703D54500938484C9FF
:1070B0006316F70083D764006382A706EF70C00BE6
:1070C00009C5835764002317F5000357A4008356AE
:1070D0008400035664008355440003453400EFD018
:1070E000FF950357440083D764006309F700854781
:1070F000F2406244D2443E8505618280FD5723936D
:10710000F400F5B78967CD07631DF50083C7250037
:1071100031476385E7004547E39BE7FCEFD08FA14C
:10712000F9B7B1476319F500B727002003C557D752
:10713000EFD01F9C6DBF41677D178147E31AE5FAC9
:1071400083C655004947E395E6FA83C545000355D4
:107150002400300023140100EF60306D49BF41115D
:1071600022C437240020834784A326C206C64AC00F
:107170001307E00FAE846386E7041307F00F1304D0
:1071800084A36387E7021145EFA09FB115C1930760
:1071900000FD2300F50089472301F5008547A30082
:1071A0009500A301F500AA8503450400EFA05FBE8A
:1071B000F9572300F400B2402244924402494101AD
:1071C00082802A891145EFA0BFAD75D5930700FDD8
:1071D0002300F50089472301F500A3009500A301D2
:1071E00025012244B7270020B24092440249AA85D3
:1071F00003C597A341016FA0BFB979714AD0372960
:107200000020832749A022D406D626D24ECE52CCC7
:1072100056CA4544D5EFB7240020938704D783C7C7
:1072200047004944958BCDC7B72700202E8A91652A
:10723000A38CA7A2AA899385757131459790FE1FEB
:10724000E78040E02322A9A04D4459C12300350125
:10725000A30005002946D28509059790FE1FE78007
:1072600020FC832749A0914603C7270063EDE60869
:1072700035EB4D472381E70003C72700136707015C
:107280002381E700930571001305F041EF20724D53
:1072900083477100F1EBB727002003C7A7C98D47CB
:1072A0006314F70CEFD0EFB42C00EF70306B2800B4
:1072B000EFD05F954545EFD05FBC014411C913067F
:1072C00000643306C50203C504D79145EFB00F86AD
:1072D0002285B250225492540259F249624AD24A4B
:1072E0004561828085466314D700754761B789463A
:1072F0006314D7004947BDBF8D466314D70041478B
:1073000095BF554785BF9546CA8A630ED7009946F3
:107310006316D70009472381E70031A01D46631497
:10732000C702238107006545EFD03FB59307F007FB
:10733000E30AF5F403A74AA08347270093E707046D
:107340002301F70081B721466314C7000547E1B761
:1073500025466315C7002381D700F1B7A946054428
:10736000E318D7F6114745BFEFF0DFC12A842DD1CE
:10737000EFF0DFB6B1BF011126CAB724002083A702
:1073800044A022CC06CE4AC84944B1C783C70700EF
:107390000D446392A70437290020034509D7894586
:1073A000EFB00FA2034509D7B72700209145239ED0
:1073B00007A2EFB0EFA083A744A001478146A380B6
:1073C00087001306F100854785450145A307F100B5
:1073D000EFB0204F2A842285F2406244D2444249D1
:1073E00005618280011106CE22CC26CA4AC8854793
:1073F000631EF506372400201304C4A3835704003A
:10740000A9CB372700200347C7C921E71307B003DB
:10741000636CF702B724002003C504D78945EFB099
:107420002F9A035604009307006403C504D733065C
:10743000F6028945EFA09FEF23100400F24062445A
:10744000D244424905618280938747FC2310F400AF
:10745000F5B7B727002083A747A0EDD36244F240D9
:10746000D244424903C50700056131B7B724002063
:1074700083A744A0E1D737270020130907D7834704
:107480004900918BC5DF89476313F5062D452EC64C
:10749000EFA01F812A845DD1B245930700FD230030
:1074A000F500E547A30005002301F50083C735007B
:1074B00015051946230FF5FE83C745009505A30F53
:1074C000F5FE9790FE1FE780A0D50345590093076E
:1074D000F00F6316F50083A744A003C50700A2853B
:1074E0006244F240D244424905616FA07F8A03455D
:1074F00007D78945EFB0CF8C6244F240D24442496D
:10750000B7270020239E07A205616FF03F9DB72794
:10751000002083C747D7958B89CFB727002083A743
:1075200087A491CBB72700200547238FE7A26FF0F0
:107530003F9D4945828041458280B727002085458F
:107540000145238F07A26FB08038B727002083C77B
:1075500047D7958B81CBB72700200547238DE7A21E
:107560006FF01F9D49458280B72700208145054562
:10757000238D07A26FB0A037B727002083C747D756
:10758000958B638F07129307C01C63FCC7000945E6
:107590008280F2406244D2444249B24909450561C1
:1075A0008280B727002083A747A0638B0710B727E7
:1075B0000020938787A303C807001307E00F631118
:1075C000E810011122CC4AC806CE26CA4EC6238036
:1075D000A700130586004205368932844181ADC972
:1075E0009165938565719790FE1FE780A0A5AA8994
:1075F0004DD1B724002003A544A4938444A409C515
:107600009790FE1FE78040B21385890023A0A90050
:107610002286814523A034019790FE1FE78060C732
:107620009C402286CA8588439790FE1FE78040BF12
:107630009C40A286F240239287006244D244424991
:10764000B249984305468D45054505616FB0E02672
:107650009165938555719790FE1FE780A09EAA893A
:107660000DD9B724002003A5C4A49384C4A409C5DC
:107670009790FE1FE78040AB1385890023A0A900E7
:107680002286814523A034019790FE1FE78060C0C9
:107690009C402286CA8588439790FE1FE78040B8A9
:1076A0009C40A286F240239287006244D244424921
:1076B000B249984305468D45054505616FB02020C8
:1076C000494582809307C01C63FCA700094582805E
:1076D0000945F2406244D2444249B2490561828080
:1076E00045CD011122CC2A8421054EC64205AE8922
:1076F00091659385657141814AC806CE26CA9790E7
:10770000FE1FE78020942A8961D5B724002003A5B5
:1077100044A4938444A409C59790FE1FE780C0A0A9
:10772000130589002320A9002286814523A0240176
:107730009790FE1FE780E0B59C402286CE85884367
:107740009790FE1FE780C0AD9C4023928700B7272B
:10775000002083A747A08DCFB727002083C747D736
:10776000958B8DCBB727002083A747A499CF98434B
:1077700083D647006244F240D2444249B2490546AA
:107780008D45054505616FB0401301478146DDB762
:10779000014581B7494535BFB727002083A747A0DA
:1077A00095C7B727002083C747D7958B95C3B727C1
:1077B000002083A747A481CB984383D64700054682
:1077C0008D450545C9B701478146D5BF0145828032
:1077D000494582809307C01C63FCA700094582804D
:1077E0000945F2406244D2444249B249056182806F
:1077F00045CD011122CC2A8421054EC64205AE8911
:1078000091659385557141814AC806CE26CA9790E5
:10781000FE1FE78020832A8961D5B724002003A5B5
:10782000C4A49384C4A409C59790FE1FE780C08FA9
:10783000130589002320A9002286814523A0240165
:107840009790FE1FE780E0A49C402286CE85884367
:107850009790FE1FE780C09C9C4023928700B7272B
:10786000002083A747A08DCFB727002083C747D725
:10787000958B8DCBB727002083A7C7A499CF9843BA
:1078800083D647006244F240D2444249B249054699
:107890008D45054505616FB0800201478146DDB722
:1078A000014581B7494535BFB727002083A747A0C9
:1078B00095C7B727002083C747D7958B95C3B727B0
:1078C000002083A7C7A481CB984383D647000546F1
:1078D0008D450545C9B701478146D5BF0145828021
:1078E000494582809307C01C63F4A7000945828044
:1078F000797122D44ECE06D626D24AD0AE892A84B9
:107900002DC121059165420593857571418197804F
:10791000FE1FE78020732A89094563060908B724FA
:10792000002003A584A4938484A409C59780FE1F26
:10793000E780807F130589002320A90022868145E6
:1079400023A024019790FE1FE780A0949C402286EC
:10795000CE8588439790FE1FE780808C9C402392C1
:107960008700B727002083A747A001458DCFB72701
:10797000002083C747D74945958B95C76C001305F1
:10798000D030EF404230B247014593F7070F81CF27
:10799000B727002083A787A48D450545944303D6C8
:1079A0004700EFA09072B250225492540259F2490B
:1079B00045618280B727002083A747A491CF03D6D3
:1079C00047008C43411106C69790FE1FE780408513
:1079D000B24001454101828009458280B7270020DD
:1079E00083A747A48DC7B727002003A7C7A489474B
:1079F00005C3035647000C43411106C69790FE1F6E
:107A0000E7800082B24081473E85410182808947FC
:107A10003E858280B727002083A747A48DC7B7275C
:107A2000002003A787A4894705C3035647000C43DA
:107A3000411106C69780FE1FE780807EB2408147D5
:107A40003E854101828089473E858280797106D6D4
:107A500022D426D24AD04ECE52CC8D4763FCA7000A
:107A60008944B2502254268502599254F249624AFE
:107A70004561828037290020034789C9C144E31248
:107A8000F7FE9307F5FF930989C993F7F70F85462A
:107A9000AE842A8403CA2900130989C963EAF60659
:107AA0008DE199452800EFC09F83B729002003C5C9
:107AB00009D7914523018900EFA09FB035E48144A7
:107AC0004DB71946814528009780FE1FE780607CEE
:107AD00019462C0026859790FE1FE780A08149F16A
:107AE00019469305F00F28009780FE1FE780607A03
:107AF00019462C0026859780FE1FE780A07F2DF178
:107B00001946A68528009780FE1FE780607171BF27
:107B1000E31DE5F803A5C9002C00EF702064AA84DA
:107B200049D52381490135BF2800EFD0AF8DAA8404
:107B30000DED930571001305F041EF20824283445F
:107B40007100B5FC8D47E31CF4F64545EFD0EFB26C
:107B50003DD5B7771800938707A03306F50203C514
:107B600009D79145EFA09F9EEDBD23014901D5BDE9
:107B7000B727002083C747D7918B8DC337250020B7
:107B80004111130505A406C6EFC0CFF4B240B727D4
:107B900000207D57239FE7C84101828001456FC0C7
:107BA0006FF3B72700207D57A38CE7A2B7270020EB
:107BB0007957238CE7A2B7270020238F07A2B72786
:107BC0000020238D07A2B7270020239E07A2B727F6
:107BD000002023A207A4B727002023A607A4B727C5
:107BE000002023A407A437870100B727002093872C
:107BF000C7CC130767E198C3377701001307473EE7
:107C0000D8C337770100130747F898C737770100C3
:107C1000130707F0D8C737770100130707F398CB8E
:107C2000B7770100372700209387E7082320F7A4C0
:107C30008280411126C2B724002083A744A006C633
:107C400022C48DCF2A840D45EFA08F85AA8505C15A
:107C5000930700FD2300F5008D47A3008500230155
:107C6000F50083A744A003C50700EFA06F9219C4D5
:107C70002244B240924441016FF04FA6B2402244E8
:107C8000924441018280797152CC372A00208327A7
:107C90004AA04AD006D622D426D24ECE56CA014990
:107CA000B1C703C91700B72400208547AA89938468
:107CB00084C96307F90483C74400054985EB0D4572
:107CC000EF901FFEAA8505C1930700FD2300F50074
:107CD0009147A30035012301F50083274AA003C57E
:107CE0000700EFA0EF8AEFF06F9F0549B2502254D2
:107CF0004A8592540259F249624AD24A45618280C9
:107D0000B727002083A747A4D28A85E30145EFD097
:107D1000CF962A8601CAB727002003C507D7894511
:107D2000EFA0CFE083A74AA081A8944303D64700E1
:107D30009305E1000545EFC00FE569D983470500CC
:107D4000858BE9D70545EFD04F939307B0032A847D
:107D500063F0A704B727002003C507D75D661306A5
:107D600006708945EFA08FFEB7270020130444FC5E
:107D7000239E87A283274AA00947A380E70083C7E1
:107D8000440081C72382040095B74E855D35B9BF95
:107D9000130600643306C502B5BF411122C42A840C
:107DA0000D4506C6EF90DFEF05C5930700FD2300E4
:107DB000F500CD472301F500A30085002244B72735
:107DC0000020B240AA8503C597A341016F905FFCD4
:107DD000B240224441018280411122C42A840D45CF
:107DE00006C6EF90FFEB05C5930700FD2300F500E5
:107DF000ED472301F500A30085002244B7270020AA
:107E0000B240AA8503C597A341016F907FF8B240A5
:107E1000224441018280035745000111896606CE44
:107E200022CC26CA13866600AA876317C7009C4720
:107E3000014583C5070009A813868600631AC70099
:107E40009C47054583C50700EFF06FB105453DA888
:107E5000138696006313C70237270020032747A025
:107E600001450DC79C4703C5070065E18547A30091
:107E7000F7000545EFA0501CD1BF1386A600631C78
:107E8000C7009C4703C50700EFF0FFDFF2406244E4
:107E9000D2440561828013866603E30AC7F813861D
:107EA0007603E30FC7F8138686036313C70A1C45DE
:107EB000372400201307E00F83C40700834784A3FF
:107EC000130484A3638EE7021307F00F6386E702AF
:107ED0001145EF90FFDCAA8505C1930700FD230043
:107EE000F5008947A30095002301F500A3010500D3
:107EF00003450400EF90DFE9F9572300F400B9B718
:107F0000B727002003A747A03E84014541D38DEC4D
:107F100085447D4523059100EFC03FF62316A1005F
:107F200013050002EFC07FF5832744A0A305A1003D
:107F30001307B100A380970074001306A1008545C4
:107F40000545EFA0101819B72685EFF09FCEFDBDAF
:107F500013869603E307C7F21386E6036317C70089
:107F60001C45094583C50700C5B59386F603631D07
:107F7000D7021C4503C5070035ED6C001305D03052
:107F8000EF307250B247414793F7070FE380E7ECB9
:107F90009305B10013056031EF30F24E0345B10097
:107FA0008545EFA0D0125DB5896613860604631679
:107FB000C7041C4503C40700B727002083C7E7A3F5
:107FC00022858DEB0D45EF90BFCDAA85E30005E836
:107FD000930700FD2300F500D1472301F500A3001E
:107FE0008500B727002083A747A003C50700EF90AF
:107FF0003FDAA9BDEFF07FDA91BD13861605631B4A
:10800000C7001C4503C5070021E985450545EFA0CC
:10801000100E2DBD938626050145E319D7E69C4732
:1080200003C40700B727002083C7A7A322858DE7D5
:108030000D45EF90FFC6AA85E30A05E0930700FD12
:108040002300F500F1472301F500B7270020A30026
:10805000850003C597A361BFEFF01FD8C5BBB72745
:10806000002083C747D7411106C6958B99CB37258A
:1080700000201305C5CCEFC04FA54D45B2404101CE
:1080800082800145EFC06FA40145CDBF03C7050045
:10809000937625009377D70F99C29367270013181B
:1080A00085011358884113F7F7076354080013E755
:1080B0000708937685009377770F99C293678700B7
:1080C0001377050293F6F70D19C393E60702238091
:1080D000D500634508009377A50281CB834706004E
:1080E00093E7C7002300F60082807DFD83470600EA
:1080F000CD9BCDBF2D456319071403C80500094763
:108100006310E814C8410347150003450500220722
:10811000498F42070D654187930825A0630B170B14
:10812000011122CC26CA4AC84EC606CEBE89B684E4
:1081300032842E8963CEE800930705A0630DF70211
:10814000130515A06300A706239004000545B5A0FC
:10815000930745A06309F7086348F706130565AA66
:10816000E314A7FE85472390F600DC4583C707008C
:108170002300F60091A0C8459780FE1FE780801479
:10818000420541814E86637335012A862390C400DF
:10819000420641828325C90022859780FE1FE78021
:1081A000200819A8DC4583D7070023900601230087
:1081B000F600A183A300F6000145F2406244D244D8
:1081C0004249B2490561828099472390F6001946D9
:1081D000D1B785472390F600DC45014583C70700EA
:1081E0002300F6008280DC45A9CB21472390E600DE
:1081F00003D707002300E60003D707002183A3006D
:10820000E60003D727002301E60003D727002183D8
:10821000A301E60003D747002302E60003D7470087
:108220002183A302E60003D767002303E60083D778
:108230006700A183A303F60041B723900600ADBFFA
:108240002390060005458280828083C80500894707
:108250006394F816DC41797122D406D626D24AD02E
:108260004ECE52CC56CA03C8170083C707002E84CF
:1082700022083368F80042088D67135808411383B9
:1082800027A0630C68102A8A3A89B684B285634CA9
:108290000301138707A0630BE802938717A063010C
:1082A000F80A854711A8138737A06303E80C1387E2
:1082B00067AA8D47E317E8FEB25022549254025940
:1082C000F249624AD24A3E8545618280484432C6BC
:1082D0009780FE1FE78000FF420541819D47E36DC7
:1082E00025FDB72A0020938A2AA583C70A00B3096F
:1082F0009900B24563D43701B5477DBF484426860F
:10830000C2094A959780FE1FE78080F103C60A00E4
:10831000484493D9090105063306364181454E95F7
:108320009780FE1FE780E0F6B727002083A747A5C8
:1083300099E3814751B79C438145E5DF52853DA0D4
:10834000AD47E31B09F6E39916FB83471600834606
:1083500006005844A207D58F2310F700B727002046
:1083600083A747A5F9D79C438545E1D78297D1B725
:10837000AD47E31309F49947E390F6F848441946EA
:108380009780FE1FE780C0E9B727002083A747A595
:10839000CDD39C43D9DF8D4555B7AD4711FF8547F8
:1083A000E39CF6F40347060093070008E3E6E6F0D3
:1083B000DC452380E700B5BF85473E858280B7272F
:1083C000002023AA07A4B7270020A38907A4B72762
:1083D0000020238907A4B7250020B707A0009385B4
:1083E0004599938707059CC1B707E803DCC137D6D9
:1083F0000300B72700209387078A130606FBD0C324
:10840000B72E002037D603000947938EFE98130637
:1084100046F8372E00202380EE00130ECE98D0C7EA
:1084200023AED70137230020B728002037280020AB
:108430003725002037D60300B7DE03008546130634
:1084400046F92300EE009388089923AEC70313036F
:1084500003A51308E8981305D598938ECEF937DE57
:1084600003002380E8002380E7002388E7002380BF
:10847000E7022388E7022380E7042300E80023843F
:10848000D70023950700D0CB238CD700239D07006E
:1084900023A2D7032384D7022395070223A607022A
:1084A000D0DB238CD702239D070223100300230077
:1084B000D500130ECEF823A2C7052388E70423AE08
:1084C00017052380E7062388E7062380E708B7D847
:1084D000030037D70300130707F99388C8FA23A2CC
:1084E000E7082384D7042395070423A66704F0CB69
:1084F000238CD704239D070423A217072384D706C0
:1085000023950706ECD7F0DB238CD706239D0706BF
:1085100023AE07072384D7082395070823A6A708B7
:1085200037870100B7270020938707931307470F6A
:1085300098C3378701001307A724D8C323A40700D3
:108540008280A54763ECA710B7D703009387078AFB
:108550000A053E951C41011122CC26CA06CE4AC806
:10856000B2842E8482879307800F63F9B700614538
:10857000F2406244D244424905618280372900209A
:108580009307098AC8571309098A09C99780FE1FEA
:10859000E78080B9B7270020238907A413061400B9
:1085A000916593850571328532C69780FE1FE780FD
:1085B00060A92326A90245DD324681459780FE1F2A
:1085C000E78020CD0325C9022286A6859780FE1F5D
:1085D000E78000C5B7270020238987A4014549BF4C
:1085E0008947E396F5F803570600B727002023983C
:1085F000E7A4EDB7A147E39CF5F637250020214617
:10860000A685130545999780FE1FE78060C1F9B7DD
:108610008547E39EF5F4B72500209385058AD04D64
:108620009385850203C50400EFF05FA645BF85472B
:10863000E39FF5F2B72500209385058AD05D9385E9
:108640008504CDB78547E394F5F203470600B727C5
:108650000020A386E79859B7094519BF09458280CC
:1086600005476302E5044111AA8706C62E8581CF1E
:1086700011476383E70425476388E7048947B240CD
:108680003E8541018280B727002083A5C78C89479A
:10869000FDD5B727002003C627A59780FE1FE780DA
:1086A00020B88147E9BFB727002083D707A52390CB
:1086B000F50081473E858280B725002021469385BD
:1086C0004599EF406210F1BFB727002083C7D798C4
:1086D0002380F500F9B7B7270020938737A503C794
:1086E000070015E305472380E700058909CDB72674
:1086F000002037250020938606934146A5451305A3
:10870000058A6F3040770145828001111388F5FF9B
:1087100006CE22CC26CA4AC84EC652C41378F80FD9
:10872000AD4563ED050BB7D503000A089385858C2D
:108730002E983E8A83270800BA893689B2848287B8
:108740008545EFB01FD72A8419E1EFF05F912285AC
:10875000F2406244D2444249B249224A05618280D1
:108760008945EFB01FD52A847DF12685EFE06FECB7
:10877000F9BF9145EFB0FFD32A8471F95286CE85B7
:108780004A85EFB07FC9EFF09F8DEFF06FBEEF70BD
:10879000C00575BFA145EFB0DFD12A844DF95286DF
:1087A000CE854A85EFB05FC72685EFE08FE8EFE022
:1087B0000FDFEF70800161BFB145EFB09FCF2A841A
:1087C00059F55286CE854A85EFB01FC52685EFE064
:1087D0004FE6EFE0CFDCEF60507F75B7094485BF0F
:1087E00079714ECEAE896C0022D426D24AD006D6FC
:1087F0002A89B284EF00707B2A840DE1CE854A85F8
:10880000EFB0AF9B2A8419E93245B74601002687AD
:108810009386C69A2D468145EF1040142285B250AA
:10882000225492540259F2494561828079714ECEA8
:10883000AE896C0022D426D24AD006D62A89B284C8
:10884000EF00B0762A840DE1CE854A85EFB00FA502
:108850002A8419E93245B74601002687938626A95E
:108860004D468145EF10800F2285B250225492541C
:108870000259F24945618280397126DAAE844C0092
:1088800022DC4AD84ED652D406DEAA893289368AEC
:10889000EF00B0712A8431EDA6856303090283D706
:1088A00004002C002314F10083D724002315F100C9
:1088B000930720302316F100930780022307F1006D
:1088C0004E85EFB06F8C2A840DE55946A6851305B9
:1088D000A100230421019780FE1FE78060941245C8
:1088E000B746010052879386669525462C00EF1007
:1088F000E0062285F2506254D2544259B259225AAB
:1089000021618280797126D2AE846C0022D44AD053
:108910004ECE06D6AA893289EF0030692A840DE14D
:10892000A6854E85EFB04F8B2A8419E93245B746AC
:1089300001004A879386A69C3546A685EF10000263
:108940002285B250225492540259F24945618280E4
:10895000BD47638CF50663E9B702A5476387F50653
:1089600063EDB7009947638CF5049D47638FF50469
:108970009547638CF50401458280B5476387F5040C
:1089800063E1B704AD47F5B7DD47638EF50263EAEF
:10899000B700C947638BF502D9476386F502C5471F
:1089A000C9BFF5476383F50263E4B700ED47D1B76C
:1089B00093072005638BF5009307200D5DBF4845A5
:1089C00082800841828008458280484182809307E6
:1089D000F00F630EF506011126CAAA8413050002E2
:1089E00022CC4AC84EC652C456C206CE3A89B6896F
:1089F000B28A2E8AEF90CFAA2A844D4515C89307D4
:108A000000FB2300F400A3005401231144012302BE
:108A1000340113058400614663050902CA85977015
:108A2000FE1FE780E07FA2852685EF906FB60145A7
:108A3000F2406244D2444249B249224A924A056114
:108A4000828081459780FE1FE780A084E9BF0945A9
:108A50008280011122CC06CE2A842306B100A3060F
:108A6000C100EF50607115C18346C500B7270020D3
:108A70002147938707D7639EE60003C56700780008
:108A80009306E0070146A2859937F24062440561EA
:108A9000828078009306E0070146A28503C557004F
:108AA000E5B7930700643306F6026F907F9D05C912
:108AB0000347050085469307270093F7F70F63F0F8
:108AC000F602411122C42A843A8506C6EF909FB669
:108AD000FD572300F400B24022444101828082808D
:108AE000035705009307000B6313F7028347450004
:108AF0004947639CE7000347150185476399E700F1
:108B00000355250085456F3090666D47C5BF82804F
:108B100001112314B1006C0022CC26CA4AC806CE2B
:108B20002A89B6842315C100EF0030482A840DE15C
:108B30002C004A85EFA09FDB2A8419E93245B7460D
:108B4000010026879386468A15462C00EF001061A7
:108B50002285F2406244D2444249056182807971A3
:108B6000930720302314B1002315C1002316F10010
:108B70002C0093078002014606D62307F100EFF090
:108B8000BFCFB25045618280C177797185073EC4FD
:108B9000894726D22316F100AE84930780024C0049
:108BA00022D44AD006D62A892307F100EF00F03FED
:108BB0002A840DE12C004A85EFA07FEB2A8419E975
:108BC0001245B746010026879386A6A345462C008A
:108BD000EF00D0582285B250225492540259456178
:108BE0008280B28605466FF03FC9797126D2AE8485
:108BF0006C0022D44AD04ECE06D6AA893289EF0024
:108C0000D03A2A840DE1A6854E85EFA05FC52A845F
:108C100019E93245B74601004A87938606840D4616
:108C2000A685EF00B0532285B250225492540259C7
:108C3000F249456182807971930720202314B100A5
:108C40002315C1002316F1002C0093078002014672
:108C500006D62307F100EFF03FC2B2504561828093
:108C6000011122CC06CE2A842EC632C436C2EF5061
:108C7000A0500DCD0345C500B7270020A14693871E
:108C800007D712472246B245631CD50003C56700CB
:108C9000B2862E86A2856244F24005616FF03FD312
:108CA000B28603C557002E86A285F5B7F24062440E
:108CB0000545056182806FF0BFB26FF07FB26FF043
:108CC0007FC46FF03FC479714ECEAE896C0022D460
:108CD00026D24AD006D62A89B284EF00102D2A84E3
:108CE0000DE1CE854A85EFA01FD12A8419E93245CE
:108CF000B746010026879386869E3D468145EF0054
:108D0000F0452285B250225492540259F2494561ED
:108D10008280B28601466FF03FB6011122CC2E84CC
:108D20006C0026CA06CEAA84EF003028DD47630A0D
:108D3000F500930710102314F400A2852685EFA0F8
:108D4000FFD5F2406244D24405618280239405003D
:108D500083D7850099E36FF07FAD09458280FDB729
:108D6000B727002003C7A7A8854763F9E7020111C9
:108D700022CC2E846C0026CA06CEAA84EF00F022F4
:108D800009E9930700102314F400A2852685EFA0BB
:108D9000FFD0F2406244D24405618280594582800E
:108DA000B727002023ACA7A48280B727002023AEDA
:108DB000A7A48280011122CC26CA06CE2A84AE84C2
:108DC000EF50803BA6852285EFA08FF40DE9228528
:108DD00023169100EF50403A1DC18346C500B727C6
:108DE00000202147938707D76390E60203C56700F9
:108DF00078009306F0070146A285EFF05FBDF240D0
:108E00006244D2440561828003C55700D5B7011181
:108E100026CA06CEB68422CCDD4663E2B608D94621
:108E200063FED50AA5466381D50A63EEB60495466E
:108E3000638CD50899466387D50A054441687D1837
:108E4000631606093AC6EFA06FF033068540324735
:108E500042064182420441803305C4004205BA857E
:108E6000418132C6EF30D041AA8749C181C4324620
:108E70002390C400B30580406244F240D2443E8552
:108E800005616F809FD5C5466380D504C9460D44F2
:108E9000E395D5FAC167FD17E31EF6FA65B7F54607
:108EA0006380D50463E4B600ED46D5B7930620058C
:108EB0006388D5029306200DE391D5F8C167FD17AD
:108EC0000D446319F600BDBF09448DBF9306200D04
:108ED000E392D5F8310642064182ADBF15445DBF2D
:108EE0000D444DBFC167FD171D447DB7F24062447C
:108EF000D24405618280011122CC26CA06CE03C667
:108F000045002E841307000281469945AA84EFF09C
:108F10001FF02AC629CD8357040003464400930559
:108F200054002310F100835724002311F1008947D6
:108F30002312F100930780022303F1009770FE1FB4
:108F4000E780002E834744008A8526852314F1009C
:108F5000EFA09F9C2A8411C532459770FE1FE780C1
:108F6000A01C2285F2406244D244056182804D44B7
:108F7000CDBF5D7186C6A2C4A6C2CAC04EDE8947F7
:108F80006306F600C1470944631AF6040144B9C5F3
:108F90002E894C0832C6B689AA84EF0010012A84B3
:108FA00032460DEDC1778507CA851305D1013ECC48
:108FB000230EC1009770FE1FE78080262C082685AF
:108FC000EFF07FF32A8419E95245B74601004E8736
:108FD0009386C68F1D462C08EF0050182285B64098
:108FE000264496440649F25961618280797122D4FF
:108FF00036844AD04ECE52CCB2892E8A3A898146E6
:10900000130710022286D94526D206D6AA84EFF08D
:109010001FE02AC629C12286CA8523148100231293
:109020004101231331019770FE1FE780601F4C0040
:109030002685EFA07FB12A8411C532459770FE1FA7
:10904000E780800E2285B250225492540259F24990
:10905000624A456182804D44F5B7011122CC26CA8F
:1090600006CE4AC8DD472A84AE84638DF502814767
:10907000035504006C002306F100EFA07FB0054506
:10908000638EA40803458400B165938505B8EF900D
:109090004F94E5472301F400B7470100938767B772
:1090A0005CC0A5A8034755013149B28633062703A2
:1090B00018499C4232971043E31BF6FA83D74600C7
:1090C00003564700E315F6FA8C4608479770FE1FD3
:1090D000E780402249DD8347540103474401850767
:1090E00093F7F70FA30AF40063F0E704B3872703AD
:1090F000184803550400BA97984783D6470003D60B
:10910000270083D50700EFF07FEE35F1034584009B
:10911000B165938505B8EF90CF8B5945F240624415
:10912000D2444249056182808347640191B70111AD
:1091300022CC26CA06CEDD472A84AE84639CF5067F
:1091400003550500EFA08FC00356C40183562401C8
:10915000035744016D162A9642064182B307D64052
:10916000C207231EC400C18363F1E7089305C5FF4E
:109170003308F740635CB802BA96918EC206184C69
:109180008355040103550400C1823E97EFF01FE6AA
:1091900015E103458400B165938505B8EF906F83B1
:1091A0005945F2406244D244056182806D159316A0
:1091B0000501F1B78147035504006C002306F10057
:1091C000EFA01F9C0545E38EA4FC03458400B16518
:1091D000938505B8EF80FFFFE5472301F400B7470B
:1091E0000100938767B75CC065BF8547E9B73971F0
:1091F00026DAAE842C0022DC4AD84ED606DE2A8936
:10920000B28965232A8421ED4A85EFA02FB483D645
:1092100044006D1563C5A60093160501C1829844EC
:1092200003D6240083D504004A85EFF03FDC2A846E
:109230001DE53146A6850808230601009770FE1F2C
:10924000E78000FE83D724002245B74601004E8701
:10925000938646B05D466C00231EF10001272285EF
:10926000F2506254D2544259B259216182806FF057
:109270001FF86FF0DFF7797126D206D622D44AD0D4
:109280004ECE52CC56CA5AC88944C5C159CE2E8436
:109290002A89BA8A368B328AEFA04FAB93054400F5
:1092A0008147711503D705006352A70A850793F715
:1092B000F70FB105E318FAFE8A854A85FD21AA84D5
:1092C0002DE531453305AA02916593851570CD448E
:1092D0009770FE1FE78000D7AA8921C9314633065F
:1092E000CA02A2859770FE1FE78080F31844835658
:1092F000440003562400835504004A85EFF01FCF35
:10930000AA841DED0245B74601008547568793861E
:1093100046B05D464C002302F1004EC423064101D5
:10932000A306010023076101152DB25022542685A2
:1093300002599254F249624AD24A424B45618280B4
:109340004E859770FE1FE78020DEC5B7ED44F1BF64
:1093500079714ECE37D60300AE89C16526D201475A
:10936000AA848946130686FBFD15054522D406D638
:109370004AD0EF10501B054431CD2A891307300223
:1093800081461146F5452685EFF07FA82AC655444B
:1093900031C18357A900CE8601462314F1009147BD
:1093A0002315F10085472300F500B2472C002685E0
:1093B000A38007003247FD572301F7003247A3017E
:1093C000F700EF10100C2A8411C532459770FE1F6C
:1093D000E78080D52285B250225492540259F24936
:1093E00045618280411106C6EFF08FD619C5B240A3
:1093F00041011773FE1F670023D3B24041018280F1
:10940000011106CE2AC6EF905FFA3245B727002039
:1094100023AC07A4B727002023AE07A49145B727A4
:109420000020A388A7D6EF300060F24005616F20CE
:10943000103A7971939705014AD006D622D426D2E4
:10944000C187014963DE070AB727002003C517D784
:109450002E89EF80FF8B2A844DC1034705009307B7
:10946000000A6319F70885474C08A305F100EFA02F
:10947000EF80AA840DED8347610171476379F70896
:10948000138717FE1377F70F9306000263F8E608B9
:10949000858BD5CBB727002083A787A5994481CB9F
:1094A000035524001306B1004C088297AA84834711
:1094B000B10099C7084409C59770FE1FE780C0C670
:1094C00095E05247B7070001938707F07D8FB707F4
:1094D000120093870710630FF70003476101ED4700
:1094E000631AF700035524008545EF304048CD4707
:1094F0006388F4002285EF808FF5A1673349F90076
:10950000B25022544A8592540259456182803707ED
:10951000301405073357F700058B3DDB3727002054
:109520000327C7A549D70347510151F32306F1008B
:1095300099472308F100035524006C00231701000C
:10954000EFA04F98ADB7B727002083A7C7A59DC34D
:10955000035524001306B1004C08829729D9AA8428
:1095600083475101A9F7834761012308910023062E
:10957000F100D1B79944EDB7397122DC26DA06DE65
:109580004AD84ED652D456D25AD0A5472A84B2844D
:109590006399F5108347450203570600835A260056
:1095A00085072302F5029307F7FFB387FA025442B7
:1095B000C207C183B69703C9170083C70700834654
:1095C000C50022093369F90085476390F602330725
:1095D0005703231006008149014A130B3501931AE2
:1095E000070193DA0A0163E15907C167FD176302B6
:1095F000F90C83570401637EF90A05094209834681
:10960000C400135909012317240105470355040019
:109610009305E400639FE6002315F10093072030D3
:109620002316F10093078002231421012307F10080
:109630002C00EFA06FB503458400B165938505B894
:10964000EF803FB95945BDA083D62400DC40834557
:109650002401ED1613865900C206C1823E965A8532
:10966000EF903FDA05C9630C3A01C84003D62400E5
:10967000B305350152959770FE1FE78060BA83D716
:1096800024003E9A83D70400420A135A0A01850730
:109690002390F40083D72400BE99C20993D909010D
:1096A00099B703474600A9476310F702834745026D
:1096B00081CF0145F2506254D2544259B259225AD4
:1096C000925A025B2161828083462401130934018E
:1096D00037D503004A868945130505FBEF907FD2F5
:1096E00019C10545C1BF8346240137D503004A8609
:1096F0008945130545FBEF90DFD065F583462401CE
:1097000037D503004A868945130585FAEF907FCF48
:1097100069F98346240137D503004A868945130534
:1097200045F9EF901FCE55FD03C74400BD47E3EA5E
:10973000E7FAA56793874712B3D7E700858BD5D3A0
:109740008347440285072302F40203D9240071BD34
:10975000B727002003C687D7B727002003A707A68F
:1097600081476315F600814636858280BA861307E5
:109770008702835587FDE389A5FE850793F7F70FD9
:10978000CDB7011106CE2EC6EFF09FFC01CD834769
:10979000A500B245138717006396E50093F707F815
:1097A0002305F500F24005618280011106CE2EC628
:1097B000EFF01FFA05C5B24591C188C18347850006
:1097C0001307E00F5D456388E7001307F00F0145BD
:1097D0006383E7005945F240056182800945E5BF92
:1097E000411122C42A84210506C626C24AC0EFF0D0
:1097F0000FAC83472400A51793F7D70F91EB0347CE
:10980000C40085476310F7061C4881443149A9E329
:10981000FD5723010400A304F400230204021305EE
:10982000C4002244B240924402496146814541014C
:109830001773FE1F6700E3A5B38724033E95084511
:1098400009C59770FE1FE780208E850493F4F40FFE
:10985000834744010848E3E1F4FE9770FE1FE78068
:10986000A08C7DB7084C75F965B7411122C44164DD
:1098700006C626C29307E4FF630EF500AA8485E1BD
:10988000EFF01FED01E91305F4FFEFF07FEC19C1D4
:1098900023109500B24022449244410182808547C2
:1098A0006395F504EFF0DFEA2A846DD5FD572310A8
:1098B000F500834784001307F00F6385E702130761
:1098C000E00F638BE70083462400034594000147C3
:1098D0005146A685EFF0AF8F2285EFF07FF0FD5760
:1098E0002304F4002305040075B78947E394F5FACF
:1098F0008545EF40D02B59FD2685EFF07FE52A8482
:109900004DF949BF39C9034785009307F00F630636
:10991000F704011122CC06CE2A8483462500835504
:1099200005000345950001475D46EFF04F8A034768
:109930002400E1476319F700035504006C00230677
:109940000100EFA0EFA3F9572304F4002285EFF004
:109950003FE9F24062440561828082809307F00F04
:109960006306F706011122CC26CA2A844EC6AE84AD
:10997000B689AA859306850037A501004AC852C456
:109980003A89328A13054590794606CEEFF06F91F9
:10999000A3042401230144012322340185C01305BB
:1099A000C4006244F2404249B249224AA685D244E8
:1099B000614605611773FE1F67008386F2406244AB
:1099C000D2444249B249224A056182808280B72747
:1099D0000020238EA79882809547639CF5068347D5
:1099E0004502854685072302F50283570600584243
:1099F00003462600FD17C207C1836318D6048A07F1
:109A0000BA9703C7170083C707002207D98F0357E8
:109A1000E50063F9E704411106C622C48507231651
:109A2000F5002A849305C50003550500EF901FEC4F
:109A300003458400B165938505B8EF808FF9B24086
:109A40002244D9473E8541018280C946B387D70267
:109A500045BF83464600294785476396E60003478E
:109A6000450211C381473E8582809D476392F5067A
:109A7000834745028356E50085072302F502835795
:109A800006005842FD178A073E9783471700034791
:109A90000700A207D98F014763F6D704411106C614
:109AA00022C485072A842316F5009305C5000355B3
:109AB0000500EFF04FC403458400B165938505B8F8
:109AC000EF802FF1B240224459473A85410182800C
:109AD00083464600A94705476396F60003474502BB
:109AE000133717003A858280411122C406C626C268
:109AF000B5472A84639BF50483474502B2848507F2
:109B00002302F50203550500EF905FA483D70400FC
:109B10001307F5FF014563C5E7020357E40003554A
:109B200004009305C400BA972317F400EF90DFEA0E
:109B300003458400B165938505B8EF808FE95945E9
:109B4000B2402244924441018280034746009D472F
:109B50000545E317F7FE0345440213351500CDB75D
:109B6000C547639EF5068357060003572600FD1779
:109B7000B387E7020347450205072302E50258427F
:109B8000C207C1833E978347370003472700A207D8
:109B9000D98F41677D176395E70081473E858280B5
:109BA000138717002316E5000357E500E3F7E7FEE8
:109BB000411122C49305C5002A840355050006C639
:109BC000EF90FFEA03458400B165938505B8EF8007
:109BD0004FE0B2402244D9473E854101828083460E
:109BE000460029478547E39BE6FA0347450255F7B8
:109BF00075B7011122CC26CA4AC852C406CE4EC639
:109C000083C7250015472A8AAE8432843689639D2E
:109C1000E7043686A2852685EFF01FDCAA8955E980
:109C200085476318F40A03474900A9476301F7020F
:109C300003C594004A8785460146D285EFE03FD9A7
:109C400019E585454A85EFE0BFD01334150083C67A
:109C5000240003C5940001476946D285EFE03FD751
:109C60002685EFF0FFB751A01D476398E7003686C1
:109C7000A2852685EFF07FDF55B725476398E7007B
:109C80003686A2852685EFF03F8F49BF354763981A
:109C9000E7003686A2852685EFF01FE541B74547E8
:109CA0006398E7003686A2852685EFF07FEBBDB787
:109CB0005D47639FE70003C7C50085473686A285D9
:109CC0002685631DF702EFF04FB98547631BF50446
:109CD0008549A5476317F402835709009DE30544AE
:109CE000E38709F6D947E39DF9F62285F2406244FD
:109CF000D2444249B249224A05618280EFF02FC323
:109D0000E9B703C594004A87A2860146D285EFE0F1
:109D10001FCC71F5A2854A85EFE09FC3133415006F
:109D2000C1B70544D9B7397122DC06DE26DA4AD834
:109D30004ED652D456D283D705001944B1E783C911
:109D400025002A89328A938759FE93F7D70FAE846C
:109D5000DDE7B727002083C6C7991307F00F938A62
:109D6000C79919446382E602F5476394F904EFF05A
:109D70003F9EAA8921C10346A5000DCE93178601F7
:109D8000E18763DD070001442285F2506254D2541A
:109D90004259B259225A925A21618280F5454A8528
:109DA000EFE03FCB83C7A90093E707F82385F900CD
:109DB000D9BF814983D64400904483C5140003C5AC
:109DC00004003800EF90DFDC2A845DFD83C62400A8
:109DD00003C50A0038000146CA85EFE05FBF2A8448
:109DE00045F5B24799C323000A0083C7240075478D
:109DF000E39BE7F8E38909F82385F90071B7EFF0F1
:109E00003F95AA8A49D185476391F90A83D54400D1
:109E100088443000EF906FF52A843DF503C72A008F
:109E2000C54763F2E70ADD476301F70CB727002057
:109E300003C59A0083C717D7639CA70A014403C7C9
:109E40002A008D47631FF7048357810003D7CA0098
:109E500063F4E7002396FA0083D5CA004A85EFE051
:109E60007FF5B727002083D7C7B86D47637BF7021C
:109E700083D5CA005D476376B70213873500910525
:109E80006349F7001307B00FBE856374F7009305AD
:109E9000B00F1166C20513060629C1814A85EF80FD
:109EA000F0165685EFF0DF93C5B5834725001144C2
:109EB000E39C37ED5C41E38907EC83D5440088449B
:109EC0003000829791BFB72702009387072AB3D744
:109ED000E700858BA1DF03C624003400D6854A85C0
:109EE000EFF03FD12300AA0045B583A70A01DDB7F3
:109EF00083C6240038000146CA85EFE05FAD2A849E
:109F00001DFD83C524002800EFE09FA405D9230090
:109F10000A0035B7011122CC3724002006CE26CA0C
:109F20004AC84EC652C4930904D703C58900930793
:109F3000800291653305F50293856570372900200D
:109F4000930409A69760FE1FE780C00F03C689002F
:109F50009307800281453306F60288C09760FE1F92
:109F6000E78020339C404D45A1C3930404D71309D7
:109F700009A60144130A8002FD5983C78400636D5A
:109F8000F40237A50100130565D2EFE07FE13795B4
:109F9000010013052578EF902FCD37A5010013059B
:109FA000A586EF40E0370145F2406244D244424981
:109FB000B249224A05618280B307440303250900A0
:109FC0006146814505041374F40F3E952310350155
:109FD0002301050023143501230505002302050292
:109FE00031059760FE1FE780C02A41BF014582808E
:109FF000B727002083C697D7814763E5D70001477D
:10A000003A8582802E87910503D6C5FFE30AA6FE16
:10A010008507E5B70DCD834725000547890793F7E9
:10A02000F70F6376F702411122C406C62A848355CE
:10A030000500034535000147F9465D46EFE03F99CD
:10A04000F9572311F400B2402244410182808280FA
:10A05000B727002003C797D7FD56814763E3E70082
:10A0600082802310D5002301050085071105FDB767
:10A0700001458280372600201306B69A9307000216
:10A080002300F60037270020FD572305F79A3727CE
:10A090000020230FF79837270020A30EF798854557
:10A0A000B72700202394B79AB7270020239207A64A
:10A0B000B727002023A607A6B727002023AE07A6B0
:10A0C000B727002023A807A6B7260020B7D703008C
:10A0D0009386069A938747FADCC2B727002023832A
:10A0E00007A6B72700209387C79309472380E60078
:10A0F0002380E7002388E7002380E7022388E70224
:10A1000037D70300130787F9D4C7D8DBB7D60300C6
:10A110000D47238CE702938646F937270020D4CBDE
:10A12000032787A637D50300B7D60300130505FB21
:10A13000938686FBC8C32384B70023950700238C2E
:10A14000B700239D0700D0CFD4D3238407022395E3
:10A15000070223A60702239D0702D8DFB7270020A6
:10A1600037A701009387C7971307C72223A00700CB
:10A17000D8C323A407008280411106C6EFF05FE731
:10A1800011C503452500B240410182800145E5BF6C
:10A19000411122C426C24AC006C6AA842E8932842E
:10A1A000EFF01FE511E94165CA857D15EFF05FE429
:10A1B000C54711C523109500230185008147B24092
:10A1C0002244924402493E854101828029E7894820
:10A1D000354763931605011106CE22CC26CA0347E4
:10A1E00016000346060093C7F7FF2207598EF18F2A
:10A1F00032C68DE7C4452A84A685EFF0FFF73246C4
:10A200000147630FA60022856244F240A685D2442E
:10A2100005616FF0FFF72D473A858280130700082C
:10A22000F2406244D2443A850561828083C80500C9
:10A2300009486395080303A84500834718000348AD
:10A240000800A207B3E70701C2070D68C18713081A
:10A2500028906395070189476FF05FF70545828075
:10A26000011122CC372400201304E4990347040091
:10A2700006CE26CA4AC84EC69307F00F6300F704FD
:10A28000AA892945B2842E89EF709FA105C9930739
:10A29000100B2310F50023020500231135012313B1
:10A2A000250123149500AA85034504006244F24069
:10A2B000D2444249B24905616F709FADF240624499
:10A2C000D2444249B249056182804111B72700203A
:10A2D00026C2AE8483A587A622C406C62A84EFF0D0
:10A2E000BFE9098909C922852244B240A685924462
:10A2F00041016FF0EF85B24022449244054541018F
:10A300008280411122C426C24AC006C6AA84130410
:10A3100045001309850B835704009DC3084409C5F4
:10A320009760FE1FE78040E02285314681459760B7
:10A33000FE1FE78000F63104231A04FEE31D24FD0E
:10A34000B2402244FD572390F40002499244410157
:10A350008280B727002003C697D7B727002003A71E
:10A3600047A781476315F600814636858280BA8605
:10A370001307870B835587F4E389A5FE850793F7B9
:10A38000F70FCDB7B727002083A7C7A789CB03D77F
:10A3900047006314A700884782809C43C5BF0145DE
:10A3A0008280411106C6EFF0FFFD09C50845B240A5
:10A3B000410182800145E5BF011126CA9384450011
:10A3C00022CC4EC606CE4AC852C456C25AC02687B0
:10A3D00081490144814681473D450356070055CEDA
:10A3E000D9E20354470083572700B286A297C207D9
:10A3F000C18385093107E392A9FE25C82E8991659D
:10A400009385457022859760FE1FE780A0C32A8B45
:10A4100029CD814A014A8C4485C503D644003305C1
:10A420004B019760FE1FE780A0DF83D7440088447C
:10A430003E9A420A135A0A019760FE1FE780C0CE77
:10A4400063890A003146814526859760FE1FE780B3
:10A4500040E4850AB104E3E03AFD232669012314B0
:10A460008900054521A0630DD6000145F2406244F4
:10A47000D2444249B249224A924A024B0561828043
:10A4800003562700E313F6FE035647003294B297B3
:10A490004204C2074180C183A9BF0545E37835FD69
:10A4A000A9BFB727002083A707A799E301458280AA
:10A4B00098470357A7006315A700138547008280BC
:10A4C0009C43E5B7411106C6EFF0BFFD11C503552A
:10A4D0000500B240410182800145E5BF411106C639
:10A4E000EFF03FFC11C503452500B24041018280D9
:10A4F0004145E5BF411122C42A842E8506C6EFF0EE
:10A50000FFFDAA8505462285EF30304A9547630551
:10A51000F500BD476313F5002145B24022444101D7
:10A5200082804111B727002022C406C603A407A7D2
:10A530008146938707A729C018440356A7001840EF
:10A540006317A60285CA98C22E8581C92146930544
:10A5500044009760FE1FE780A0CC22859760FE1F15
:10A56000E78080BC0145B240224441018280A2863E
:10A570003A84D1B798C3C9BF0545F5B7372700203E
:10A580008327C7A701461307C7A7A9C703D8470052
:10A590009443631CA802011106CE22CC26CA0DCA20
:10A5A00014C2AA843E852E849760FE1FE780C0B740
:10A5B0002C002685EFF0FFF601E519C0B2471CC05C
:10A5C000F2406244D244056182803E86B68775BF00
:10A5D00014C3C1BF05458280411122C42A840905E4
:10A5E00006C6EFE0CFCCFD57A301F400B2402244F1
:10A5F00041018280B727002003C797D7B7270020E3
:10A6000083A787A72A86050781463E8583D707004B
:10A610006388C700850693076500E3E8E6FE014509
:10A620008280411122C4416406C626C29307E4FF1A
:10A63000630EF500AA8485E1EFF0DFFB01E9130565
:10A64000F4FFEFF03FFB19C123109500B240224404
:10A6500092444101828085476394F504EFF09FF9AD
:10A660002A846DD5FD572310F50083472400130776
:10A67000F00F6384E7021307E00F638AE7000345E6
:10A6800034000147F9465146A685EFE04FB42285D4
:10A69000EFF09FF4FD572301F400230204007DB77F
:10A6A0008947E395F5FA8545EF30705045F12685E9
:10A6B000EFF05FF42A8455F951BF1D71A6CACEC6CA
:10A6C00086CEA2CCCAC8D2C4D6C2DAC05EDEAE8400
:10A6D00083C52500F947AA896397F504EFF09FF138
:10A6E0002A8411ED01442285F6406644D644464949
:10A6F000B649264A964A064BF25B2561828083471B
:10A7000025000547890793F7F70FE37DF7FC03451D
:10A7100035000147F9460146CE85EFE04FAB228573
:10A72000EFF09FEBC1B703AB0400B70700019387BD
:10A7300007F037071200B377FB0013070710B28A40
:10A740000149638AE7022EC6EFF0DFEA2A89B245A3
:10A750001DC10346450005C293178601E187E3C387
:10A7600007F84E85EFE0EFAE8347490093E707F81F
:10A770002302F90085BF372A00200347AA9A9307CE
:10A78000F00F130AAA9A1944E30FF7F4E147E3EC38
:10A79000B7F493D71500FD1713973700B7D7030009
:10A7A0009387878FBA9703A80700E30E08F283AB5D
:10A7B0004700E38A0BF2420B135B0B0163050B00AE
:10A7C000C947E392F5F283D64400904483C5140050
:10A7D00003C50400380802982A84E31605F02C0803
:10A7E0004E85829B2A8421C983C71400E39D07EE0E
:10A7F00083C72400230AA10039472308F100639985
:10A80000E70262478347170003470700A207D98F73
:10A810000C084E852319F100EF80DFEAE30405EC14
:10A8200014080546D9454E85EFE08FC32A8465BDDF
:10A8300083578101F1BF83C624009147E384F6EA80
:10A8400003450A0038080146CE85EFE04F982A8478
:10A85000E31B05E883C524002808EFE06F8F19C1CA
:10A8600023800A009840B7070001938707F07D8F87
:10A87000B707120093870710E306F7E6E30409E63B
:10A8800083C724002302F900B9BD011106CE2EC6EC
:10A89000EFF05FD601CD83474500B245138717001F
:10A8A0006396E50093F707F82302F500F24005618F
:10A8B0008280B727002003A707A719E3014615A840
:10A8C0001C4703D8A700636B050183584700B38674
:10A8D00008016355D5008146639416011843F1BF02
:10A8E0003E86C10703D3A7FF6317A30099C1239036
:10A8F0000501328582808506C206C182F1BF3971A9
:10A9000052D42E8A4ED69305E101AA89528522DCC3
:10A910004AD856D206DE26DA328936C63AC4BE8A0C
:10A92000EFF03FF9054435C5AA840355E1013944E8
:10A93000EFF05FA539CD03284500630C08042247DA
:10A94000B246D6874A86A6854E8502982A8431E18A
:10A950009307E00F638FFA0203C704008947631A65
:10A96000F702D8408347170003470700A207D98F93
:10A97000C2070D67C18713072790639CE7008347D1
:10A98000190003460900D285A2075D8E4E85EFF0BF
:10A990003F8D2285F2506254D2544259B259225A04
:10A9A000925A21618280797122D4035425004ECEBF
:10A9B000AA89228556CA06D626D24AD052CC5AC86F
:10A9C0005EC662C4AE8AEFF0DF9801E92285EF909F
:10A9D0006FEF594429E90144B9A003C789008547AD
:10A9E000AA840144631AF702AA8513858900EFF04F
:10A9F000BF9C29CD03D7640083D68400D04483D57F
:10AA0000440003D52900E147EFF07FEFD9472A84BE
:10AA10006318F50223A604002685EFF09F8E49C037
:10AA2000D947E30AF4FA2285B250225492540259CB
:10AA3000F249624AD24A424BB24B224C4561828073
:10AA400061DD83D744002390FA00F9B713894400ED
:10AA5000014AB94B594C3D4B83550900D5DDE147BF
:10AA600063067A010357C90011C3D9470357290068
:10AA7000835649000326890003D52900EFF03FE8FB
:10AA80002A846319850123240900050A3109E31585
:10AA90006AFD59B77DD9835709002390FA00F5B7AD
:10AAA00003D529002DB701112317C1009307E00F2B
:10AAB0001306E1000147894606CEEFF05FE4F2405D
:10AAC00005618280797122D42A840355850026D2BB
:10AAD000AE849305210106D64AD0EFF09FDD6308CE
:10AAE000050E834785002AC693F707028DCF0355CD
:10AAF0002101EFF01F8BAA87B24501ED8357840037
:10AB000039452390F400B2502254925402594561C1
:10AB10008280035524004946829711C583578400DB
:10AB20002390F400CDB7035924004A85EFF07F82CB
:10AB300011ED41657D15EFF0DF8119E58357840044
:10AB400025452390F400C1B72310250113074500C4
:10AB50008147BD46035607002DE63147B387E7021C
:10AB6000130984003146CA8591073E959750FE1F10
:10AB7000E780006B3146CA8548089750FE1FE78082
:10AB8000206A0356C4000355240041478146DD4531
:10AB9000EFE0EFA72ACE19E58357840045452390BF
:10ABA000F40095B70C480356C4009750FE1FE78089
:10ABB0002067035524004C08EF908FCC29D55945C8
:10ABC00099B785073107E397D7F8254581BF054534
:10ABD000B1B7797122D42A840355850026D2AE8478
:10ABE0009305E1014AD006D63289EFF09FCC51C5DA
:10ABF0008347850093F70702A9E7034714019307EA
:10AC0000200519E3834744008356A400504483552C
:10AC10008400035524000147EFF07FCEAA8721E985
:10AC20008347140199E703552400EF908FC0D9475B
:10AC300011E18147B2502254925402593E85456138
:10AC400082802AC60355E101EFF0AFF5AA8705C956
:10AC5000B2450355240049468297AA8759DD035718
:10AC600084002390E4000347140161F7E1B75947DA
:10AC7000E317E5FE230009006DBF8547CDB7B9474F
:10AC8000F9BF397122DC4AD84ED652D406DE26DA14
:10AC9000AA892E8A32C63689EFF0DF95094415C598
:10ACA000834725001307E00FAA845D44638FE70004
:10ACB0001307F00F5944639AE700324605E2D28544
:10ACC0004E85EF900FC42A8415CD2285F250625430
:10ACD000D2544259B259225A2161828003550A0046
:10ACE0009305E101231F0100EFF0BFBC0355E10113
:10ACF000EFF0CFFEAA8505464E85EF30004B2A8443
:10AD00005DDDE1B79307F00FE301F9FC37A5010022
:10AD1000938624007946A68513054501EFD07FD898
:10AD2000A38124015DB73971B727002026DA83A4F7
:10AD300007A752D45AD05ECE62CC06DE22DC4AD8B7
:10AD40004ED656D266CA2A8BAE8B328C368A99E0A2
:10AD50008149B9A0804483DC44000149835AA4009E
:10AD6000631499018440E5B78357A400A28963F86E
:10AD7000670105094209135909014104D5B7E3EAFE
:10AD8000FBFE630C0A00834504004840D2866286BD
:10AD90003AC6EF800FE7324769DD19C32310570128
:10ADA000F25062544E85D2544259B259225A925AA4
:10ADB000025BF24B624CD24C2161828003D70500CA
:10ADC00083D62500854763E9E60439C7411183C668
:10ADD000450026C237D503009384550022C4268639
:10ADE0002E84130505FB894506C6EF808FE1C14718
:10ADF00011CD8346440083552400035504000147C8
:10AE00002686EFF05FF2814711E1A947B240224464
:10AE100092443E85410182803E8582802E86035584
:10AE2000060083D52500854763E2A50205C1834658
:10AE3000460041110147150606C6EFF0DFEE8147D7
:10AE400011E1A947B2403E85410182803E85828062
:10AE50002E860355060083D52500854763E2A502AB
:10AE600005C18346460041110147150606C6EFF0AD
:10AE70009FEB814711E1A947B2403E8541018280A5
:10AE80003E85828039714ED683D7250083D905004F
:10AE900006DE22DC26DA4AD852D456D25AD05ECE0A
:10AEA00062CC66CA6AC863E037198547638E0914A5
:10AEB000416BAE8A2A8A2314010002C6014401496B
:10AEC0007D1B894B054CC94C054D83D52A00014794
:10AED000814601464E8523130100EFF0DFE4AA848A
:10AEE0006300051209EC13072002930661005A86DD
:10AEF00095455285EFD0BFF12A84630805120357A8
:10AF0000810083C7040045C70347A100630CA7075E
:10AF100041476385E7022C005285EF807FDF09CD32
:10AF200034001546D9455285EFD09FD311C532451F
:10AF30009750FE1FE780401F8147F9A083D7A400E8
:10AF40004146130524002300F40083D7A400A18305
:10AF5000A300F400CC409750FE1FE780602C49040A
:10AF6000835781008507C207C1832314F10063F969
:10AF7000270983D7A400638567098509C20993D986
:10AF80000901A1B7E39977F983D7A400094613050E
:10AF900024002300F40083D7A400A183A300F400BD
:10AFA000CC409750FE1FE780A027110455BF22C652
:10AFB0000359610003C7A4001305240063827703CB
:10AFC00033599903230571012300E40083D7A400BA
:10AFD0004146A183A300F400CC401379F90FA5BF2B
:10AFE000230581012300E40083D7A400135929001D
:10AFF0001379F90FA183A300F4000946CC4055B79B
:10B000008357810089FBA947F2506254D2544259B8
:10B01000B259225A925A025BF24B624CD24C424DC8
:10B020003E85216182808547C5B7C547F1BFB727F7
:10B03000002003C7A7A8854763F3E706011122CCC8
:10B0400026CA4AC806CE2A843289AE84EFF08FDA47
:10B0500001C9034725009307E00F5D456308F7002A
:10B06000631C0900A6852285EF908F86F24062441A
:10B07000D24442490561828003D504009305E10072
:10B0800023170100EFF0FF820355E100EFF00FC539
:10B09000AA8505462285EF30401169D5C1BF5945C3
:10B0A000828013F7050201C7B2856FF0AFC441116A
:10B0B00026C24AC006C622C413F98500AA846317B3
:10B0C0000900139785016187635D07023285368425
:10B0D000EFF0CFC0AA850546631309000146268517
:10B0E000EF30A00C01E90145B240224492440249EC
:10B0F0004101828083479400E5DB83478400E5F7C4
:10B10000E5B793F72500E5F30D45F9BF7971AE86F4
:10B1100022D42A8403D506009305E10106D636C65B
:10B12000EFF02FF909CD83458500B2460356E101C2
:10B130002285EFF01FF7B250225445618280054509
:10B14000DDBF13F7050201C7B2856FF0AFBA411139
:10B1500022C426C206C693F485002A8491E413977C
:10B1600085016187635007023285EFF02FB7AA850A
:10B17000054691E0014622852244B24092444101B5
:10B180006F30A00293F72500014591E30D45B240D1
:10B1900022449244410182807971AE8622D42A846D
:10B1A00003D506009305E10136C606D6EFF06FF031
:10B1B000B24601CD834585000356E1012285EFF0BB
:10B1C0005FF8B2502254456182800545DDBF797138
:10B1D00026D2AA840355A500C16722D44AD04ECEF8
:10B1E00006D623170100FD173284B6890149630D85
:10B1F000F500050583C60400D04042051307E100B1
:10B200004181EFF05FB22A8983C60400D04037D570
:10B2100003008945130505FBEF80AF9E1DC503D4D0
:10B22000A4002285EFF00FAA09C57D142A944204D8
:10B2300041806384090023908900B25022544A85DA
:10B2400092540259F2494561828083C60400D0407D
:10B2500037D503008945130545FBEF808F9A61F1CF
:10B2600083C60400D04037D503008945130545F94E
:10B27000EF802F9919C9E30609FA8357E100E39299
:10B2800087FA0354A9007D145DB703D4A40055B711
:10B29000397122DC26DA4AD84ED652D456D25AD048
:10B2A00062CC06DE5ECEBE8983C785002A8AAE8464
:10B2B000C18B328C36843A89C28A468B9DE783CB18
:10B2C00004008947638BFB046285EFF0AF8B1DC1DF
:10B2D00083280500638008025A88D6874E87CA866D
:10B2E0002286A6855285829839A03285EFF06F8B31
:10B2F000AA8711ED3945F2506254D2544259B259DD
:10B30000225A925A025BF24B624C2161828029469A
:10B31000A6855285829745D5F9BFD8408347170047
:10B3200003470700A207D98FC2070D67C18793069D
:10B3300007906384D72263CEF60693062780638E38
:10B34000D70C63C1F60213070780E3CFE7F62D455C
:10B35000E39309FADC4403C60700CC432310C90079
:10B36000228569A213073780E390E7F62D45E39421
:10B3700009F885472310F900DC44814583C707009D
:10B380002300F40003D5A400050542054181EFF038
:10B390004FD2835709006317051291072310F90054
:10B3A00011468145130514009750FE1FE78060EE9B
:10B3B00029A2930627906383D71863CED7129306EA
:10B3C0003790638CD71813074790E39FE7EE2D451E
:10B3D000E39309F2DC441D472310E90003C707008B
:10B3E0002300E40003C71700A300E40003D72700ED
:10B3F0002301E40003D727002183A301E40003C74E
:10B4000047002302E40003D76700A302E40083D7C8
:10B410006700A1832303F4004DA02D45E39D09ECB3
:10B42000DC446C0083C9170003C70700A209B3E915
:10B43000E90011472310E90083C707004E85230068
:10B44000F400DC4483C71700A300F400EFF06FC6DC
:10B45000AA8435C50356C100C1659306E100FD15F8
:10B460008329C500EFF0BFD619ED83C60400D04094
:10B4700037D503008945130545FBEF709FF801E5BB
:10B48000FD572317F10003C7090089476310F7022E
:10B4900083A549000946130544009750FE1FE78025
:10B4A00020D88357090089072310F9008357E1004A
:10B4B0002301F400A183A301F40001452DBD23174E
:10B4C0003101EDB7034705008907BA972310F9004A
:10B4D0008357A500A300F4008357A500A18323018F
:10B4E000F400034605004C41130534009750FE1F3D
:10B4F000E78000D3D9B7C8449750FE1FE78080DCAF
:10B5000093170501C1832A871D45E3E637DF639959
:10B51000F90023100900CC4403560900CE9589B5E3
:10B520004207B3863A01418363C7E600B3873741D8
:10B530002310F900CDB723105901F1BF2D45E39C2D
:10B5400009DACC445285EFE03FC323107901230090
:10B55000A4002181A300A4008DB72D45E39D09D847
:10B56000DC442310790183C707002300F400DC4486
:10B5700083C71700A300F40089B71D71CAC82A89C0
:10B5800003552500A2CCCEC6D2C4D6C2DAC05EDE38
:10B5900062DC66DA6ED686CEA6CA6AD8AE8AEF704C
:10B5A000FFFA130CF5FF93170C01B72B0020C18392
:10B5B0002A8A814913840BCE3EC6372B0020B72C34
:10B5C0000020C16D8357C90063F6F900835704005A
:10B5D00063CC87010355290093850BCEEF80FF993B
:10B5E0002A8D15CD594D25A8832789001397190059
:10B5F0009305E101BA9783C4170083C70700A2042B
:10B60000DD8C2685EFF0EFAAAA8515E923909A0034
:10B610004840054D09C59750FE1FE780E0B0F64051
:10B6200066446A85D6444649B649264A964A064B38
:10B63000F25B625CD25C425DB25D25618280324821
:10B640008348490083A6CCA60356E101035529008F
:10B65000814713074BA6EFF0BFC32A8D1388CCA6F2
:10B6600009C523909A00484075B75C4085E70355AB
:10B670002900514781461386FDFFBD45EFD02FF9C4
:10B68000B727002048C01388C7A609E523909A0071
:10B69000454D71B78357040003574BA693044BA63F
:10B6A0003E976347470113C7F7FF52972390E40083
:10B6B000484003D60400832508003E95850997502D
:10B6C000FE1FE780E0B58357040003D70400C209DA
:10B6D00093D90901BA972310F400EDB5397122DC32
:10B6E0002A840355250006DE26DA4AD84ED652D4DF
:10B6F0005AD05ECE62CC66CA2E8B56D26AC8EF7024
:10B70000FFE42A8A8346C4008355A40003558400BD
:10B7100078001306D400130CBAFF651AEFF0AFE0FF
:10B72000420A37290020AA898144135A0A01B72BFB
:10B730000020B72C0020130909CE6386090463D4C6
:10B740008405938ACCA68348440083A60A00035646
:10B75000C100035524005288814713874BA6CE852C
:10B76000138D4BA6EFF0DFB215C5814A0356C10019
:10B770008355A4004E859306E100EFF05FA5AA89EA
:10B78000639D0A065DF9E5E083578400294523108F
:10B79000FB0089A083570D0003560401E317F6FC54
:10B7A00083A50A0048489750FE1FE780A0B455DDE6
:10B7B00083274900A1E3035524004166454781469C
:10B7C0007D169D45EFD0AFE405E5835784004545E0
:10B7D0002310FB00F2506254D2544259B259225AFB
:10B7E000925A025BF24B624CD24C424D21618280F4
:10B7F0002322A90083DAA90095BF83274900A697D1
:10B80000238057019387140013970701832749006A
:10B81000418393DA8A00BA97238057011387240063
:10B820008326490093873400420791044183C2076D
:10B83000C204C183C180369711CD8356E100230035
:10B84000D70003274900BA970357E10021832380DB
:10B85000E700E5B5FD562300D70003274900BA9756
:10B860002380D7000DB703552400B7250020898019
:10B87000239095CE938505CEEF802FD621DD5945B7
:10B8800091BF411122C406C693F705012A8432856F
:10B8900085C3EFE0BFC4AA8505462285EF20F010DE
:10B8A00095476305F500BD47631DF502214515A8C1
:10B8B00093F7450099CBEFE07FC20546AA85228524
:10B8C0002244B24041016F20500E93F7050489C70E
:10B8D000EFE0DFC00146DDB713F5150013351500A5
:10B8E0000605B24022444101828079714AD04ECE91
:10B8F00052CC06D622D426D22A8AAE89014983D7D1
:10B9000049006364F9000145A1A083A7090013144D
:10B910001900930414003387970003470700A29788
:10B9200003C5070022079305E100598DEFE07FF87A
:10B9300005E983A7090005453E94034704002380D9
:10B94000E70083A70900BE9403C70400A380E700B3
:10B95000B250225492540259F249624A456182809F
:10B96000834585000356E1005285EFF09FF105C144
:10B9700083A709003E94034704002380E70083A7C0
:10B980000900BE9403C70400A380E700D1B70509EE
:10B99000420913590901A5B7011122CC2A8403D504
:10B9A00005009305E10006CEEFE0BFF001CD834531
:10B9B00085000356E1002285EFF0BFECF2406244BF
:10B9C000056182800545DDBF1D71CAC82A890355FE
:10B9D000250086CEA2CCA6CAD2C4D6C2DAC05EDE0C
:10B9E00062DC66DA2E8ACEC66AD86ED6EF701FB6D3
:10B9F0002AC68346C9008355A900035589007808E3
:10BA00001306D900EFF02FB2B247B7240020416BE4
:10BA1000938AA7FFC20AAA8B014493DA0A01372C42
:10BA20000020B72C0020938404CE7D1B63860B1866
:10BA30000356C10183C58B0003552900EFF07FE455
:10BA4000AA8D631605168348490083A6CCA6035623
:10BA5000C101035529005688814713074CA6DE858E
:10BA6000EFF01F83AA8D93094CA6138DCCA663100B
:10BA7000051429C003D7090083D724001107639751
:10BA8000E7003247A2976D1763CAE706B725002083
:10BA9000938705CE03D7270003552900938505CE4C
:10BAA0003354E40223908700EF80AFD0AA8D15C1F4
:10BAB000D94D05A003552900494781465A86C545F9
:10BAC000EFD0EFB4C8C015E583D7AB00C54D231048
:10BAD000FA00F64066446E85D6444649B649264A81
:10BAE000964A064BF25B625CD25C425DB25D2561B8
:10BAF000828083D7090091072391F400DC4003D7AB
:10BB0000AB009306E101A2972380E700930714009E
:10BB100013970701DC4041835E85BA9703D7AB00DA
:10BB200021832380E7000356C1018355A900EFF06C
:10BB30000FEAD440130724000356E1014207418372
:10BB400036972300C700D84093073400C207C1834B
:10BB5000BA970357E101AA8B110421832380E700E0
:10BB6000C8404204418003D6090083250D00229578
:10BB700063950B029740FE1FE780806A83D7090018
:10BB80003E9442044180E31304F08357890023105C
:10BB9000FA00E3900DF4A94D2DBF9740FE1FE780FA
:10BBA000206883D709003E944204418041B583D781
:10BBB000AB002310FA00C1BF814DF1B75D71A6C281
:10BBC000CAC0AA840359850003552500A2C44EDECD
:10BBD00052DC5AD85ED662D466D286C656DA6AD0AD
:10BBE0006ECE2E8BEF709F96930BD5FF7115131AA7
:10BBF0000501B72900200144135A0A01372C0020FF
:10BC0000B72C0020938909CE6359741583C6C400EC
:10BC100083D5A4001307E1001386D4004A85EFF012
:10BC20008F902A8D630B05120359A500834585006B
:10BC30000356E10003D52400EFF0BFC463140512DE
:10BC400083C8440083A6CCA60356E10003D5240094
:10BC50005288814713074CA6EA85EFF06FE3930DF6
:10BC60004CA61388CCA6631F050E1DC883D70D00F4
:10BC700003D729008907630CF706B725002013872F
:10BC800005CE8357270003D52400938505CE335472
:10BC9000F40223108700EF800F9E15C5594525A09B
:10BCA00003D5240041664D4781467D16A545EFD05A
:10BCB0000F96B727002023A2A9001388C7A61DE16D
:10BCC00023102B014545B640264496440649F259B7
:10BCD000625AD25A425BB25B225C925C025DF24DC8
:10BCE0006161828083D70D0089072391F90083D792
:10BCF0000D00A29763D3770783A749000357AD00D0
:10BD0000930A2400A2972380E700050493170401F7
:10BD100003A44900C183C20A3E948357AD00832522
:10BD2000080093DA0A01A1832300F40003A5490067
:10BD300003D60D0056959740FE1FE780604E03D452
:10BD40000D00C167FD17569442044180E30EF9EAE5
:10BD5000050942091359090145BD294519FC23105C
:10BD60002B0195B76DDC11BF8357050081E789472B
:10BD70003E858280411126C2444122C406C64AC083
:10BD800083C60400D0402A8437D5030089451305B3
:10BD900005FBEF700FE719C9834724002547E51716
:10BDA00093F7F70F6377F702E14729A883C60400EA
:10BDB000D04037D503008945130545FBEF706FE48C
:10BDC00061FD8947B2402244924402493E854101C7
:10BDD0008280372900208356899A85471309899ADA
:10BDE000F5D2035704003697C166E3CDE6FC9165B2
:10BDF0009385257031459740FE1FE780A024AA84D3
:10BE0000CD4769D1314681459740FE1FE7806048A4
:10BE1000835704008355090001460147B386E500B6
:10BE2000C206C182636BF702AE97C207C18319C213
:10BE30002310F90023A004002146A28513854400A5
:10BE40009740FE1FE780C03DB7270020938707A7D4
:10BE5000984311EF84C38147B5B75040131547008D
:10BE600005072A962315D60005464DBF3E871C437D
:10BE7000F5FF04C381BF011106CE22CC26CA4AC8F1
:10BE800009E98944F240624426854249D244056169
:10BE900082802AC62A84280036892314B10023050B
:10BEA000C100EFF07FECAA8471FDE30D09FC83571C
:10BEB000A400E1DB91659385557031459740FE1FE5
:10BEC000E780401815C58357A400232005002324CC
:10BED00025012312F500B72700209387C7A79843B1
:10BEE00001E788C345B73E871C43F5FF08C359BF28
:10BEF000CD4449BFB7270020938767A603C7070033
:10BF000015E305472380E700058909CDB726002002
:10BF1000372500209386C697414691451305C59362
:10BF20006FF07FF501458280B7270020238FA79807
:10BF30008280C167FD176315F5002E856FE04F9174
:10BF4000411106C6EFE0CF8A11C5FD572310F50059
:10BF500023010500B2404101828001114AC806CE8A
:10BF600022CC26CA85472A896393F5044A85EFE0E7
:10BF70004FBE39E9C16437D603009385F4FF130738
:10BF8000E1008946130686F90545EFE0DFD92A84EA
:10BF9000FD140DC44C444A85EFF0BFF90356E1008F
:10BFA00022858146A685EFF08FA22A84DDB78947D6
:10BFB0006396F5008545EF20803F4DD9F2406244FD
:10BFC000D244424905618280EFE0AFB365B7011109
:10BFD00026CAB7240020938404D722CC03C594003A
:10BFE00037240020130444A7B72700203727002058
:10BFF00006CE4AC84EC62320040023AC07A623243D
:10C0000007A649C9138987A79307200C3305F502B2
:10C01000916593851570930987A61905420541819D
:10C020009740FE1FE780000203C694009307200C90
:10C0300081453306F60208C019069740FE1FE780C7
:10C0400040251C4003C7940081459386870B7D558E
:10C0500063ECE5069306800BB306D7020146FD5557
:10C060000507B6972320F900BE862390B600A3816A
:10C07000B6002381B6002382060005069906E36612
:10C08000E6FEF9562390D70099463307D702BA97B0
:10C0900023A0F90037A501001305A56BEFC0FFD061
:10C0A00037B501001305A588EF70AFBC37A50100B7
:10C0B00013052562EF20C026F2406244D244424973
:10C0C000B2490145056182802394A6F41386C6F423
:10C0D00023100600232406003106E31BD6FE850547
:10C0E0009386860BB5B7411106C622C42A84EFC0D9
:10C0F0000FADEFD03FF8B7270020A38E8798B72762
:10C10000002003A587A6EFD0BFF4B7270020238522
:10C11000879A2244B24037C501001305A5F54101B5
:10C120006F20002093970501C18763D30734B72799
:10C13000002003C5D799797122D45AC806D626D2D1
:10C140004AD04ECE52CC56CA2E8BEF507FBC2A849A
:10C1500029C9034705009307000B6311F704B724AF
:10C16000002085479384C4A6A304F1009C402315B6
:10C170000100A9E7EF00007F916593853570974036
:10C18000FE1FE78020EC88C015E98347910099C71E
:10C190008345440013058400EFD0CFA42285EF50DF
:10C1A0001FABB250225421653345AB009254025963
:10C1B000F249624AD24A424B45618280372A0020C6
:10C1C0006146814513050ACE9740FE1FE780600C4B
:10C1D00003494400894793040ACED289930A0ACEC0
:10C1E0006314F906EF0000782390A400035524009F
:10C1F00093050ACEEF705FAD0357240083D7040088
:10C200008356840011ED63E4F6002314F400835593
:10C2100084003A85EFC01FBA2285EFC07F8CB5B786
:10C2200063E4F6002314F40083578400D945938611
:10C2300009CE0D463A852390FA00EFC07FA28D45C6
:10C2400061DD138509CED1A09947631AF9029305E0
:10C25000A1002285EFF08FC8AA845DDDD9476396DF
:10C26000F40E0509035524001379F90FD945938677
:10C2700009CE4A86EFC0DF9ECA8559DDD9B7A147EE
:10C280006318F9009305A1002285EFF03F93E9B709
:10C29000A947631FF906035584006C00EFE06FE1C6
:10C2A0002A89630D05140355240041669306E100B5
:10C2B00055477D16AD45EFC09FB5C8C0AA8649C198
:10C2C000834844000358E1000356C100035524008D
:10C2D000814713070ACECA85EFE09FFBAA84631E3D
:10C2E000050E0355240093050ACEEF70BFBE0DD591
:10C2F0000355240093060ACE2D46D945EFC05F961C
:10C30000E30C05F0AD4513050ACEEFD0AF8D29B78C
:10C31000B147631BF90E035584006C00EFE06FD941
:10C32000AA8469CD0355240041669306E10059476C
:10C330007D16B545EFC0BFAD23A2AA00AA8629E9A4
:10C3400083578400C5442315F10003471400D147E7
:10C35000E304F7EC8347440003552400938509CE9A
:10C360002380FA008357A10023829A002391FA00C8
:10C37000EF704FB5E30205EA03552400938609CE1A
:10C380000546D945EFC0DF8DE30805E8854555BD75
:10C39000834844000358E1008357A4000356C100BA
:10C3A00003552400A68513070ACEEFE07FEEAA848A
:10C3B0000DE50355240093050ACEEF707FB7E30D1A
:10C3C00005E403552400D94593060ACE3546EFC04F
:10C3D0003F89B545E30205E4ADB5D9476393F40061
:10C3E000814403A54A009740FE1FE780E0D3E38520
:10C3F00004E2835784002315F10081BF8357840032
:10C4000085442315F10091B7B9476318F9009305E6
:10C41000A1002285EFF06F9681B5C1476318F9003E
:10C420009305A1002285EFF02FDA3DB5C947631AC5
:10C43000F900130691009305A1002285EFE06FF942
:10C4400021BDD947631DF9009305A1002285EFE0C6
:10C450006FE7AA84E31405E0A304010075BBE1477C
:10C46000E31CF9DA9305A1002285EFE0CFD3EDB309
:10C4700001458280EDC2011152C42E8A854522CC2D
:10C480004EC656C206CE26CA4AC8AA8AB689328481
:10C49000EF10F071D1471DC5B727002037270020C6
:10C4A00083C787A8834697A8814419E0B684BE86CF
:10C4B00037270020032707A893974400BA9763ED16
:10C4C000D400D547F2406244D2444249B249224A9C
:10C4D000924A3E85056182803E89C10703D727FFC6
:10C4E00009C7850493F4F40FD9BF25C095659385DA
:10C4F00025C0130500029740FE1FE780A0B4232645
:10C50000A90061D113060002814593840404974079
:10C51000FE1FE78000D82311990023000900231390
:10C5200059011DC43727002083479400032607A91B
:10C530002304F900118C8327C90011841180238EF4
:10C54000870023A029018147B5BF23260900F1B741
:10C5500023044901FDB785473E858280B727002027
:10C5600083C587A8B727002003A707A8814763953D
:10C57000F50081463685828003562700BA8619C2A7
:10C58000E30AA6FE850793F7F70F4107CDB7B72754
:10C59000002003C687A8B727002003A707A8814764
:10C5A0006315F60081463685828083552700BA865A
:10C5B00089C583454700E388A5FE850793F7F70FF4
:10C5C0004107F9BFB727002083C5B7A8B7270020C8
:10C5D00003A707A981476395F500814636858280C8
:10C5E00003560700BA8619C2E30AA6FE850793F729
:10C5F000F70F4107CDB7B727002003C897A8B72783
:10C60000002083A707A801476315E8008146368507
:10C61000828003D62700BE8619CA03D66700631836
:10C62000A600D04709C603562600E302B6FE05075A
:10C630001377F70FC107C9BF411122C4404526C275
:10C6400006C6AA8415C0484409C59740FE1FE78066
:10C65000A0AD484809C59740FE1FE780E0AC2285A1
:10C660009740FE1FE78040AC2685414681459740B4
:10C67000FE1FE78000C2B2402244FD57A384F400AD
:10C68000924441018280011122CC2A840355250065
:10C6900006CE2EC6EF10901A324622858145EF0055
:10C6A000F07222856244F24005616FF0FFF80DC51B
:10C6B00003572500411122C406C62A8411CBDD454B
:10C6C000EF00B07422852244B24041016FF0DFF6E2
:10C6D000B2402244410182808280411126C2B1468B
:10C6E0009304C5FFB386D402B7270020138787CFF2
:10C6F00006C622C436978356A7006398B6024843FD
:10C700000DC5138487CF9307F00F6306F6008347A8
:10C710000500639CC7009740FE1FE780E0A0B1477B
:10C72000B387F402A29723A20700B24022449244A6
:10C7300041018280411122C42E8426C24946AA8426
:10C740008145228506C69740FE1FE78080B4A5C0BC
:10C7500083C7C40113974700B727002083A707A901
:10C76000BA9703D707002310E40003D7270083D725
:10C7700067002311E40037270020035767A823121E
:10C78000E40003D704002313E40003D72400231498
:10C79000E40003D744002315E40003D76400231604
:10C7A000E40003D784002318F4002317E400B24008
:10C7B0002244924441018280B727002083C587A884
:10C7C000B727002003A807A9B727002003A607A8BA
:10C7D000014781476394E5003E85828083460600D9
:10C7E00081CE544691CA83C6C6019206C29663158D
:10C7F000D500850793F7F70F05071377F70F410665
:10C80000D1BF130600643386C50293069500AA853E
:10C8100037C501001305E56A6F509FC6411122C458
:10C8200006C62A8403459500EF50DFE0FD57A304B8
:10C83000F400B240224441018280011122CC4AC856
:10C840004EC652C456C25AC006CE26CA2A89AE89DE
:10C850000144372A0020B72A00201D4B83479AA89D
:10C860006365F40463990902B7290020372A002080
:10C87000930AF00F83C789A86367F4061144A144A3
:10C880002285050442041306F00FCA854180EFF0AB
:10C89000DFE4E31794FEF2406244D2444249B249D5
:10C8A000224A924A024B0561828083A70AA8931408
:10C8B0004400BE9483C704009DC383D76400639083
:10C8C00027036396690103D52400EF10207726859E
:10C8D0004E868145EF00904F2685EFF0FFD5050489
:10C8E0001374F40FA5BF83270AA893144400BE94C1
:10C8F00083C704009DC383C794006380570383D715
:10C900006400639C27012685EFF05FF12685D14501
:10C91000EF00B04F2685EFF03FD205041374F40FFB
:10C9200091BF41677917630BE502411122C406C626
:10C9300085472A846399F50022852244B2408145C7
:10C9400041016FF09FEF89476396F5008545EF1031
:10C9500010267DD1B24022444101828082809D45D3
:10C960006FF0BFEDB727002003D567A88280B727F7
:10C97000002003C747A8011106CE2317A1002316E4
:10C98000B10085476318F70070009305E100054585
:10C99000EF509068F24005618280A947631CF6045D
:10C9A00083C7150003C70500A207D98F2310F50020
:10C9B00083C7350003C72500A207D98F2311F500CF
:10C9C00083C7550003C74500A207D98F2312F5007E
:10C9D00083C7750003C76500A207D98F2313F5002D
:10C9E00083C7950003C78500A207D98F2314F500DC
:10C9F000014582800545828091476314F60283C712
:10CA0000150003C70500A207D98F2310F50083C7BF
:10CA1000350003C72500A207D98F2311F500014572
:10CA20008280054582809387C5FF93960701C18266
:10CA30000D476360D70231473387E702B7270020ED
:10CA4000938787CFBA972381A7002390B70001452A
:10CA50008280094582809306402037270020AA87DC
:10CA600063F4A60093074020F1172313F7A8B72714
:10CA700000202385B7A8B72700202386B7A8828087
:10CA80001905956542054111938535C0418106C65A
:10CA90009730FE1FE780005B11C5B240E9554101A8
:10CAA0006F50AF93B24041018280B72700202385A9
:10CAB00007A8B727002079710547238207A8B72761
:10CAC0000020A382E7A852CCB7270020372A0020F5
:10CAD00022D426D24AD037240020B7240020238D28
:10CAE00007A837290020B7270020130ABAA806D6BE
:10CAF0004ECE2AC6230404A8A38404A8239307A81F
:10CB0000232009A823000A00EF10005C3245B72754
:10CB1000002013060003238AA7A837250020130549
:10CB200085CF8145B72900209730FE1FE7806076CA
:10CB3000938989A903C50900130484A8938494A840
:10CB4000130909A805CD9565938545C01205973051
:10CB5000FE1FE780204F372700202328A7A819CDE4
:10CB600003C6090083C7190081452300CA001206C5
:10CB70002380F4009730FE1FE780A071B7270020C4
:10CB800003C587D783C704009565938555C03E9537
:10CB90001375F50F2300A40012059730FE1FE780E0
:10CBA000604A2320A90049C50346040081451206B6
:10CBB0009730FE1FE780E06D0327090083460400DD
:10CBC000814725077D56639EF604EF10C074B14778
:10CBD0003305F5029565938565C04205418197301F
:10CBE000FE1FE7802046B727002023AEA7A82A848F
:10CBF00001CDEF10407231463306C50281452285D2
:10CC00009730FE1FE780E0682254B25092540259D8
:10CC1000F249624A37D501001305259245616F102C
:10CC2000207085072300C70093F7F70F410761BF06
:10CC3000230004002380040049BF4111939705019C
:10CC400026C206C622C44AC0C187AE8463D3070A7F
:10CC500037290020034549A9130949A9EF504F8BF3
:10CC60002A8429CD03470500930700096315F704BB
:10CC700003471500CD47631CF706B726002003487D
:10CC8000250003C5B6B8372700208347A7A8130699
:10CC90006400814581461307A7A8AA886318D802B3
:10CCA00099C12300F7008347070091C70345090096
:10CCB0008545EF50CFC82285EF407FF92165258D4E
:10CCC000B2402244924402494101828083450600D9
:10CCD000AE9793F5F70F93F7F80F63F4A50093F76A
:10CCE000F50F850693F6F60F0906854545BF012D1C
:10CCF000D9B793F715000145E1D7EF00107009CDC2
:10CD0000B727002083C7A7A881CBB727002003C57A
:10CD100047A98545EF50AFC213C5140055B78546E6
:10CD20002A8763FBC60483C7150003C60500A20754
:10CD3000D18F2310F500639CD70083C7350083C6CD
:10CD40002500A207D58F2311F50001458280894671
:10CD500001456394D70283C7350083C62500A20727
:10CD6000D58F2311F70083C7550083C64500A2075E
:10CD7000D58F2312F7008280054582809147631486
:10CD8000F60283C7150003C70500A207D98F231039
:10CD9000F50083C7350003C72500A207D98F2311EB
:10CDA000F500014582800545828091476314F602B3
:10CDB00083C7150003C70500A207D98F2310F5000C
:10CDC00083C7350003C72500A207D98F2311F500BB
:10CDD0000145828005458280A1476314F60483C71C
:10CDE000150003C70500A207D98F2310F50083C7DC
:10CDF000350003C72500A207D98F2311F50083C78B
:10CE0000550003C74500A207D98F2312F50083C739
:10CE1000750003C76500A207D98F2313F5000145EC
:10CE20008280054582808947631CF60083C7150010
:10CE300003C70500A207D98F2310F50001458280A2
:10CE4000054582808357260079714ECE06D622D4BE
:10CE500026D24AD01307F007AE896372F70209475A
:10CE60003AC42316F100300093F5F50FEF10E01BE4
:10CE7000B250225492540259F249456182800357BC
:10CE80004600D9462A89328463F8E6008357660053
:10CE900063F4F6006379F70023140100300093F582
:10CEA000F90F4A85E1B70355060002C4EFF08FF190
:10CEB000AA8459C1EFF05F9083C784006369F500CD
:10CEC0001146A246CE854A85EF10A00B55B7340017
:10CED00026869305F00F4A85EFF0CFD975F1A2476A
:10CEE00003578400DC472390E70003572400239175
:10CEF000E700035744002392E7000357640023939D
:10CF0000E70003D744002394E700DC4485CB93F487
:10CF1000F90F2286A6854A858297C167FD172A8662
:10CF2000E311F5FA22459947F9452300F50023025C
:10CF30009500EFF01F8D2DBF094661B7014651B72F
:10CF4000A947631CF60483C7150003C70500A207A1
:10CF5000D98F2310F50083C7350003C72500A2072A
:10CF6000D98F2311F50083C7550003C74500A207D9
:10CF7000D98F2312F50083C7750003C76500A20788
:10CF8000D98F2313F50083C7950003C78500A20737
:10CF9000D98F2314F500014582800545828083C71F
:10CFA00005002300F50083C71500A300F50083C723
:10CFB000350003C72500A207D98F2311F500828011
:10CFC0002322050003C7450089476304F700054590
:10CFD000828083D665000D47E37BD7FE9C45011117
:10CFE00006CE22CC26CA4AC84EC683C4170003C642
:10CFF0000700A204D18C138644006311D60403C435
:10D00000370083C72700AE8922045D8C9307C4FFD5
:10D01000C207C1832A89636FF70003A58900231122
:10D02000990023108900F155EF403FBB2322A9004E
:10D03000014531A02285EFF06FD265F10545F24040
:10D040006244D2444249B24905618280397122DC8E
:10D050002E84834704004AD806DE26DA4ED61947C6
:10D060002A89B285639AE706034624002800EFF078
:10D07000FFD0AA8415E903558100EFF02FCEAA89CD
:10D080008345140015C937E701002E861307A7F55D
:10D0900034009D454A85EF00D0424E8509468145C2
:10D0A00035234E85EFF04FD9F25062542685425910
:10D0B000D254B2592161828089472310F1008357ED
:10D0C00081000A862311F1008357A1002312F10089
:10D0D0004A85EF009075C9BF4947639DE702035633
:10D0E00024002800EFF05FCFAA845DFD37250020E3
:10D0F000130585CF8357C50099E3814475B703476E
:10D100001400834604000345E5003C000146CA853F
:10D11000912659BF51476390E70203562400280027
:10D12000EFF0BF87AA8449F18345140030004A8597
:10D13000EFF05FD195BF59476393E706035624008C
:10D140002800EFF07F8BAA8425F1835581004A8562
:10D15000EFF06FCA1DC958458356A10083570700D9
:10D16000B697C207C1832310F700C1DB5C47D1D754
:10D17000B727002083C7A7A8C9D3B727002003C5B6
:10D1800047A98545EF40BFFB05B789473EC0835798
:10D1900081000A86834514002312F10015BF8345E0
:10D1A00014000A8623100100EF003068B9B75D71E2
:10D1B000A6C256DA86C6A2C4CAC04EDE52DCAA8A0D
:10D1C00003C51500AE8432C6EFF06FBCB24501ED69
:10D1D0008144B6402644268506499644F259625A4F
:10D1E000D25A61618280230205002311050083C9A0
:10D1F000040085472A84639AF90003C6240028089E
:10D20000EFF0FFB1AA8405492DA09D476394F9046E
:10D21000034705008D47E31DF7FA03C624002808DD
:10D220000549EFF09FB8AA8409E5054681452285A6
:10D23000712E2285EFF08FDE034584003C08014704
:10D24000CE862686D6853924E30509F82285EFF0B7
:10D25000AFBE41B7CD47639DF90003470500914735
:10D26000E318F7F603C624002808EFF0DFBB59BF28
:10D27000D547E39FF9F4034A05008947E31AFAF416
:10D2800003C6240028080549EFF09FCBAA8455F176
:10D2900083570102BDE3035781011306F0035C4489
:10D2A000930607FCC206C182636CD6000356A10137
:10D2B000D94663F7C6008356C101D94563EFD5004F
:10D2C000035524002391E7000549EF00305703562A
:10D2D0000102D2852285692CA9BF8355E1012391E2
:10D2E000E7002392C7002390B7002393D700854718
:10D2F0002300F400014A0149D9BF014AC9BF79712D
:10D30000AA8522D426D203542500AA84280806D64A
:10D31000EFF01FCBF24599E535E985452285EFF021
:10D320000FE5C1A0835781011547639BE7060357AB
:10D33000A1018D4763FCE7046800EFF05FC6035767
:10D34000E100DD4763FCE7008345D100B707170024
:10D350008507100822853EC8EF00304D8357E10055
:10D360000357A10191076305F7002285EFF02FDF36
:10D370008347C10072466C00858B1106228591CFD0
:10D38000EFF0FFE201C52285EFF06FDD884451D553
:10D390009730FE1FE78040D949B7EFF03FCBDDB7AC
:10D3A00011476389E7001387A7FF4207418385463A
:10D3B00063EEE6023147F117B387E7023727002013
:10D3C000130787CFBA9703D7070069D303C5270090
:10D3D0003008A2850D205DF9035781019147E31EB6
:10D3E000F7F2B25022549254456182802C08228573
:10D3F000812E49FDFDB701114AC82A89314526CA47
:10D4000006CE22CC2EC6B284EF409F8931C1B245F0
:10D410009307000A2310F5002311B5002A84214642
:10D4200011058DC0A6859730FE1FE78060DFA285BD
:10D430004A85EF40FF950145F2406244D24442499B
:10D440000561828081459730FE1FE78080E4C5B783
:10D450000545DDB7797126D2AA841305000206D6E8
:10D4600022D42ECE32CC36CA3AC83EC6EF405F83B5
:10D4700031C96246F2454247D246B2472A84130573
:10D4800020FA2300A400A300C4002311B400230247
:10D49000E400A302D40013058400614691CFBE8549
:10D4A0009730FE1FE780C0D7A2852254B250268550
:10D4B000925445616F40DF8D81459730FE1FE780B4
:10D4C00040DDDDB7B2502254925445618280584508
:10D4D000797122D406D62A84AE8649C383572700A1
:10D4E000231DF10093072006639FF504B727002052
:10D4F00003D667A8835767006373F600B28713F6F5
:10D50000F70F83552701834707018D8F93F7F70F97
:10D5100081E5890793F7F70FB297FD17B3C7C702E5
:10D52000231EF100835724008355640003458400C3
:10D53000231CF10001473C080146EFF0BFF1B25057
:10D540002254456182800347C701B727002083A783
:10D5500007A91207BA9783D76700D9B72EC619460D
:10D56000814528089730FE1FE780A0D2B2465DBFF4
:10D57000797122D406D626D22A848DC181470147EB
:10D58000930600062E868355640003458400EFF061
:10D590007FECB2502254925445618280B2842800BC
:10D5A00059469730FE1FE780C0CE2314910089E8CA
:10D5B0008357240048446C002315F100EFF08F9747
:10D5C0003C00014793060006014675BF797106D6F7
:10D5D000814799ED8357250058452316C100231430
:10D5E000F1003C0011C7835727002315F1003C00D0
:10D5F0002E86835565000345850001479306000686
:10D60000EFF05FE5B25045618280411122C406C649
:10D610008347050011472A846395E7022E868355C8
:10D6200065000345850081470147CD46EFF09FE245
:10D630004946835564002244B240154541016FF0CC
:10D64000CF8913F7B70F89466317D7000146EFF06C
:10D650003FF25146F9BF0D476398E7002244B240BC
:10D66000014641016FF09FF6B240224441018280A1
:10D6700003D70500B146B727002071173307D7023B
:10D68000938787CFBA97D84319EBD8412395A70042
:10D690000145D8C303D725002394E700828059456C
:10D6A0008280797122D4404526D24AD006D6AA84F7
:10D6B0002E8925C0484419C59730FE1FE780C0A6B3
:10D6C000232604008357040083D5640003C5840027
:10D6D0002315F100835724000147930640062316C3
:10D6E000F100835784004A862317F1001C483EC886
:10D6F00083D724002314F1003C00EFF0BFD5A30E24
:10D70000240123280400B250225492540259456146
:10D7100082802800314681459730FE1FE78060B740
:10D7200083D7240083D5640003C584002314F1004B
:10D7300001473C00930640064A86EFF0BFD1E1B7AF
:10D74000797152CC2A8A03D5050026D206D622D476
:10D750004AD04ECE56CAAE84EFE05FE019E185476D
:10D76000BDA84045AA8965DC83576500E39947FF5A
:10D7700083578400638707128346C401B72A0020B9
:10D7800003A70AA99206FD173697C2070357670039
:10D79000C1832314F4006316F70093053006EFF0FD
:10D7A0001FD35C48A5EFC840034915008347050017
:10D7B00022093369F90083D7240013072900631A6B
:10D7C000F702F955EF406FC1C8C02391240103C58A
:10D7D00089002686D285EFF01FC2814721E1B25031
:10D7E000225492540259F249624AD24A3E85456116
:10D7F00082809565938515C04A859730FE1FE78026
:10D80000608448C8C840231C2401F955EF40EFBC90
:10D8100083D72400C8C0F9172391F400484859C59C
:10D8200003D624008356A401835784013308D6000D
:10D8300063C007090347C40183A70AA995451207D6
:10D84000BA9783D7270063CF0705CC40369597302A
:10D85000FE1FE780E09C0357A40183D72400BA97FA
:10D86000C20703578401C183231DF400E399E7EE47
:10D8700003D7290003C5890030002314E10058486C
:10D88000D2852315F1003AC6EFF0FFB611C548481E
:10D890009730FE1FE7804089232A0400232C0400D0
:10D8A0007DBD99454E85EFE01FDE55BDA545DDBF29
:10D8B0009145CDBF03D725007DC3B727002083D670
:10D8C00067A8ED4763EEE60C011122CC2E8426CA30
:10D8D000AA844840914506CEEF402FB083572400DC
:10D8E000AA862300F50083572400A183A300F50036
:10D8F000835704002301F50083570400A183A3018B
:10D90000F50003562400C167F9171106420641824B
:10D910006396F4042AC4314532C6EF406FB8AA8535
:10D92000CD471DC5930700F92300F5003246F9578E
:10D93000A2462311F50089472302F500B7270020EE
:10D940002313C50014C503C547A9EF406FC4814721
:10D95000F2406244D2443E8505618280814526853D
:10D96000EF40B07DAA8711E9B726002003C7A6A81B
:10D9700065D37D172385E6A8E1BF09476304E50267
:10D980001D476303E50249476302E5027D47E31152
:10D99000E5FCB726002003C7A6A88147D1BFED4705
:10D9A0003E858280D1476DB791475DB789474DB7B6
:10D9B00001114AC831471309C5FF3307E902B727E8
:10D9C000002026CA938487CF06CE22CCBA94D840B2
:10D9D00029CB138487CFB727002083C6A7A8854704
:10D9E00095CA2314A10083D7840003D5A4002C007A
:10D9F0003AC62315F100EFF0FFEB11C5C8409720A0
:10DA0000FE1FE7806072B147B307F902A29723A215
:10DA100007008547F2406244D24442493E85056191
:10DA200082808147C5BF797126D2444537270020BF
:10DA30004AD083D76400035967A852CC06D622D4B3
:10DA40004ECE56CA2A8A63F327013E8903D72401A2
:10DA500042091359090183D7040141CB998F4A84A4
:10DA600063D5270113940701418089452285EFF092
:10DA70002F81AA89CD4A25C183D724002AC6231520
:10DA800081002314F10083D7240185E383D70401A7
:10DA9000930925002300F50083D70401A183A30087
:10DAA000F5006376240503D4040183D72401CC4414
:10DAB00022864E85BE959720FE1FE780607603552F
:10DAC0006A002C00EFF01FDFAA8A15C54E8597204B
:10DAD000FE1FE7806065B250225456859254025969
:10DAE000F249624AD24A4561828089078DBF791422
:10DAF000420441805DBF03D7240183D704003A94D8
:10DB0000FD17C207420403D70401C183418023905B
:10DB1000F400239984006377E400D5FFFD57A38EBA
:10DB2000F40055BF81455285EFF0BFB76DB77971ED
:10DB30004AD03729002052CC034AA9A922D456CA78
:10DB40005AC85EC662C406D626D24ECE5284B72AC2
:10DB50000020054B930BF00F372C002083A70AA859
:10DB600093144400BE9483C90400639D6907DC4498
:10DB7000B5CBD84725CB03D7070029CBB727002043
:10DB800083C7A7A899CF2685EFF0FFE9AA8515E9F5
:10DB9000B727002083C797A805046351F402230D1B
:10DBA00089A8B25022544E8592540259F249624AD1
:10DBB000D24A424BB24B224C45618280230D09A8C8
:10DBC000CDB72685EFF0FFAD8149E1BF83C7D7010F
:10DBD000639A7701930520062685EFF05F8FDC447A
:10DBE000A38E070083479CA805041374F40F636396
:10DBF000F4000144E31444F7C1BF4111154506C6C2
:10DC0000EFF01FDB09C50545B2404101828019458F
:10DC1000EFF01FDA6DF91145EFF09FD96DF51D4555
:10DC2000EFF01FD96DF1B727002083C797A8E9DF70
:10DC3000B24041016FF0BFEF83D705000D47F117E8
:10DC4000C207C1836365F706DC41B5C3411122C435
:10DC50002E84854526C206C6AA84912F39C92685F9
:10DC6000AD25C167F9176381F40219ED83572400CC
:10DC700081CF8356040019476393E60437270020B9
:10DC8000035767A863FDE702B727002083C7A7A84B
:10DC9000A285268599C72244B240924441016FF083
:10DCA0007FC12244B240924441016FF07F9C0945FC
:10DCB00082805145B24022449244410182806D45A8
:10DCC000D5BF397126DA4ED6AA84AE895D4589451D
:10DCD0004AD806DE22DC328936C63AC4EFE05FDA83
:10DCE00035C522472A84014511C7B24613054400B1
:10DCF000B68502979357850023003401A3002401C1
:10DD0000A301F4009547231CF100B727002083C727
:10DD1000A7A82301A4001105231DA10022CE2C08D1
:10DD2000268595C3EFF01FB9AA8411C522859720D7
:10DD3000FE1FE780603FF250625426854259D2545C
:10DD4000B25921618280EFF0BF92F9BFCD44E5B7AF
:10DD5000797126D24AD052CC56CA06D6BA8A22D473
:10DD60004ECE19472E89B284368A639DE506035547
:10DD700026000944EFE08FFE2AC62DCD5C4583596D
:10DD8000650083D727002390F400B247B726002010
:10DD900015472380570103C656A82391E7001307B0
:10DDA00016001377F70FA382E6A82382C70001E7C6
:10DDB0000547A382E6A85147631AE9001547239156
:10DDC000E400DC4703D784002394E7005287A6864B
:10DDD000CA854E85EFF0FFEE2A84324515C4EFE088
:10DDE000BF8509A842867400BE85AA89EFE08FE846
:10DDF0002A8441DD2285B250225492540259F249BC
:10DE0000624AD24A45618280F945EFE09F9FDDB7C3
:10DE100083D705002300F50083D70500A183A30065
:10DE2000F50083D725002301F50083D72500A183C2
:10DE3000A301F5001145828083D705002300F5007A
:10DE400083D70500A183A300F50083D72500230114
:10DE5000F50083D72500A183A301F50083D74500F2
:10DE60002302F50083D74500A183A302F50083D7E1
:10DE700065002303F50083D76500A183A303F500A4
:10DE80002145828083D705002300F50083D7050054
:10DE9000A183A300F5000945828083D705002300F4
:10DEA000F50083D70500A183A300F50083D72500E3
:10DEB0002301F50083D72500A183A301F50083D7B3
:10DEC00045002302F50083D74500A183A302F50096
:10DED00083D765002303F50083D76500A183A303DF
:10DEE000F50083D785002304F50083D78500A1833F
:10DEF000A304F5002945828003D705008546AA873B
:10DF00002300E50003D705002183A300E50003D724
:10DF10000500631DD70003D725002301E50003D7C3
:10DF200025002183A301E500114582800945631581
:10DF3000A70203D7250019452381E70003D7250051
:10DF40002183A381E70003D745002382E70003D79D
:10DF500045002183A382E700828083D70500230048
:10DF6000F50083D70500A183A300F50083D7250022
:10DF70002301F50083D72500A183A301F5001145F6
:10DF80008280797126D24AD04ECEB2842A89AE8957
:10DF900029468145480022D406D636849720FE1FA4
:10DFA000E780202F231691008DEC83572400231245
:10DFB000F100B727002083D767A82314F1005C4441
:10DFC0008DC383C6C70137270020032707A9920600
:10DFD00083D787003697035727002315F1002313B3
:10DFE000E10037E701004A851307A7E9540013F65B
:10DFF000F90FD545EFF0FFCC2A8911C19DE0854787
:10E000002300F40023020400014681452285EFF03D
:10E010002FD6B25022544A8592540259F249456192
:10E0200082802285EFE04FE1EDB737E70100B2864D
:10E03000130787EF2E8685456FF0BFC801112317A0
:10E04000A100B7E601004165700001489307F00F99
:10E050000D47938606E199457D1506CEEFF05FCF1B
:10E06000F24005618280B7E60100B28701482E8642
:10E070001147938686E3C9456FF09FCD37E70100CE
:10E08000B286130747E82E86CD456FF09FC3011176
:10E0900022CC37240020130484D226CA4AC84EC694
:10E0A00006CE2A89AE89930404031C4081C7CE851D
:10E0B0004A8582971104E31A94FEF2406244D244E6
:10E0C0004249B2490561828041113727002022C4AC
:10E0D00006C626C21307C7B78347C7030345D7033E
:10E0E00037240020130404D7A304F400AA9793F75D
:10E0F000F70F2304F400A5CF1305C0033385A7024F
:10E10000A5658505B7240020938404AA9720FE1FE7
:10E11000E78040F3034684009307C003814533063C
:10E12000F60288C09720FE1FE780A0169C40834619
:10E130008400014789077D566341D7022244B240DB
:10E14000924437250020130600038145130585D22C
:10E1500041011723FE1F6700C3132390C7002381CB
:10E16000070023A5070205079387C703F1B7B2404D
:10E170002244924441018280B727002003C687D7FA
:10E18000B727002003A707AA81476315F600814639
:10E1900036858280BA861307C703835567FCE389F7
:10E1A000A5FE850793F7F70FCDB7011122CC2EC638
:10E1B00032C406CE2A84EFF03FFC2246B24511E974
:10E1C000C167F9176303F4005145F24062440561E9
:10E1D000828054558347450095C213F72701414576
:10E1E0006314A700154575F2C18B3D45F9DF83C760
:10E1F000A6010145E3FBB7FC3145C1BFC18B014519
:10E20000E9F71545D9B7797126D24AD0B72400204D
:10E21000416922D44ECE52CC56CA5AC806D6AA89D3
:10E220000144938404D7372A0020930AC0037D1940
:10E23000054B83C784006364F400014535A8B30728
:10E24000540303270AAABA9703D7270063162701A6
:10E2500005041374F40FF1BF03C557003000938514
:10E260006700EFB0F16F1946CE8528009720FE1F9A
:10E27000E7804008E31E65FDB250225492540259D3
:10E28000F249624AD24A424B45618280B727002058
:10E2900083C587D7C166B727002003A707AAFD1645
:10E2A00081476395F5000146328582800358270037
:10E2B0003A866306D80003480700E307A8FE8507EF
:10E2C00093F7F70F1307C703E9BF411106C6EFF035
:10E2D000BFEA11C503554501B240410182800145A5
:10E2E000E5BFB727002083C687D7B727002003A73D
:10E2F00007AA0145814711076393F6008280034610
:10E30000070001C605051375F50F850793F7F70F8D
:10E310001307C703D5B7B727002003C587D7828067
:10E3200037270020930687D28147130787D23146CB
:10E330008C4291E58A07BA9788C301458280850798
:10E340009106E397C7FE4D458280411106C622C45F
:10E35000EFF09FE21DCD2A84035525008545EFF09F
:10E360001FD3485409C59720FE1FE780E0DB2285B4
:10E370001306C00381459720FE1FE78080F1FD57FB
:10E380002311F400230204000145B240224441015C
:10E3900082800945DDBF411106C6EFF0FFDD11C5E2
:10E3A0000345C500B240410182800145E5BFC16718
:10E3B000F9176304F502411122C406C62E84EFF05A
:10E3C000BFDBAA87014591C703C54700698C333578
:10E3D0008000B240224441018280054582800111C3
:10E3E00006CE2EC6EFF05FD9854711C90357450108
:10E3F000B24585476305B700231AB5008147F2404F
:10E400003E850561828031CD01114AC84EC637294B
:10E410000020C16922CC26CA52C456C206CE01448D
:10E42000AA84130909D7372A0020930AC003FD19CB
:10E4300083478900634BF400F2406244D24442496E
:10E44000B249224A924A05618280330554038327E8
:10E450000AAA3E95835725006383370182940504F9
:10E46000C1BF8280B727002003C687D7B727002007
:10E4700083A707AAC166014589070147FD16914593
:10E480006313E600828003D807006309D80003C83D
:10E49000A7006315B80005051375F50F0507137779
:10E4A000F70F9387C703E9BFB727002003C687D7B5
:10E4B000B727002083A607AA01478147910663106A
:10E4C000E602858393C7F7FFC207C18305456364EE
:10E4D000E50285473395A70042054181828083C5C7
:10E4E000060081C583D5C602CD8F05071377F70FC8
:10E4F0009386C603E9B793F61700E1FE0505858309
:10E500001375F50FE9B7797156CAAA8A2E8526D2F6
:10E510004AD04ECE52CC5AC85EC662C406D622D469
:10E52000AE84328B368CBA8B3E8AC2894689EFF034
:10E53000BFC449E141657D15EFF01FC42A845545EC
:10E5400031CC1946DE8513056400A30284019720AF
:10E55000FE1FE780E0CC83570103231194002302C0
:10E5600064012319F4008357410323005401232637
:10E570000402231AF400230644012317340123184C
:10E580002401EFF07FF22318A402232A0402268537
:10E59000232C04028145EFF09FAF0145B250225475
:10E5A00092540259F249624AD24A424BB24B224C2F
:10E5B000456182804545DDB7B727002083C687D7F0
:10E5C000B727002003A707AA81476395F600416596
:10E5D0007D1582803A861307C703835547FF6395ED
:10E5E000A500035526008280850793F7F70FF1BF3A
:10E5F000B727002003C887D7B727002083A607AA1C
:10E60000416601477D16954811436314E8000145B2
:10E61000828083D7260036856380C704CC5A8DCD8F
:10E6200083C7350083C5250089CD938597FD93F574
:10E63000F50FE37FB3FC9387D7FA93F7D70F89EFF2
:10E6400082809385F7FD93F5F50FE3F3B8FC93878C
:10E65000D7FA93F7D70FCDDF05071377F70F938618
:10E66000C60365B7B727002083C587D74166B7279C
:10E67000002003A707AA7D16814725486394F5006B
:10E6800001458280835627003A85638CC600545B1F
:10E6900089CA83C636009386E6FD93F6F60FE372C9
:10E6A000D8FE850793F7F70F1307C703C1BF011102
:10E6B00022CC2A84494506CEEF602FFC15C12AC61C
:10E6C0002285EFF07FAB09CD6244B72700203246A8
:10E6D00083550503F24003C537D705616F301FC569
:10E6E000F24062440561828039714ED652D4AE89BF
:10E6F0002A8A93053005414526DA4AD856D206DEE5
:10E7000022DC32C63689BA8A9720FE1FE7808093C2
:10E71000CD4431C92A848944638209043246814543
:10E72000231AC10041469720FE1FE78080B6568617
:10E73000CE8522859720FE1FE78080AE2146630E9E
:10E740000902CA8528089720FE1FE78060ADA286CF
:10E7500050082C085285EF40E00FAA8422859720AC
:10E76000FE1FE780609CF250625426854259D254C5
:10E77000B259225A925A21618280814528089720F5
:10E78000FE1FE78000B1E1B7411122C4405926C203
:10E7900006C6AA8429CC085409C59720FE1FE78025
:10E7A000A098285809C59720FE1FE780E097685871
:10E7B00009C59720FE1FE7802097285C09C5972090
:10E7C000FE1FE7806096685C09C59720FE1FE78002
:10E7D000A0950325040809C59720FE1FE780C09473
:10E7E00022859720FE1FE780209423AA040222445A
:10E7F000B727002083D50403B240924403C537D71E
:10E8000041016F30FFDB411126C206C622C4AE842F
:10E81000EFF09F9621C54C592A84A9C183A8C5074A
:10E8200003A88507FC59B85983C6650003D60500BF
:10E8300083C525002685EF608FEC2285EFF0DFF49D
:10E84000EFF05FE201CD2244B7270020B2409244AE
:10E8500003C537D7854541016F307F8EB2402244D2
:10E86000924441018280011122CC06CE2A842EC618
:10E87000EFF09F905C5991CF83D70700B245639A20
:10E88000870085476397F5006244F24005616FF0A9
:10E89000BFEFF240624405618280411106C622C486
:10E8A00026C2EFF0FFD421C54059AA8429C083476E
:10E8B00024008DCBB727002083A787AA89C7DC4314
:10E8C00099C322858297034734009307F0026310AF
:10E8D000F702224403D52400B2409244814541010D
:10E8E0006FF07FF2B727002083A7C7AAC1BFB2404D
:10E8F0002244924441018280411126C24AC006C688
:10E9000022C4AA842E89EFF03F8731C140595DCCE3
:10E9100083570400639C970A83473400130710024F
:10E92000639CE70883472400D9C37C540327040869
:10E9300083D7470105E713F717000DC31854035792
:10E940004700058B01CF93072002A301F400B240DA
:10E9500022449244024905454101828013F7270071
:10E9600009CB185403574700098B01C7930740028E
:10E97000E9BF918B89CB1C5483D74700918B81C70A
:10E9800093076002D9B7B727002083A787AAE1D3EE
:10E99000DC43D5DF22858297034734009307F002DA
:10E9A0008145E316F7FA2685EFF0FFE54DB7B72767
:10E9B000002083A7C7AAE1BF1307A0026398E7005E
:10E9C0006304090013092003CA85F1BF631C090011
:10E9D0002685EFF06FFA19C58347450093E70701D5
:10E9E0002302F500A6854A85EF509FE68DB7797121
:10E9F00026D29947231DB100AA842E858D4522D4A5
:10EA000006D632C636C4231CF100EFE06F872ACE4B
:10EA10004D441DC13246A246AA85328582962A847B
:10EA200019E52C082685EFF02FA12A8411C572451F
:10EA30009710FE1FE780406F2685EFF05FC72285A5
:10EA4000B25022549254456182804111B7060200AF
:10EA500022C42E862E8493868645894506C626C204
:10EA60004AC02A89EFF0BFF883450400AA844A858A
:10EA7000EFF07FD9B24022442685024992444101F9
:10EA80008280B727002083A7C7AA95CB9C4385CB5C
:10EA90001D71A2CC86CE984110082A843AC8D8416C
:10EAA00085453ACA829701C92306A100035524006F
:10EAB0006C00EFF09FF9F640664425618280828009
:10EAC000AE8715C5785505C7834607002380D50056
:10EAD00083461700A380D500834627012381D500F4
:10EAE00083468701584BA381D500D8C18280414617
:10EAF00081453E851713FE1F6700A379B7270020C5
:10EB000083A787AA91C703A3870063030300028337
:10EB100009458280372700200327C7B31DC7584304
:10EB2000AA8705450DC703A50708411106C6930628
:10EB300005021306050C9305050613050504029747
:10EB4000B2401375F50F41018280054582808280B5
:10EB50004DC9357122CD2A840355050026CB4AC9FB
:10EB60004EC756C306CF52C55AC1DEDEB68AB28939
:10EB70002E89EFF06FE0AA8439C50C182285EFF0DA
:10EB80003FF483472400138A6400A9CBEF50DFA52C
:10EB90002A8B014583CB5400EF50DFA2AA840C10CE
:10EBA0000818EF10206D08542C10EF10406DD2881B
:10EBB000268A56C05E88D2875A8714103010CE85B8
:10EBC0004A85EF207028FA406A44DA444A49BA4933
:10EBD0002A4A9A4A0A4BF65B0D618280EF50DFA009
:10EBE000AA8B014503CB5400EF50DF9D2ACE085479
:10EBF0000C10EF1020682C100818EF104068F24835
:10EC00004DBF8280C14709CD1455C14791CA78557F
:10EC100001CB83C73600BD4663F4F6008347870106
:10EC20003E8582808947630905106387051041117D
:10EC300006C622C426C2834715002E842380F50011
:10EC400083472500A380F500834735002381F50025
:10EC500083474500A381F50083475500858B939634
:10EC6000870083D7450093F7F7EFD58F2392F50000
:10EC70008346550093F7F7DFA20693F60620DD8E54
:10EC80002392D5000347550093F6F6BF220713776A
:10EC90000740558F2392E50083475500FD76938604
:10ECA000F67F8D87858B758FAE07D98F2392F50000
:10ECB00083466500F99B858ADD8E2392D500034744
:10ECC00065009377270013F7D6FF5D8F2392E50049
:10ECD0008347650093F647009377B7FFD58F23925C
:10ECE000F50003476500DD9B4D45218BD98F2392AD
:10ECF000F500EF608F98AA845145EF600F980347A5
:10ED0000340093F4F40FC947636297021375F50F4B
:10ED1000636EE500834604001147E1476368D7004E
:10ED20008346140005476363D7008147B2402244FD
:10ED300092443E85410182803E85828015C1AA872A
:10ED400009458DC141112E8541469385170006C6A0
:10ED50009710FE1FE780C04CB24001454101828000
:10ED600009458280828089471DC595C5411106C627
:10ED700003471500AE8719462380E500930525005B
:10ED8000138517009710FE1FE7808049B240814726
:10ED90003E85410182803E85828015C1AA87094552
:10EDA0008DC141112E8541469385170006C69710E7
:10EDB000FE1FE780E046B2400145410182800945DF
:10EDC0008280828089471DC995C9411106C60347C3
:10EDD000250083461500AE872207558F2390E50056
:10EDE000214693053500138527009710FE1FE78005
:10EDF0002043B24081473E85410182803E8582802A
:10EE000015C1AA8709458DC141112E8541469385BB
:10EE1000170006C69710FE1FE7808040B2400145EC
:10EE200041018280094582808280894719C991C940
:10EE300003471500BD46E14763E5E6002380E50092
:10EE400081473E85828015C1AA8709458DC1411140
:10EE50002E8541469385170006C69710FE1FE78052
:10EE6000203CB24001454101828009458280828078
:10EE700015C1AA8709458DC141112E85414693854B
:10EE8000170006C69710FE1FE7808039B240014583
:10EE9000410182800945828082801DC1AA8709457F
:10EEA00095C141112E85130600049385170006C6EF
:10EEB0009710FE1FE780C036B240014541018280B5
:10EEC00009458280828015C1AA8709458DC14111FB
:10EED0002E8541469385170006C69710FE1FE780D2
:10EEE0002034B24001454101828009458280828000
:10EEF0001D71A2CC2A84084586CEA6CA230601002D
:10EF00008344050035479387F4FF93F7F70F636A4F
:10EF1000F70C37D703008A0713078795BA979C43E6
:10EF200082870C08EFF01FD0C9476312F50299479A
:10EF30002306F100035524006C00EFF01FB1F640EA
:10EF40006644D644256182800C08EFF07FEB29C926
:10EF50008347C100E5F303552400EFF04FF5C5B733
:10EF60000C08EFF05FEEE5B70C08EFF01FECC5B74B
:10EF70000C08EFF0BFDCE1BF0C08EFF0BFE4C1BF4D
:10EF80000C08EFF09FE1E1B70C08EFF0DFDDC1B74F
:10EF90000C08EFF0FFED65BF834715002308F10073
:10EFA00003552400EFF04F9DA1470DC10347C50055
:10EFB000631BF702B727002003A787AA9D4719C73D
:10EFC000184309C71008A6850297AA872306F100EF
:10EFD00041B70C08EFF07FEC9DBF0C08EFF0BFEEDF
:10EFE000BDB79D47B1B7B727002003A7C7AAF9B798
:10EFF000011122CC06CE26CA4AC84EC603470500D8
:10F00000930720092A84631BF712834715003947A9
:10F010006394E70A83564500096761078147639750
:10F02000E610B7240020938944AA03A5090093841D
:10F0300044AA630D050E0C4403C90500631E0900B4
:10F040008347050085052146A9CB29059710FE1F9A
:10F05000E780001D9C40B9CF4945EF207FC42A843A
:10F060000DC5930710FC2300F500A30025018C407B
:10F070000905414689059710FE1FE780601A9C40EC
:10F08000A28503C51700EF20BFD088409710FE1F50
:10F09000E780800923A0040031A809059710FE1F0E
:10F0A000E7800018EF30C07A05494DF583A70900C5
:10F0B0002380270185479DA81307E003639EE70887
:10F0C000034725009547631FF70203554500EFF0FE
:10F0D0008FAC9147E310F5FEB727002083A7C7AA9E
:10F0E000F1DB03A38700E30703FC0356E4000355A9
:10F0F0004400930564006244F240D2444249B2495C
:10F1000005610283A147631EF70083456400035530
:10F1100044006244F240D2444249B24905616FF072
:10F12000AFFD930600038147E301D7FEF24062443E
:10F13000D2444249B2493E85056182809306000A65
:10F140008147E315D7FEEFF0BFDA084425D59710C5
:10F15000FE1FE78060FDB9BF8147C9BF011126CA04
:10F1600006CE22CC89441DCD95CDAA842E8468007C
:10F170008D45EF50CF968347E1002685228693F791
:10F18000F70393E707046C002307F100EF20C04268
:10F19000AA8409E90D466C00130534009710FE1F80
:10F1A000E7800008F24062442685D24405618280EF
:10F1B0005D714EDE86C6A2C4A6C2CAC052DC56DA53
:10F1C0005AD85ED6894945CD5DCA138B4500420B9E
:10F1D000135B0B01AE8A2A8A930530055A85B284E7
:10F1E0009710FE1FE78000E62A84CD4949C9EF50F9
:10F1F0008FC12A895686D285935A8900135A0901EC
:10F20000937BF90F1305440093FAFA0F137AFA0F60
:10F21000135989019710FE1FE780A012A301740102
:10F2200023015401A300440123002401EF500FBD2A
:10F23000AA85414608089710FE1FE78080102147E5
:10F2400034005A86A2850808EF20A05DAA891DE136
:10F2500021462C0023807401A380540123814401A2
:10F26000A3812401138544009710FE1FE780600DE1
:10F27000EF502FBA22859710FE1FE780E0EAB640D4
:10F2800026444E8596440649F259625AD25A425B48
:10F29000B25B6161828001114AC82A892E8506CE3F
:10F2A00022CC26CA2EC6EFE03FED71C5405971C48D
:10F2B000834754000947B24593F6B70F6387E600CA
:10F2C00011471305E00F6392E708835704000945CF
:10F2D000639DB706930484004146CA85268597102E
:10F2E000FE1FE780E0F34146CA85130584019710AD
:10F2F000FE1FE780E0F20347340085469307F7FEE0
:10F3000093F7F70F63E9F6041306C4033285C1458A
:10F3100032C6EF40DFFC32469306C402A685228542
:10F32000EFF01F838347240089CB22856244F2409B
:10F33000D244424905616F10601B03473400C9473E
:10F34000E305F7FEA301F4000145F2406244D24414
:10F35000424905618280930710050145E317F7FED6
:10F3600083472400FDD322856244F240D2444249BF
:10F3700005616F10201E0945C9BF4945F9B73971AC
:10F3800052D42A8A328526DA4ED606DE22DC4AD8C4
:10F39000AE8932C6EFE05FDEC94459C54059C94461
:10F3A00041C48357040032466390C7088347540022
:10F3B000A18BB1CB372900208327C9B39304E00F79
:10F3C000A5C79C47B5C39304840126854146D285D1
:10F3D0009710FE1FE780C0E48327C9B38325040884
:10F3E00026869C4793850504180881462E858297BA
:10F3F000AA844146CE8508089710FE1FE78080EF5B
:10F4000093F4F40F11E18944034734009307B005E6
:10F41000631CF7002285EF10A0108347240091CFD2
:10F420009307C005A301F400F250625426854259A7
:10F43000D254B259225A216182809307E005DDB788
:10F4400029CD011126CA06CE22CCAA840945A9C11C
:10F450000D4628002E848D059710FE1FE78040DCA6
:10F460008347A10070002C0093F7F70393E707048C
:10F4700026852305F100EF20201419E90D46A28509
:10F4800068009710FE1FE780E0E67D153335A00089
:10F49000F2406244D24405618280094582800111B4
:10F4A00052C42A8A32854EC656C25AC006CE22CCD3
:10F4B00026CA4AC82E8BB28AB689EFE0FFCB09ED87
:10F4C0008944F240624426854249D244B249224AE4
:10F4D000924A024B056182805C592A89C544F5F342
:10F4E0004D45EF509F991374F50F5145EF50FF981C
:10F4F000E38809FC83C78901E3E487FC1375F50FF2
:10F50000E360F5FC93053005130540089710FE1FD6
:10F51000E78040B3232AA9022A84CD445DD1130693
:10F52000400881459710FE1FE780A0D6A301040084
:10F5300023014401230264012310540123263407CC
:10F5400023240402A30204008144E30C0AF622856A
:10F55000EF00D073AA8435D54A85EFF0EFA295B7B6
:10F56000397122DC06DE26DA4AD84ED652D456D27B
:10F570005AD05ECE62CC66CA0944630B061063099A
:10F580000710AA8B3A89368BB28A2E8CEFE0DFBE49
:10F590002A8A5144630E050E9305300541459710A4
:10F5A000FE1FE78020AAAA894D447DC1834419002B
:10F5B00083472900A204C207BE9483470900BE9472
:10F5C00083473900E207BE9483278A0263E69700E7
:10F5D0007D5709446399E70A63070C0083474A0093
:10F5E0000544898BCDC3930C4B00214681450A8588
:10F5F000C20C9710FE1FE780C0C993DC0C01930575
:10F60000300566859710FE1FE780C0A32A8C4D4405
:10F610003DC95A86D68511059710FE1FE78060D236
:10F620001146CA8562859710FE1FE78080D141464A
:10F6300093058A014E859710FE1FE78080D02147F1
:10F640008A866686E2854E85EF20A01D2A841DE508
:10F6500021468A8528009710FE1FE78080CE21462C
:10F660009305490028009710FE1FE780A0C8854732
:10F67000631EF502A6855E85EF509FB662859710E2
:10F68000FE1FE78060AA4E859710FE1FE780C0A985
:10F690002285F2506254D2544259B259225A925A97
:10F6A000025BF24B624CD24C216182800544F9B777
:10F6B00079719397050122D406D626D24AD04ECE30
:10F6C000C1872E8463D50704B7240020938404D710
:10F6D00003C53400EF20CFE32AC611CDEFF05F91D0
:10F6E000B24519E503C524009307F00F631EF5002A
:10F6F0002E85EF20CFD52165218DB2502254925412
:10F700000259F24945618280EF208FE8EDB793F707
:10F71000150091C7EFF06F9813451400F9BFA1E1F0
:10F720000145E1BF850493F4F40FEFE0DFBEE3F998
:10F73000A4FE339599001319050113590901B377F4
:10F740002401EDD34A85EFE03FE7C167FD1763056C
:10F75000F500DD45EFF02F8B3345240179BF85445B
:10F760008549E1B7B727002023A207AAB7270020C1
:10F7700023A407AAB727002023A607AA3707020059
:10F78000B7270020938787D5130707DA98C3370771
:10F7900002001307C7AAD8C337E701001307876E13
:10F7A00098C7B727002037170200938747D613075B
:10F7B000A7D398C3371702001307278AD8C3371770
:10F7C0000200130767B898C78280B727002083C755
:10F7D00047D7A18B89C7B7270020938787D53727BD
:10F7E00000202324F7AA01458280B727002083C781
:10F7F00047D7918B89C7B7270020938747D63727EC
:10F8000000202326F7AA01458280011106CE2AC6D0
:10F81000EFF05FF53245B72700209945A389A7D6B9
:10F82000EFD06FA0F24037F5010013056586056142
:10F830006FE01FAF1C5581C7A1473E858280011133
:10F8400022CC26CA2A84AE84130500049305300511
:10F8500006CE9700FE1FE780E07E08D46305051002
:10F8600013060004A6859710FE1FE780609B78545E
:10F870008347270193F68700638E0610145483C6CE
:10F880002600A18A6388061083270408E9EF930500
:10F890003005130500109700FE1FE780A07A232093
:10F8A000A4088D4771C1A3020400785483C71400D3
:10F8B0008346170081EF81EE83C72400918BDDEB37
:10F8C00083472701918BDDE7854711A889C621472A
:10F8D000A302E40099C78347540093E70701A302FA
:10F8E000F4006C5483C72501858B91CF1C540547C8
:10F8F00083C727008D8B6398E7008347640093E7F5
:10F9000017002303F4008327040899C78347640082
:10F9100093E787002303F400834754000547639867
:10F92000E70C930484004146814526859710FE1F0D
:10F93000E780209641468145130584019710FE1FFC
:10F94000E78020951306C4033285C14532C6EF40D7
:10F950001F99832704083246BDC72285EF00903FD8
:10F960009307000525CDA147F2406244D2443E856D
:10F970000561828083C70400834607001547B3876B
:10F98000E70237D703001307C79ABA97B69783C71A
:10F990000700B1B783C6140091C68346170099C209
:10F9A000E14735BF83C62400D58F918B91DF83C794
:10F9B0000400834607001547B387E70237D70300E3
:10F9C00013070799D9B722859306C402A685EFF0DD
:10F9D0002F982285EF00903159F5C1470355040057
:10F9E000A301F4008145EF500FEA8147B5BF13F73B
:10F9F000870149C3C18B930484004146A9CB890583
:10FA000026859710FE1FE780A0814146814513059A
:10FA100084019710FE1FE780C087834764001306A8
:10FA2000C403328593E747002303F400C14532C67F
:10FA3000EF40FF8A8327040832468DC32285EF00FA
:10FA400070319307200505F1A301F40079BF8145CA
:10FA500026859710FE1FE780C08345BF9306C4022A
:10FA6000A6852285EFF0CF8E2285EF003028CD4786
:10FA700061DDD5BD094785456388E70093F7D70F5A
:10FA800011476397E700894503550400EF50AFDF46
:10FA90008347640093E747002303F40083270408A7
:10FAA00081C7930710054DB7C54779BF8347250028
:10FAB00063830726797122D406D626D24AD083479B
:10FAC0003500130750052A84639FE7060349750034
:10FAD0001306C503C14593573900AA97328583C4DD
:10FAE000870032C6EF40AFFFB727002083A7C7B318
:10FAF000A9C79C47B9C30325040893767900B3D6F8
:10FB0000D4403246858A93050504180893E6060812
:10FB10001305050882971375F50F05E141460C089A
:10FB20001305C4029700FE1FE780806F2285EF0057
:10FB3000F01B93076005A301F400B25022549254C5
:10FB4000025945618280130710026395E7021C5534
:10FB50000327050883D7470069EB13F7071071C720
:10FB60007855035747011377071061C39307700255
:10FB7000A301F4008347340013077002639FE70C6E
:10FB80003C5885E39305300571459700FE1FE780DB
:10FB9000604B28D819C5714681459700FE1FE78044
:10FBA000406F2458B9C883C7A40191E72285EFF0BC
:10FBB0006F85238DA4002858814541469700FE1F7C
:10FBC000E780206D28583D478345A5019387F5FFC1
:10FBD00093F7F70F6364F700EF406FF0EF208FB5F6
:10FBE0003C58A1452398A70013852701EF402FEF2C
:10FBF0002C5803550400EF00D040930780020355B2
:10FC00000400A301F400EFE02FD7414611C583574C
:10FC1000E50013D617003E96B727002003C537D757
:10FC200006068545EF208FF009BF13F7072011CB9B
:10FC30007854035747011377072001C793079002B1
:10FC400005BF93F707409DD77C5483D7470193F7AF
:10FC500007408DD39307B00221BF13078002639B37
:10FC6000E7023C5889CB83D507010355040013866E
:10FC70002701EF00903E1C5483D7470013F707205D
:10FC80002DC37854035747011377072039CB9307C7
:10FC90009002B5B713079002639CE700EF407F9591
:10FCA000AA8503550400EF00503A9307A00281BFD4
:10FCB0001307A0026393E704EF401F93AA858547CB
:10FCC00001456384F500814505452EC6EF409F8FB1
:10FCD0002A86B24503550400EF00B0331C5483D785
:10FCE000470093F707408DC77C5483D7470193F7AC
:10FCF000074099CF9307B00219B71307B002639971
:10FD0000E700EF40BF8FAA8503550400EF0070386D
:10FD10009307F0020DB58280411122C4405926C2DA
:10FD200006C67C54AA8483D7470113F7071019C766
:10FD3000185403574700137707101DE313F70720E4
:10FD400019C71854035747001377072011EB93F78F
:10FD500007408DCF1C5483D7470093F707409DC7BA
:10FD600093071002A301F4002285EFF03FD403476C
:10FD700034009307F0026310F702224403D52400F5
:10FD8000B2409244814541016FE0FFA79307F00222
:10FD9000A301F400DDB7B2402244924441018280C5
:10FDA000397122DC405926DA4AD84ED606DEAA89B5
:10FDB000AE843289630F043C035525008357040049
:10FDC0006384A700A14429A08347240091EB9D44AC
:10FDD000F250625426854259D254B2592161828030
:10FDE0009387E5FF93F7F70F2D47E362F7FE37D7C9
:10FDF00003008A071307879CBA979C438287B285C2
:10FE00002285EFF03FA3AA84E1B74146CA851305D6
:10FE1000C4049700FE1FE780A04022851127AA8412
:10FE200011C1A14483473400130740056397E700DD
:10FE300093079005A301F40061BF13076005639564
:10FE4000E7009307A005FDB7D147EDB79309C405B7
:10FE50004E854146CA859700FE1FE780603C03251A
:10FE6000040855C983473400130790056399E700D8
:10FE7000228591279307E005A301F40059A81307F1
:10FE8000A0056394E7088347740013D737002297CF
:10FE9000834687009D8BB3D6F640B727002083A703
:10FEA000C7B3858A93E606F893F6F60F81DF9C4781
:10FEB00091DB9305050818084E8613050504829703
:10FEC0009374F50FE39004F041460C081305C40445
:10FED0009700FE1FE7800042834774004D47850767
:10FEE00093F7F70FA303F4006377F7002285E1256A
:10FEF0009307E00581B7B727002003C537D78545AD
:10FF0000EF20EFA39307500535B71307C005E38132
:10FF1000E7F6814475BD130984004E86CA852285A3
:10FF20001408EFE0FFC241469305C4040808970097
:10FF3000FE1FE780203CE30D05E88A861306C40314
:10FF4000CE854A85EF1090040DE12285EFE09FCB2E
:10FF5000B72700202A8783A707D6035504008146C8
:10FF600001468A858297AA8411C1A1449307200281
:10FF7000D1B583450600EFE01F8961BF0347340018
:10FF800093072002E315F7E47C5889EB93053005CD
:10FF900071459700FE1FE780E00A68D86858E308BB
:10FFA00005E24146CA859700FE1FE7806027645836
:10FFB0002285EFE03FC5238DA400930730026DBD7D
:10FFC0000347340093073002E313F7E0835706003A
:10FFD00068582146930529002318F5004905970024
:10FFE000FE1FE780E0237C5483D7470113F72700E7
:10FFF00035CB185403574700098B2DC79307400290
:020000022000DC
:10000000A5BD0347340093074002E312F7DC3C5CD4
:1000100081EB85455D459700FE1FE780A00228DC47
:10002000285CE30805EE834709004146CA85230B97
:10003000F5009700FE1FE780A01E930750022DBD1C
:100040000347340093075002E313F7D8285C19469E
:100050009305190041059700FE1FE780601C7C5442
:1000600083D74701918B9DCF1C5483D74700918B39
:1000700095CB9307600209B57C5C89EB930530054D
:1000800051459700FE1FE780E0FB68DC685CE30BEE
:1000900005D24146CA859700FE1FE78060187C5C48
:1000A0007D5798CB4E85EFF03FC7A5B503250408D3
:1000B00013060004CA85130505049700FE1FE78098
:1000C00020162285EFE01FA58347340013070005A3
:1000D0006395E7009307400545B313071005639C3C
:1000E000E700B727002003C537D78545EF202F85C8
:1000F0009307500551B313072005E39CE7E0B727AA
:10010000002083A7C7B3E38F07CA9C47E38C07CAC5
:100110008325040893048400180893850508814604
:1001200026862E858297035504001008A685EF4089
:100130007FFE9307B00589B3034734009307E005BA
:10014000E317F7C88325040841464A859700FE1F38
:10015000E780401AAD44E30D05C603250408414677
:10016000CA859700FE1FE780A00B2285EFE09FA9BC
:10017000B72700202A8783A707D62C5803550400E9
:10018000814601468297AA8411C1A14493071002B7
:1001900055B1AD47E39FF5D683460600835525004C
:1001A0001306650003450500EF402FFB9DB389470B
:1001B00061C2DDCD2300A60083C70500A300F600C1
:1001C00083C715002301F60083C72500A301F600AD
:1001D00083C73500A30206002302F60083D745003B
:1001E000A183858BA302F60003D745001377072070
:1001F00009C793E72700A302F60083D7450093F7CA
:10020000074099C78347560093E74700A302F600CB
:1002100083D745001397470163580700834756006B
:1002200093E78700A302F6002303060083C7450077
:10023000858B2303F60003D74500098B09C793E795
:1002400027002303F60083D74500918B99C7834786
:10025000660093E747002303F60003D74500814774
:10026000218B19C703476600136787002303E60045
:100270003E8582802E86AA8505456FF05FF32E8627
:10028000AA8509456FF0BFF289478DC505C54111A3
:1002900006C6AE870D47AA852380E70013851700A1
:1002A00041469700FE1FE780A0F7B24081473E8598
:1002B000410182803E85828089478DC505C54111F7
:1002C00006C6AE871147AA852380E700138517006D
:1002D00041469700FE1FE780A0F4B24081473E856B
:1002E000410182803E85828089478DC505C54111C7
:1002F00006C6AE871947AA852380E7001385170035
:1003000041469700FE1FE780A0F1B24081473E853D
:10031000410182803E85828089479DCD15CD411166
:1003200006C61D472380E50003570500AE8721461A
:10033000A380E5000357050021832381E500930591
:100340002500138537009700FE1FE78060EDB2405F
:1003500081473E85410182803E85828089478DC5E7
:1003600005C5411106C6AE872147AA852380E7004F
:100370001385170041469700FE1FE78060EAB240F0
:1003800081473E85410182803E858280894795C9AB
:100390000DC9411106C625472380E5000347050026
:1003A000AE871946A380E500930515001385270045
:1003B0009700FE1FE780C0E6B24081473E854101BD
:1003C00082803E85828089478DC505C5411106C65C
:1003D000AE872947AA852380E70013851700414689
:1003E0009700FE1FE780C0E3B24081473E85410190
:1003F00082803E858280894795C50DC5411106C61C
:10040000AE873147AA852380E700138517001306BE
:1004100000049700FE1FE780A0E0B24081473E85C0
:10042000410182803E85828089478DC505C5411185
:1004300006C6AE873547AA852380E70013851700D7
:1004400041469700FE1FE780A0DDB24081473E8510
:10045000410182803E858280894791C909C99547BB
:100460002380F50083470500A380F50081473E8582
:100470008280894791C909C9AD472380F500834728
:100480000500A380F50081473E85828015C55D711A
:100490008A8586C6A2C42A84EFE08FE20355040051
:1004A000B70602000A86938646279D45EFE02FD4C3
:1004B000B6402644616182800545828015C55D7124
:1004C0008A8586C6A2C42A84EFE08FDF0355040024
:1004D000B70602000A869386E6279D45EFE02FD1F6
:1004E000B640264461618280054582805D71A2C468
:1004F0009305C5022A8441460A8586C69700FE1FD9
:10050000E78000D203550400B70602000A869386EE
:100510008628C545EFE0AFCDB640264461618280B4
:100520005D71A2C49305C5032A8441460A8586C627
:100530009700FE1FE780C0CE03550400B7060200F7
:100540000A869386862BC545EFE06FCAB6402644DF
:1005500061618280B727002083A7C7B3B1CB9C43DA
:100560005D71A2C486C62A841305E00F95CF0325CA
:1005700004089305050C13050508829783250408D4
:10058000130600040A85938505089700FE1FE7807F
:1005900020C903550400B70602009386663F0A8609
:1005A00093051004EFE0AFC4B64026446161828039
:1005B0001305E00F8280317122DD2A840355050086
:1005C00026DB06DF4AD94ED752D556D35AD15ECF55
:1005D00062CDEFD07FBA3C58AA8489EB93053005F1
:1005E00071459700FE1FE780E0A528D82858CD4721
:1005F0000DC9714681459700FE1FE78080C9032918
:1006000004072285EFE00FE0230DA90083472400B3
:1006100037290020638A07128327C9B385E393072C
:10062000E00FFA506A54DA544A59BA592A5A9A5A77
:100630000A5BFA4B6A4C3E852961828083AB0701D5
:10064000E38F0BFC032B0408EF301FFA2A8C0145C3
:10065000EF305FF783C754003858130B0B02930930
:10066000C403130AC405938A64003AC0B337F00088
:100670002A87930801045688B33680015286CE85B6
:100680005A85829B1C5403C727002307E10203C736
:100690001700A306E10283C707002306F1028327A0
:1006A000C9B3B5DF03AB4701E30B0BF683C75400B7
:1006B000B337F0003ECEEF303FF3AA8B0145EF3069
:1006C0007FF003270408F2472AC03AC2B33870010A
:1006D00056887810930684004E86D2858800029B47
:1006E0007C5403C727012305E10203C71700A304B5
:1006F000E10283C707002304F1028327C9B303A9DA
:100700004701EF307FEE2A8B0145EF30BFEB83C806
:1007100054009C082A883EC2B3381001B3376001E8
:100720003810930684015286CE8556C088000299FF
:1007300003550400B7060200938686429008C5451B
:10074000EFE0EFAAAA87F1BD83C654008327C9B39F
:10075000032B0408B336D00083AB070136CEEF304D
:10076000BFE82A8C0145EF30FFE53C58F246130BF9
:100770000B02130AC4059309C403938A64002A88F0
:10078000930801044E86D2853EC05687B337800158
:100790005A85829B1C54130B010303C727002307B0
:1007A000E10203C71700A306E10283C7070023067F
:1007B000F1028327C9B383AB470183C75400B33722
:1007C000F0003ECEEF305FE22A8C0145EF309FDF34
:1007D000F2472AC0B3388001568878109306840007
:1007E0004E86D2855AC28800829B832504084146E2
:1007F0005A859700FE1FE780E0AFAD47E31205EE94
:100800000DB5B70602002E869386862EC5456FE08D
:100810000F9E5D71B287A2C42300B1002A84BE85F9
:1008200013051100194686C69700FE1FE780409FFA
:10083000B70602000A8622859386C638A145EFE0F6
:100840000F9BB640264461618280B70602002E8667
:100850009386C635C5456FE08F995D71B287A2C496
:100860002310B1002A84BE8513052100214686C6C7
:100870009700FE1FE780C09AB70602000A8622850D
:1008800093868631AD45EFE08F96B6402644616190
:100890008280B70602002E869386663CC5456FE0CF
:1008A0000F95797122D406D626D2834735001307D7
:1008B00030052A846384E708130750056396E70828
:1008C0009307A005A301F50083477500C14513D721
:1008D00037002A97834687009D8B1305C503B3D63F
:1008E000F640858A93E606F893F6F60F36C6EF30A3
:1008F0001F9FB246B727002083A7C7B39DCB9C4755
:100900008DCB0325040818081306C40393050504BA
:100910001305050882971375F50F01ED1305C40241
:1009200041460C089700FE1FE780808F2285EFF07C
:10093000FFBBB250225492544561828093079005C8
:10094000A301F50081467DB7130710026396E70205
:100950007C550327050883D747016316070E13F755
:1009600017006302070E185503574700058B61CF28
:1009700093072002A301F4008347340013072002E9
:10098000639DE70E3C5889EB93053005714597F060
:10099000FD1FE780206B28D82458C9C02285EFE0CE
:1009A0006FA6238DA4002858814541469700FE1F5D
:1009B000E780208E28583D478345A5019387F5FFA2
:1009C00093F7F70F636DF702B727002083C747B28D
:1009D000D5C34146814508089700FE1FE780608B1C
:1009E000B72500201946938505CB08089700FE1F00
:1009F000E780008330580C082E85EF10A10BEF1014
:100A00006FD33C58A1452398A70013852701EF30E9
:100A10001F8D2C5803550400EFF0BFDE9307300202
:100A200003550400A301F400EFD00FF5414619C1AE
:100A30000356E500B727002003C537D706068545CE
:100A4000EF10DF8EFDB513F7270009CB18540357BD
:100A50004700098B01C79307400229BF918BE38DA3
:100A600007F01C5483D74700918BE38707F0930767
:100A7000600209B7EF30BF8659B713073002639A97
:100A8000E7023C5889CB83D5070103550400138640
:100A90002701EFF09FDC7C5483D7470113F7270031
:100AA00021CF185403574700098B39C793074002D9
:100AB00085BF13074002639CE700EF309FB3AA8510
:100AC00003550400EFF07FD89307500291BF13073E
:100AD00050026390E704EF303FB10DE981450545D1
:100AE0002EC6EF303FAE2A86B24503550400EFF024
:100AF0005FD27C5483D74701918B9DC71C5483D709
:100B00004700918B95C39307600219BF8545014546
:100B1000C1BF130760026399E700EF303FAEAA85BB
:100B200003550400EFF0FFD67C540327040883D755
:100B3000470119EF13F7071001CF18540357470067
:100B40001377071011C793077002A301F400D5B300
:100B500013F7072011CB18540357470013770720CA
:100B600001C793079002D5B793F7074091CB1C5468
:100B700083D7470093F7074081C79307B002F1B7C7
:100B80009307F002D9B7397122DC26DA4ED652D457
:100B900006DE4AD8AE89328AAA84EFD0EFDD40590A
:100BA000414681450A8597F0FD1FE780806E25C884
:100BB0000359040063159906034734009307100294
:100BC000631FF7028327040899CF2C58A9C94A85C7
:100BD000EF1050490545F2506254D2544259B2596F
:100BE000225A216182808A861306C4059305C403B4
:100BF00013058400EF0090391DE18A85C9BF2C5888
:100C000099CD83D70501639C47012146C9054E85CF
:100C100097F0FD1FE780006E19C12C584DBF268547
:100C2000EFD08FD52A8405455DD44C54A1C983D714
:100C30000501639547052146C9054E8597F0FD1FBF
:100C4000E780406B8547631BF502B727002083C709
:100C5000379B91C74C5483C7B501639BA70CBD4517
:100C60002685EF10703AB727002083A7C7BA014541
:100C7000BDD31D45894582970145B1BFB7270020E7
:100C800003C777B1B72900209389C9B7058B3E897F
:100C900031C3B72700200347540083C707B1631B44
:100CA000F702B72500201946938515B11305640096
:100CB00097F0FD1FE78000648547631DF50083A75B
:100CC000090381C791451D458297BD452685EF10D3
:100CD000B03309B737270020034747B283A709037A
:100CE00031CB034779B1098B09CB81C795451D45A8
:100CF00082972685EF105037F1BD81C78D451D4580
:100D0000829741468145080897F0FD1FE7806058AB
:100D1000B72500201946938505CB080897F0FD1FDD
:100D2000E78000500C082E850A86EF00B1588A85AE
:100D3000268579BD8545C5FF6DBF797122D440599F
:100D40004AD04ECE52CC06D626D2AA892E8A3289D5
:100D5000630D046A0355250083570400638CA700C4
:100D6000A144B2502254268502599254F249624A53
:100D7000456182808344240099C09D44DDB79387F8
:100D8000F5FF93F7F70F3147E369F7FE37D7030015
:100D90008A071307879FBA979C4382871C54E9F3FD
:100DA000930530051305000497F0FD1FE7808029A7
:100DB00008D45DD503470900914763F4E7008D44EB
:100DC0004DB7034719008547E3EBE7FE1306000420
:100DD000CA8597F0FD1FE780A0440C547054A3020D
:100DE0000400D4415C4A858AFD8E83574601F99BF5
:100DF000D58F231AF600D841544AF59B0583058BFD
:100E00008582F98E8606DD8E231AD600DC41584A8B
:100E1000ED9A8983858B09837D8F0A07558F231A65
:100E2000E600D4415C4A5D9B8D82858A8D83F58F77
:100E30008E07D98F231AF600D841544A93F7F7EF5B
:100E40002183058BA182F98EA206DD8E231AD6009E
:100E5000DC41584AA583858B25837D8F93179700A6
:100E600013F7F6DF5D8F231AE600D4415C4AA982AE
:100E7000858AA983F58F9396A7009377F7BFD58FBF
:100E8000231AF600D441584AAD82858A2D83758F86
:100E9000FD769386F67F2E07F58FD98F231AF600FD
:100EA0008347260103250408A18B6387071083C7A6
:100EB0002500A18B63820710E31405EA9305300532
:100EC0001305001097F0FD1FE780C0172320A4082A
:100ED000E30705EE7C54A30204000347190083C610
:100EE000170089EA45C38347540093E70701A3022B
:100EF000F40029A0A147A302F40075F72285EFF0C2
:100F0000EFDB6C5483C72501858B81CF1C5483C7CD
:100F100027008D8B99C78347640093E7170023034D
:100F2000F4008327040899C78347640093E7870088
:100F30002303F4008347540005476393E70C4146BD
:100F400081451305840097F0FD1FE78080344146FA
:100F500081451305840197F0FD1FE7808033C1456B
:100F60001305C403EF30AFB7032704089307000548
:100F700011E3C14703550400A301F4008145EF408C
:100F80008F90C5B303C72701118B19E703472900C9
:100F9000118B19E38547A1BF83C707001547834617
:100FA0000900B387E70237D703001307C79ABA9738
:100FB000B69783C7070025BF19C597F0FD1FE780C7
:100FC000A016232004087C5403C7170011C7034749
:100FD000190019C3E14721BF03C72701118B09E796
:100FE00003472900118B5DD783C707001547834648
:100FF0000900B387E70237D703001307079945BFF6
:1010000013F7870131CFC18B130584004146A9C373
:10101000890597F0FD1FE780A02041468145130513
:10102000840197F0FD1FE780C02683476400C14517
:101030001305C40393E747002303F400EF302FAAFE
:101040008327040881CF93072005A301F40011BB77
:10105000814597F0FD1FE780C023C1B7CD47F5B7A5
:10106000094789456386E70011476398E70085458E
:1010700003550400EF402F8121A01947E389E7FEC3
:101080008347640093E747002303F40083270408A1
:1010900081C79307100555BFC54745BF4146CA855F
:1010A0001305C40497F0FD1FE780801783473400C1
:1010B00013076005639CE700B727002003C537D7F7
:1010C0008545EF10CF879307500541B745476383A8
:1010D000E7029306C4021306C40393058400228525
:1010E000EFD01FA72285EFF06FC0AA8411C1A144E1
:1010F000D147A1BFC94791BF9309C4054E85414659
:10110000CA8597F0FD1FE780A0110325040861CD73
:1011100083473400130790056398E7002285EFF0BA
:101120002FC09307E00515B71307A005639EE706D8
:10113000B727002083A7C7B3E38107C403A88700AC
:10114000E30D08C283477400930505084E8613D744
:1011500037002297834687009D8B0A87B3D6F640D7
:10116000858A93E6060813050504029841468A8598
:101170001305C40497F0FD1FE780C01711E1D28466
:101180002285EFF0EFB983477400CD461307E005E1
:10119000850793F7F70FA303F40063E4F600130742
:1011A0006005A301E40075BE1307C005E39BE7BA21
:1011B000B727002083A7C7B3E38107BC9C47E38E12
:1011C00007BA93050508130984000A8781464A86F1
:1011D0002E858297035504000A86CA85EF309FF357
:1011E0009307B0059DB58A864E86930584002285B7
:1011F000EFD01F9641469305C4040A8597F0FD1F62
:10120000E780400F8547D284E31DF5B42285EFF0D7
:101210002FB1AA84E31605B4930710023DB5034726
:10122000340093077002E31AF7B47C5889EB9305F6
:101230003005714597F0FD1FE780C0E068D8685819
:10124000E30D05B2CA85414697F0FD1FE78040FDDA
:10125000032944072285EFD0FF9A230DA9009307A5
:101260008002E5B30347340093078002E317F7B029
:101270008357060068582146930529002318F50076
:10128000490597F0FD1FE780A0F97C5483D74701FB
:1012900013F7072025CF185403574700137707206B
:1012A00035C79307900255B3034734009307900264
:1012B000E315F7AC3C5C89EB930530055D4597F091
:1012C000FD1FE78020D828DC285CE30805AA4146FA
:1012D000CA8597F0FD1FE780A0F49307A002B5B37D
:1012E000034734009307A002E319F7A883470600D9
:1012F000285C194693051900230BF500410597F06A
:10130000FD1FE780E0F17C5483D7470193F7074046
:10131000B1C71C5483D7470093F70740A1C3930775
:10132000B00225B3034734009307B002E317F7A4D4
:101330007C5C89EB93053005514597F0FD1FE780F4
:1013400060D068DC685CE30D05A04146CA8597F073
:10135000FD1FE780E0EC7C5C7D5798CB03D529002E
:101360008145EFD04FCAF5BA034734009307F00424
:10137000E3F8E79E03250408E304059E1306000432
:10138000CA851305050497F0FD1FE78060E92285F3
:10139000EFF04F9CAA842285EFD0CFF7834734002B
:1013A00013070005639FE700B727002003D6E90075
:1013B00003C537D785450606EF005FF7930730056D
:1013C00069B1130710056395E70093076005B5B988
:1013D00013072005E397E7989307C005BDB10347BE
:1013E00034009307E005E31DF79603250408414602
:1013F000CA8597F0FD1FE780A0E22285EFF0AF9B42
:10140000AA8419BD83450600A9BF85478144E39A94
:10141000F594032846008347360003472600834699
:10142000160083552500034606000145EF308FC99D
:101430000DBA8147C1463307F500B388F50003476D
:10144000070083C808003308F600850733471701F3
:101450002300E800E391D7FE82800147BD471308CF
:10146000F00F3306F50083460600B388F500FD173C
:101470008606558F2380E8000347060093F7F70F91
:101480001D83E39007FF82808147930800F841485D
:1014900093F6F70F3387F50063FCC600B306F5003B
:1014A00083C606002300D7008507E39307FF8280E9
:1014B0006395C60023001701C5BF23000700EDB7E1
:1014C00001114AC856C22E89AA8A930530054145A2
:1014D00006CE22CC26CA4EC652C4328A97F0FD1FD1
:1014E000E78040B6AA8493053005414597F0FD1F7B
:1014F000E78040B52A84CD49A5C431CD4146814518
:1015000097F0FD1FE780E0D82686A2855685EF007C
:10151000615AAA8929E18387040063D30706A2855B
:101520002685EFF09FF3B7D503004A869385C5A2C1
:101530002285EFF01FF08307090063D80704A28516
:101540004A85EFF09FF1B7D5030052869385C5A277
:101550002285EFF01FEE268597F0FD1FE780C0BCC7
:1015600011C4228597F0FD1FE78000BCF240624461
:101570004E85D2444249B249224A924A056182804C
:10158000CA852685EFF07FED7DB7D2854A85EFF0DD
:10159000DFECD1B781474146B306F5003387F5004C
:1015A0000347070003C80600850733470701238068
:1015B000E600E393C7FE8280011126CA4EC6AE84C0
:1015C000AA8993053005130500034AC806CE22CC2C
:1015D000328997F0FD1FE780E0A62DC513060003B2
:1015E00081452A8497F0FD1FE780A0CA4146CE8539
:1015F000228597F0FD1FE780C0D4A6850D46130510
:10160000D40197F0FD1FE780C0D3130604029305B1
:1016100004012285EF00014AAA840D469305D402F5
:101620004A8597F0FD1FE780C0D1228597F0FD1F06
:10163000E78080AFF240624426854249D244B249F5
:1016400005618280CD44FDB75D714EDE62D4AE8906
:101650002A8C9305300513050003A6C2CAC052DCCC
:1016600056DA5AD85ED686C6A2C4B28B368BBA84F6
:10167000BE8A4289468A97F0FD1FE780A09C6305D9
:1016800005101306000381452A8497F0FD1FE780AB
:1016900040C04146E285228597F0FD1FE78060CA81
:1016A000414681450A8597F0FD1FE78080BE1D46B3
:1016B000DE850A8597F0FD1FE780A0C81D46DA8504
:1016C0001305710097F0FD1FE780A0C73339200193
:1016D000B334900041468145080823072101A30740
:1016E000910097F0FD1FE780C0BA1946D6854808DB
:1016F00097F0FD1FE780E0C41946D2851305A101CC
:1017000097F0FD1FE780E0C3930404014146CE85B6
:10171000268597F0FD1FE780C0C28A852685EFF0F9
:101720007FE7930904024E86A6852285EF00813863
:101730002A890DE94146CE85268597F0FD1FE78071
:1017400020AE0C082685EFF0FFE44E86A6852285A4
:10175000EF0041362A8946454146CE8597F0FD1F68
:10176000E78020BE228597F0FD1FE780E09BB64012
:1017700026444A8596440649F259625AD25A425B37
:10178000B25B225C616182804D49D5B7011126CAE6
:1017900052C4AA842E8A13050003930530054AC853
:1017A0004EC606CE22CC3289B68997F0FD1FE7805F
:1017B000608935C52A84A685414697F0FD1FE780DC
:1017C00040B8930404012146D285268597F0FD1F79
:1017D000E78020B7CA8521461305840197F0FD1FD5
:1017E000E78020B613090402A6854A862285EF0009
:1017F000612CAA844146CA854E8597F0FD1FE7807B
:1018000040B4228597F0FD1FE7800092F2406244C9
:1018100026854249D244B249224A05618280CD449C
:10182000F5B739715AD05ECE2A8BAE8B4145930500
:10183000300506DE26DA52D456D262CC66CA6AC8B1
:10184000368C328DBA8C22DC4AD84ED697E0FD1FFA
:10185000E780407FAA8A93053005414597E0FD1F48
:10186000E780407E2A8ACD44638E0A0859C52A86BD
:10187000D6855A85EFF0DFC4AA8441E1930530058F
:10188000414597E0FD1FE780E07B2A8993053005FD
:10189000414597E0FD1FE780E07AAA89630A090EB7
:1018A0006306050E1304FD0011841376FD0049C084
:1018B0007D144204418035EE131544004E86D685D2
:1018C0005E95EFF01FB7414681454A8597F0FD1FB1
:1018D000E780209C014D93170D01C18363F48708B5
:1018E000BDC04A8597F0FD1FE7800084638709002B
:1018F0004E8597F0FD1FE7802083568597F0FD1FEA
:10190000E780808263070A00528597F0FD1FE78019
:10191000A081F250625426854259D254B259225ABB
:10192000925A025BF24B624CD24C424D2161828052
:101930000144131544008A855E95EFF0FFB44E868E
:10194000D2850A85BDBF93154D000A86DE954A856E
:10195000EFF03FAE4A868A855A85EF00A115AA842A
:10196000050D95BFBDFC0A86CE854A85EFF07FAC9C
:101970004A868A855A85EF00E113AA846686CA855D
:10198000628597F0FD1FE780A089A1BFCD4491BF7C
:10199000CD44A9BF397162CC2A8C594526DA4AD880
:1019A0004ED652D456D25AD05ECE06DE22DCAE8B54
:1019B000328BB68A3AC63E8AC2894689834401047C
:1019C000EF000FAE49C19167938717E92310F50027
:1019D00085472301F5002A8432472105630C0C0456
:1019E00093071003A301F4001946814597F0FD1FEA
:1019F000E780208A23036401A3035401230A94008F
:101A000023127401231744012318340123192401DC
:101A1000A285B72700206254F250D2544259B259DD
:101A2000225A925A025BF24B624C03C507D72161DE
:101A30006F000FB6A30104001946BA8597E0FD1F99
:101A4000E780007E45BFF2506254D2544259B259E9
:101A5000225A925A025BF24B624C21618280797168
:101A600056CAAA8A1305100326D24AD04ECE52CCAB
:101A700006D622D42EC6328AB684BA893E89EF00B1
:101A80002FA22DC1B24537460201930785001306E8
:101A900016E92A845CC110C123045501A304B500D2
:101AA0001946D285290597E0FD1FE7806077CE852E
:101AB0002308940013051401268697E0FD1FE78094
:101AC000207623082403A285B72700202254B25091
:101AD00092540259F249624AD24A03C507D7456176
:101AE0006F000FABB250225492540259F249624A2D
:101AF000D24A45618280011122CC2A84314506CE2A
:101B00002EC632C436C23AC0EF008F9929C1916700
:101B1000938717E92310F500B24522469246024703
:101B20008D472301F500A30185006244B7270020FB
:101B30002312B5002313C5002314D5002315E50097
:101B4000F240AA8503C507D705616F006FA4F24074
:101B500062440561828001114AC82A89394526CA32
:101B600006CE22CC2EC6B284EF008F9331C1B2458F
:101B70009167938727E92310F50091472301F5002A
:101B8000A30125012312B5002A84A6851905214643
:101B900097E0FD1FE780C068A285B7270020624458
:101BA000F240D244424903C507D705616F004F9EFA
:101BB000F2406244D24442490561828001114AC820
:101BC0002A89414526CA06CE22CC2EC6B284EF0011
:101BD0002F8D29C19167B245938727E92310F5001E
:101BE00095472A842301F500231225012146190572
:101BF00097E0FD1FE780C062A28523179400B727F6
